:020000040000FA
:1000000021EF01F01200FFFF10EF04F01200FFFFDC
:100010000000909400000000909000000000908686
:10002000016A1E0E015C32E20150EA6A000FE96EBD
:10003000060EEA22EF50046E909204B090829084F3
:100040009094909204B2908290849094909204B490
:10005000908290849094909204B690829084909430
:10006000909204B8908290849094909204BA908276
:1000700090849094909204BC9082908490949092FA
:1000800004BE908290849094012ACBD79092000075
:100090000000000090961200000090800000000018
:1000A0009086010E016E100E015C0DE000500114EF
:1000B00002E0908201D09092000090840000909421
:1000C000019E0146F0D7909200000000909600003B
:1000D0000000909012000000016A1E0E015C09E20F
:1000E0000150EA6A000FE96E060EEA22EF68012A63
:1000F000F4D712000000016A1E0E015C09E20150F3
:10010000EA6A000FE96E060EEA22EF6A012AF4D7C6
:10011000120000000068C0DF0168010606E00A0E58
:10012000026E020601E0FDD7F8D7550E006EB4DF6F
:10013000E1DF12000000EDDF06010F6B0601106B1E
:100140000601390E116F0601080E126F0601136BBE
:100150000601A80E146F0601156B0601166B060149
:10016000900E176F0601800E186F06010A0E196FA8
:100170000601810E1A6F0601BA0E1B6F0601200ED2
:100180001C6F06010A0E1D6F43DF12000000810E76
:10019000C96E37D8FC0EC96E34D88E8E00000000B0
:1001A000000000008E9E120009014E6B09014A07F3
:1001B000000E4B5B09014D5109014C5D01E0C96A1C
:1001C0004E2FFED709014D5109014C5D02E04CC98B
:1001D000C9FF4E2FFED78E8E8E8E8E9E4CC94DF946
:1001E000120000000900F5CF49F90900F5CF48F9E0
:1001F00009014851090146270901495109014723CD
:10020000120000000901486B496B0901540E485D5A
:100210003D0E495905E20901482B000E4923F5D747
:1002200012000000210EC26EC09EC2820000C2B247
:10023000FED7C4504D0802E2010E02D0000E00D0DD
:100240001200C16A210EC26E896A300E8A6E030ED8
:100250008B6E700E8C6E320E8D6E040E8E6E8F6AEB
:10026000800E906E916A92680F0E936E900E946E4F
:10027000956A9D0E966E7B0E976E070E986E300EE9
:10028000996E9A688D8CC79EC698C78CF00EC6165C
:10029000C680C68A240EAC6E190EAF6E900EAB6E81
:1002A00075DF0901516BBDDF000904E10A0E090188
:1002B000515D09E2640E0901515D05E2A2DFA1DF93
:1002C0000901512BF0D709015151630802E289EF6E
:1002D00001F00901466B476BF66A080EF76EF86A83
:1002E00080DF000009014851491102E102EF04F0EA
:1002F00078DF800EF61805E1FD0EF71802E1010E19
:10030000F81801E0F5D709014651471102E102EF63
:1003100004F001D8120000000DDF09014C6B090147
:100320004BA703D00901010E4C6F3EDF9EAA29D0D6
:10033000ABA209D0AB980000000000000000000054
:100340000000AB881ED0AECF4FF9ACA2FED7490E4D
:1003500009014F5D0BE14B0EAD6EACA2FED7330E23
:10036000AD6EACA2FED7410EAD6E06D0FF0E0901F8
:100370004F5D02E04FC9ADFF440E09014F5D01E141
:1003800001D0CBD709014A6B4B6B0901020E4C6FB0
:1003900009014AA902D009014C6B06DF2FD8020ED1
:1003A000F85C05E1420EAD6EF86A0ED8FF000CD87D
:1003B000410EAD6EEAD712000000550EA76EAA0ED0
:1003C000A76EA68200001200940EA66EF5DF000E46
:1003D000E96E090EEA6E0A000901080E446F090170
:1003E000080E456FEE50F56E0F00452FFBD7840EBB
:1003F000A66EE2DF442FF3D7A69412000000090195
:10040000506B0901446B440E0901445D1FE29EAA32
:10041000FED7ABA209D0AB9800000000000000009E
:1004200000000000AB8802D0AECF4FF90901445163
:10043000EA6A000FE96E090EEA224FC9EFFF0901CF
:100440004F51090150270901442BDDD709015051B3
:100450000BE1030E0901425D07E240C9F6FF41C905
:10046000F7FF42C9F8FF03D04E0EAD6EC8D7120099
:10047000FFFFFFFFFFFFFFFFFFFFFFFFFFFFFFFF8C
:10048000FFFFFFFFFFFFFFFFFFFFFFFFFFFFFFFF7C
:10049000FFFFFFFFFFFFFFFFFFFFFFFFFFFFFFFF6C
:1004A000FFFFFFFFFFFFFFFFFFFFFFFFFFFFFFFF5C
:1008000000001200280EE66E21ECFDF0E552D5EF57
:10081000FCF01200FFFFFFFFFFFFFFFFFFFFFFFFE6
:10082000FAEF2AF01200FFFFFFFFFFFFFFFFFFFFBD
:100830000000D9ECE4F0E20E4A6EEE0E4B6E010EB3
:1008400075EFEFF0D9ECE4F0550E4A6EEF0E4B6EFB
:10085000010E75EFEFF0D9ECE4F0300E4C6EF00EB7
:100860004D6E010E4E6EFE0EDBCF4FF0506A516A98
:10087000D8904F36503651364C504F24F36E4D5071
:100880005020F46E4E505120D6ECEFF00900F5CF19
:100890004AF00800F5CF4BF0EDECF2F0DEEFE4F0BB
:1008A00041ECEFF0010EE66EFD0EDB500301A725D3
:1008B0004A6EFE0EDB50A8210001F6ECF3F0F1ECDD
:1008C000EDF0E4ECECF0DF50E552DEEFE4F069EC43
:1008D000EFF04B6A020F4A6E010E93ECEFF0DEEF81
:1008E000E4F0D9ECE4F0850E4A6EEE0E4B6E010E8C
:1008F00075EFEFF069ECEFF0D4ECF1F0FD0EDB50AA
:10090000BFECE5F0EF50DEEFE4F02FC1E6FFA3DF30
:10091000E5521200100E5FEFEBF0D9ECE4F0A50EFB
:100920004A6EEA0E4B6E010E75EFEFF069500EEC59
:10093000F4F0B3ECEFF0006E1200AEEFE9F00A0E47
:100940004A6E4B6A90EFF4F0D7ECEEF090EFF4F0D3
:10095000E80E4A6E030E4B6E90EFF4F0D7ECEEF01B
:100960004AC23EF04BC23FF089ECE5F03E50006ECB
:10097000120001012B51010B1CE07851200B19E0F2
:10098000E251010B16E0CA51080B13E0100E2C5D6A
:1009900010E22C5105080DE23C51100B0BE0E6EC87
:1009A000E8F008E0100E0101615D03E26151050805
:1009B00001E3000C010CECECEAF00EE00201BB518B
:1009C000100B0AE03450400B08E00101D751010B35
:1009D00003E0E6ECE8F001E1000C010CE66A6EECE5
:1009E0002EF0E5521200C60EE66EEC0EE66E010E1B
:1009F00065ECEBF0E5521200010E06EFE5F0020E99
:100A000006EFE5F0B2C2E6FFE50EEEEFE4F0E66ACF
:100A1000E50EEEEFE4F07DEC14F0000918E07DEC5B
:100A200014F0000914E0960E64ECE5F06CEC0FF0A5
:100A30002BB00DD07DEC14F0000909E07DEC14F032
:100A4000000905E0DB0E73ECE5F083EC0FF012001B
:100A50000101E151010B03E05751080B02E1000EC7
:100A600001D0010E000903E00201B9511200020198
:100A7000B5511200D9ECE4F00101E151010B07E09E
:100A80005751080B04E0FE0EDBCFB9F203D0FE0E87
:100A9000DBCFB5F2DEEFE4F002011881178B17818E
:100AA0000501BF0E3B6F12000301D2510201EF5D41
:100AB0000301D3510201F05913E3EF510301D45D57
:100AC0000201F0510301D5590BE3D2510201ED5D52
:100AD0000301D3510201EE5903E34DECECF008E2BF
:100AE000D2C3EFF2D3C3F0F2D2C3EDF2D3C3EEF22E
:100AF000120065ECEFF0FF0805E1F6ECE4F0090EFA
:100B0000A8ECE8F0F2ECF2F04A6E0A0E4A5C0BE355
:100B1000F6ECE4F00F0EEF14000990ECF3F0090E80
:100B200009ECF0F0EF8E120054ECE7F003E1040E54
:100B3000495D1200495112006BECEBF013941396CF
:100B4000198C049091EC55F001018F51400B09E193
:100B50004A51320806E2320E4A6FEAEC7FF0020197
:100B600017870C500EE101018FAD09D070ECEBF04E
:100B70000A01D76BE66A09EC91F0E5521200B1EC7C
:100B80004BF01200800E081406E02150010B03E127
:100B90000201315101E0000C010C800E081403E049
:100BA0002150010B01E0000C010C0C500AE1010185
:100BB0008F51400B06E03550400B03E12150800B74
:100BC00001E0000C010C0201010E4D6FE20E73EC0E
:100BD000E5F01E0E096E1200EBEFECF069ECEFF0A1
:100BE00004080FE0F1ECE5F00EE0FE0EDB500A0821
:100BF00008E0FE0EDB500D0804E0FE0EDB50090895
:100C000002E1010E01D0000EDEEFE4F00701C7079C
:100C1000C551C52BEA6A000FE96E0C0EEA22EF50AF
:100C200012000101E051100B03E00401BA510AE186
:100C3000420EE66E460EE66E4DECCCF0E552E55205
:100C40000101E0891200D9CFE6FFE1CFD9FFFE0E06
:100C5000DB50D80805E1300EF36EFE0EF3CFDBFF5C
:100C6000060EAB1406E0AB98000000000000AB8855
:100C70008ED1FE0EDB50100805E0FE0EDB50110891
:100C800001E02AD10201050E296FFE0EDB5011088A
:100C900037E1020134510DE12150800B0AE10501D9
:100CA00005013B51010B0AE1050105013B51400BD8
:100CB00005E1100EE66E85D9E55222D00501050149
:100CC0003B51400B02E00F0E01D0060EE66E79D9C3
:100CD000E552BFC1E6FF75D9E552C0C1E6FF71D943
:100CE000E552C1C1E6FF6DD9E5520A0E0101C2030A
:100CF000F3500101C325E66E64D9E55205013B912D
:100D00000401B0514A6E4B6AD8904B5004E6D30EA2
:100D10004A5C000E4B5801E3DED005013B5101E176
:100D2000DAD00201345101E0D6D02150800B01E02D
:100D3000D2D0049005013BA11AD001010101E0517C
:100D4000080B03E00401BA510DE1410EE66E460EB8
:100D5000E66E4DECCCF0E552E5520101E08705016D
:100D60003BB35FDF05013B9305013B91B4D0050127
:100D70003BA304D056DF05013B93ADD005013BA753
:100D800024D0440EE66E4D0EE66E4DECCCF0E552EE
:100D9000E5520480440EE66E4D0EE66E4DECCCF04E
:100DA000E552E552030E0C5C03E0030E7D5C08E1A6
:100DB000540EE66E440EE66E4DECCCF0E552E55274
:100DC00005013B9705013B8586D005013BA524D055
:100DD000570EE66E420EE66E4DECCCF0E552E55253
:100DE0000480570EE66E420EE66E4DECCCF0E552F6
:100DF000E552530EE66E490EE66E4DECCCF0E55230
:100E0000E552490EE66E460EE66E4DECCCF0E5522C
:100E1000E55205013B955FD005013BA90BD0410E82
:100E2000E66E500EE66E4DECCCF0E552E552050153
:100E30003B9951D005013BAB0BD0410EE66E520EF3
:100E4000E66E4DECCCF0E552E55205013B9B43D0FC
:100E500005013BAD13D04F0EE66E520EE66E4DEC23
:100E6000CCF0E552E552540EE66E520EE66E4DECB5
:100E7000CCF0E552E55205013B9D2DD005013BAF7D
:100E80002AD04E0EE66E4C0EE66E4DECCCF0E552DE
:100E9000E552560EE66E440EE66E4DECCCF0E55291
:100EA000E552420EE66E530EE66E4DECCCF0E55286
:100EB000E552570EE66E430EE66E4DECCCF0E55271
:100EC000E5524E0EE66E420EE66E4DECCCF0E5526B
:100ED000E55205013B9F5BD0200EF36EFE0EDBCF8B
:100EE000F4FFF350F45C04E3FE0EDB507E0807E2EF
:100EF000FE0EDBCFE6FF72DEE552000948E0FE0E93
:100F0000DB503B0804E0FE0EDB507C0802E10401EC
:100F1000B92B01010101E351800B0BE0FE0EDB5008
:100F20003B0807E17EC1E6FFBAEC0EF0E552010195
:100F3000E39FFE0EDB50210804E0FE0EDB5040086C
:100F40000AE13B0E0401BE5D04E07C0E0401BE5DBF
:100F500002E10401B92BFE0EDBCFBEF40401B15156
:100F6000EA6A000FE96E0B0EEA22FE0EDBCFEFFFFE
:100F70000401B12B0401B02B0401B05108E10401BC
:100F8000BE6BBEC4B9F4BEC4B1F4BEC4B2F4E55283
:100F9000E7CFD9FF1200ACA212000401B851EAEC6D
:100FA000EFF0006E0050E66E90ECFCF0E5523B0E68
:100FB000005C03E07C0E005C01E12A900401B82B88
:100FC0001200D9ECE4F0ACA2FED77FECE5F090EC97
:100FD000FCF0E552DEEFE4F088EC13F094EC13F053
:100FE000F29EF66A080EF76EF86A940EA66E550E1B
:100FF000A76EAA0EA76EA682000000EC00F01200F9
:101000000401B007B25188ECE8F0EF50006EB22B4B
:101010001200050E0C5C0AE12050020B07E10201F0
:10102000B451020B04E1B451010B01E1000C010CBD
:10103000040E0C5C04E10101CD51080B01E1000C30
:10104000010CC70E3FECF4F0320803E33050400BC4
:1010500009E0309C88EC13F094EC13F05AECB5F0F6
:10106000D9EC13F0120045ECEFF09C0EDE6E030E8F
:10107000DD6E0301A551A61127E0090EE66EFD0EF7
:10108000DB50090DF350A5254A6EF450A621F6EC6D
:10109000F3F09C0EE66E030EE66EE4ECECF0DFCFB0
:1010A000E9FFDF2A010EDBCFEAFF01E3DB2AEFCF06
:1010B00000F0EF5024E0FE0EDB5003E10FEC97F060
:1010C000EED73AEC97F0EBD7FE0EDB500BE1A3EC3A
:1010D00093F07C0EE66EF20EE66E010EE66E26ECE6
:1010E00097F00AD0AFEC93F0740EE66EF20EE66E57
:1010F000010EE66E4DEC97F0E552E552E552020E18
:10110000E15C02E2E16AE552E16EDEEFE4F00490B8
:1011100043ECF4F038E004800101DEAB34D0F6ECAF
:10112000E4F00492EF50010B01E00482F6ECF2F0DF
:10113000016E050EEB50026EEF50080B01E0010E40
:101140003DECF2F0FE0EEF14F31090ECF3F0070E0E
:10115000EB50E66E040E5AECF4F0080EEB50E66E1F
:10116000050E5AECF4F00450020B02E0EF8601D0B9
:10117000EF96F6ECE4F0070E01C0EBFFF6ECE4F0BE
:10118000080E02C0EBFF12000501005102012A11F6
:101190003D1107E11C50010B03E14A514B1101E1E4
:1011A000000C010CD9ECE4F00101DE9D0701108573
:1011B00070EC5EF07FECE5F034EC29F0E5520701CD
:1011C000109570EC5EF0080E64ECE5F0DEEFE4F0F4
:1011D00000000000000000008C98000000000000EB
:1011E0000000120000000000000000008C880000D9
:1011F000000000000000120051EC29F002016A6BAF
:101200006AC22AF23D6B4A514B1102E021949CD9EB
:1012100051EF80F00701EF51010B07E0030E0C5C6A
:1012200004E0050E0C5C01E0000C010C0101279D9F
:10123000010E0E6E27BF0E681200030E06ECE5F0DD
:10124000268E12004D0EF1EFE4F04E0EF1EFE4F0B9
:1012500001018F51010B08E0C8EC11F0000904E016
:1012600001013C51800B01E0000C010C040E06EC66
:10127000E5F03C0E096E1200268E050E06EFE5F035
:10128000D1ECF1F0D1ECF1F000010F6ED1ECF1F006
:10129000106E120047ECF4F088C1E6FFDD0EEEECB4
:1012A000E4F094C100F0DBECEEF005E1090E010181
:1012B0009603F350006E0050E66EDE0EEEECE4F0A6
:1012C00054EFEFF0D9ECE4F0490E8DECF1F00F5053
:1012D00010100BE0FE0EDB50EA6A900FE96E010E73
:1012E000EA220FC0EEFF10C0EDFFDEEFE4F025A80C
:1012F00006D0010E696E020EE66EE4DFE552696A01
:10130000E66AE0DFE5521200D9ECE4F0FE0EDB50B5
:10131000B3ECE5F0EF5010E1FE0EDBCF4AF0FD0E2E
:10132000DB50D8804A5408E3FE0EF6ECEDF0B3EC47
:10133000E5F0100EEF6EEAD7DEEFE4F0830E0A6EF2
:10134000FA0E9CECE5F000500F6E0FC010F00F6A23
:10135000FB0E4BECF4F0005091EFF1F00101CB519A
:10136000800B01E0010E76ECEBF03BC1EFFF1200C9
:101370000101CB51800B01E0010E76ECEBF0EFCFD9
:101380003BF13B51140804E2010E3B6F2CA63B6B72
:10139000E9EFC4F0D9ECE4F0B2ECECF002E1EBC719
:1013A000EAF7FE0EDB0402E1EAC7EBF7DEEFE4F05A
:1013B000695003E03450400B02E00C5012007D50A5
:1013C00012000C50DCECE5F055EFECF043C1E1F21B
:1013D00043C1E0F20C501FECF2F0400B03E00201BD
:1013E000040EE06F7D501FECF2F0400B03E00201B1
:1013F000040EE16F120041ECEFF02950010B29E1DE
:101400002A0E675C06E108507AECEAF001E14B50E5
:1014100020E00C0E675C0AE108504C6E4D6A810EAC
:101420004C1804E14D5002E16F5013E070ECB5F040
:10143000000909E01A50400B06E11850080B03E1BF
:101440002150100B06E0190E675C05E137ECE8F05F
:1014500002E1000E01D0010EDF6E2D50800B03E182
:101460002D50400B02E0010EDF6E2990DF50E55257
:10147000DEEFE4F01B9C248A1200010137AF05D097
:1014800004A002D01B8812001B8A120047ECF4F063
:10149000580EF1ECE4F01DBE02D0D6ECEBF054EFA8
:1014A000EFF0010137AF07D0060E12ECF1F0280E75
:1014B00064ECE5F0EBDF12000601980ED880B4551D
:1014C0003A0EB55509E20F50B45D0101D26F1050CC
:1014D0000601B559010108D0B4510F240101D26FA2
:1014E0000601B55110200101D36F12000101DFBFC9
:1014F00011D0160EF1ECE8F0050E436E446A4AC2B4
:101500003EF04BC23FF0EBECFCF03EC04AF23FC075
:101510004BF21200110EF1ECE8F0020E0F0B02017B
:1015200005E0D8904B334A33E806FBE112001AB4C9
:1015300004D0370E93ECF3F0000C010C970EFBEC8B
:10154000F2F0980E0AEFE5F00101E0931C921C9076
:101550001A9A14921FEC1EF002014A6B4B6B54DB7B
:101560009EEF0AF045ECEFF0580EDE6E050EDD6ED4
:10157000560E0F6E010E106E0101DFAF07D0A80EE0
:10158000DE6E030EDD6EEA0E0F6E106A0D044A6EFB
:101590004B6AE8ECF3F0A1ECEFF096ECF8F03CC00D
:1015A000D2F13DC0D3F101018BA706D0CFECE7F01B
:1015B000EE50D227EE50D323020EE15C02E2E16A44
:1015C000E552E16EDEEFE4F0320E64ECE5F09F0EE2
:1015D000DCEFF1F0D9ECE4F0F7DF2250800B08E00B
:1015E000350E675C05E10F681068410E06ECE5F00A
:1015F000049001018BB70480C5EC8EF000C70AF09F
:10160000FC0E016E10C000F0FDEC4CF0012A0FC082
:1016100000F0FDEC4CF00A6ADEEFE4F041ECEFF094
:10162000010EDF6E21AC06D0030EDF6E0101E083F8
:101630001FEC1EF0800E4FECF4F0980E0AECE5F073
:10164000D6C30FF0D7C310F0950E64ECF0F0E5525E
:10165000DEEFE4F0550EF1ECE4F01A801200540EC7
:10166000F1ECE4F01A90120041ECEFF0FBEC26F004
:10167000DF6EF0ECEAF007E01AA00ED0F0DFDF50EA
:101680000BE1006A07D01AB007D0E4DFDF5004E1B5
:10169000010E006E37EC91F0E552DEEFE4F001014F
:1016A00060B702D02CC161F12EECE7F0FBEFEDF05A
:1016B000AAECEAF005E02050020B02E163ECE6F050
:1016C0001200C9ECE8F009E02150800B06E13C5122
:1016D000100B03E02050080B01E1000C010CAAECF8
:1016E000EAF00EE02150800B0BE12050080B08E0DF
:1016F0003C51200B05E12E50400B02E1095001E066
:10170000000C010C8DECE5F003E03550400B04E0DB
:1017100001015851040B01E1000C010C41ECEFF008
:1017200001018BA10AD0FBEC26F0DF6EDF0403E0A1
:10173000020EDF5C02E1010E01D0000EE552DEEF89
:10174000E4F0E3ECEEF005E1FBEC26F0040801E048
:10175000000C010CF6DF000904E1E7ECEEF001E01B
:10176000000C010C8150080B0DE08150010B0AE0C8
:101770008DECE5F003E0B6ECECF004E11A50020B5E
:1017800001E1000C010C8150080B19E08150020BA3
:1017900016E08150040B13E08150010B10E00501AD
:1017A00000510DE12150040B0AE12150010B07E12A
:1017B0008DECE5F003E0B6ECECF001E1000C010C7F
:1017C000810EEAECE8F0010137BF268E120010C24C
:1017D000E6FF0FC2E6FFC80E0AEFE5F01E9C076A9F
:1017E000796A33DDEA0EEAECE8F0268E120069EC45
:1017F000EFF00A0DF3CF5AF3F4CF5BF3000E0301C1
:101800005A27030E5B23DEEFE4F00F0E07010E13E1
:101810000E990E9F040E0101445D02E107010E8F37
:10182000100E01012C5D14E2020E815D25E22C51A7
:1018300002E107010E9101012C0502E107010E935F
:1018400001012C51020818E22C1D07010E1714D0BB
:10185000815112E0100E2C5D19ECE8F08BC200F003
:101860000A0E005C01E1006A001C07010E17A8ECDB
:10187000F4F0020B01E10E89049007010EB7048019
:101880000E970EB30E870E9304B00E831200CAECAF
:10189000F0F004E68A0E4A5C000E4B5802E2E0EFDC
:1018A0000BF0CAECF0F004E6A90E4A5C000E4B58AF
:1018B00004E20201E051795E1200CAECF0F002E6A7
:1018C000FFECEDF003E20201E05179261200140E64
:1018D00033ECE7F0B0ECEFF000501C0806E31450D6
:1018E000100B04E000500C0801E2010C000CC9ECE4
:1018F000E8F003E1D951100B07E18B51400B03E0F5
:10190000D951040B01E1000C010CE6ECE8F002E017
:10191000060E01D0070E06EFE5F069CFC7F2696A3F
:1019200079C101F07AC102F0AEECEAF004E20701FD
:101930000551026E016E01900142029002424D0E6D
:10194000012444ECF2F0010E696E4D0E022444ECC9
:10195000F2F0C7C269FF120007010E9B0101CCAB78
:1019600002D007010E8B12A007D007010E9B0101C8
:10197000CCAD02D007010E8B1200695006E0345046
:10198000400B03E10201B15112000101E2A903D0B1
:101990000201B05112000A01D55112000201630E7A
:1019A000C36F010EC46F695004E05D0EC36F010E7A
:1019B000C46F120095ECF1F00FC1DFFF010E10C1F2
:1019C000DBFF34AC05D0DB50DF6E010E0FC1DBFF57
:1019D0003EECE6F0C9ECE8F037E107011051200BCE
:1019E00033E01051010B07E0DF500A0804E2010E5A
:1019F000DB500A0829E3010EDB50DF5C25E00A0E0C
:101A0000DF5C22E0DF50070804E20A0E15ECE5F087
:101A10001BE3DF50050804E2080E15ECE5F014E3C3
:101A2000DF50030804E2060E15ECE5F00DE3DF508D
:101A3000010804E2040E15ECE5F006E3DF0406E11C
:101A4000020E15ECE5F002E2020EDB6A020EDB503C
:101A500007E0080E06ECE5F0FA0E096E19861C8800
:101A6000030EE15C02E2E16AE552E16EDEEFE4F0D2
:101A700007010797E6ECE8F006E049ECE9F003E03F
:101A80000701078797DFF4EFEAF0D9ECE4F02BA425
:101A900009D0C6ECEAF064EC2EF0CBECF3F0500E7B
:101AA000096E2B94DEEFE4F0159E0A01DA51800BEB
:101AB00006E1050E0C5C03E082ECE6F001E0158E19
:101AC00012000C50080D38ECE7F0010EEBECEEF0D4
:101AD000E806FCE10250080D4C50F3244A6E4D50CC
:101AE000F4204A50016E12000A01DA8FDDDF020194
:101AF0009651D5ECE5F01AE24A509608000E4B5488
:101B000015E20268950501E1026A030E955D02E1A6
:101B1000010E026EFF0E025C10E0F1ECECF09AECAC
:101B2000F1F0015032ECF0F00A6A07D05DECE9F018
:101B300039ECECF0178B05013B850201956B188E93
:101B4000500E096E2596328C12000201C669C6C27B
:101B5000C5F2C6C2BCF7C6C2BBF7C6C2BAF7C6C298
:101B6000B9F7C6C2B8F7C6C2B7F70701C369C469F7
:101B7000C169C269C1C7BFF7C2C7C0F7C1C7BDF756
:101B8000C2C7BEF712000101470503E18450100BE4
:101B900007E0020E475D03E18450100B01E1000CE9
:101BA000010C96880101475101E19698120041EC21
:101BB000EFF00101A45103E19A51200821E2DF6A0C
:101BC000090EDF5C10E2DF5009ECE6F0EF50040B89
:101BD00008E0100EDF24E66E07EC35F0E552000950
:101BE00002E1DF2AEDD7090EDF5C0AE2100EDF26E4
:101BF0002A86DFCFE6FFC6EC34F0E552DF5001D095
:101C0000000EE552DEEFE4F02086076A796A189844
:101C1000189A2682248A1200010138BB02D08C9ABD
:101C200001D08C9C000000000050E66E13EC7AF0AE
:101C3000E5520000C950006E00008C8C8C8A030EA7
:101C4000E66E3DECFDF0E55212002C880701108194
:101C5000108D10990101E0A502D00701108907013C
:101C6000129712002C9807011091109D109912875D
:101C7000120020EC7AF0F00EC616C680C68A12005A
:101C8000800EE66EE66A010EE66EE2ECFAF0CBEC50
:101C9000F3F039EF0EF01382138006011091020168
:101CA0001E0E406F1200139020A21380139220B2D8
:101CB000138212001DECF4F01FECF2F0EFECEEF0EA
:101CC000DF6E000EDF94DF96DF98DF9ADF9CDF9EE9
:101CD0000A0E006EFE0EDB5009E1030EDF5C02E22D
:101CE000050E006EDF5043E1010E40D0FE0EDB50CA
:101CF000030804E1DF5002E1010E006EFE0EDB502E
:101D000004080EE1DF0402E1320E006E020EDF5C19
:101D100002E15A0E006E030EDF5C02E1640E006EFB
:101D2000FE0EDB50050810E1320E006EDF0402E10A
:101D3000640E006E020EDF5C02E17D0E006E030E8B
:101D4000DF5C02E1FA0E006EFE0EDB0403E0B2EC93
:101D5000ECF00DE1DF5002E1010E006EDF0402E164
:101D6000050E006E030EDF5C02E1190E006EE552F7
:101D7000DEEFE4F0D9ECE4F0F00E07010F17FE0EF1
:101D8000DB50320F97ECE5F007010F1399EC5EF092
:101D9000DEEFE4F06950E3ECF1F0B3ECEFF0050DA9
:101DA000F350006E6AECE8F0EF50200B02E0050EF5
:101DB00000260701BB51005C07E000C0BBF70050E4
:101DC000E66EAE0EEEECE4F01200139A20B2138A27
:101DD0006ADFB1EC4BF0E4EC1CF02050020B05E0A4
:101DE0007D500C5C02E01B8C12001BAC02D03AEC64
:101DF0000AF01200D9ECE4F02050020B06E007ECE8
:101E0000B9F0000902E120922ED02050020B08E028
:101E100082ECE6F005E098ECB8F0A0ECB8F0208297
:101E20002050020B06E0C9ECE8F003E0139E3C935F
:101E3000CA99FE0EDB5004E120B204803DEC0AF0AA
:101E4000C4DF050E0C5C08E12050020B05E0020126
:101E5000B493B49169EC38F0A9ECB8F0FE0EDB5005
:101E600002E102011783DEEFE4F041ECEFF0CFC1B5
:101E7000DFFF54ECE7F002E1040EDF265CECE6F055
:101E800003E00D0EDF5C11E35CECE6F00CE154ECDA
:101E9000E7F003E0140ECF5D08E30A0E2C5D03E1CA
:101EA0000A0ECF5D02E3000E01D0010EE552DEEF17
:101EB000E4F00A6A700EE66E290EE66E010EE66E1A
:101EC000E66A39EFE5F07E0E0A6E0F0EE66EED0E55
:101ED000E66E020E4DEFF1F0F00E8C16FDECF3F015
:101EE00011E25CECE6F00EE02B50010B0BE1320E40
:101EF00064ECE5F0FDECF3F005E22B807B0E77EC73
:101F0000E5F001D812000101320E496FACECE8F0A7
:101F10007EEF28F00701875106E14C0E3DECE7F01B
:101F20000501141501E1000C010C2D9E2D9C69EC9E
:101F300038F0D8EFB5F007011D891D975CECE6F08D
:101F400009E001012C0506E16051400B03E10701A6
:101F50001D991D871200D9ECE4F002ECEEF007E1C8
:101F60002C50010B04E101018B51200B09E155C2FA
:101F700058F254C257F253C256F2F8ECECF009D0C2
:101F8000FE0EDB5006E058C255F257C254F256C25C
:101F900053F2198C04802CA002D004902C9091EC68
:101FA00055F0320E096EDEEFE4F0006A01013A519D
:101FB000060802E2DDC700F000AE02D007011CD027
:101FC0002BA002D007013ED00701DF5106E10050EF
:101FD000240825E3E05140E022D0DF050FE1005066
:101FE000290803E3E051010802E2020EDF6F230E2D
:101FF000005C32E2E05130E1DF6B2ED0020EDF5D9B
:1020000010E10050310803E3E051020802E2030E40
:10201000DF6F280E005C20E2020EE05D1DE2010E83
:102020001AD0030EDF5D10E10050360803E3E051E3
:10203000030802E2040EDF6F300E005C0DE2030EB7
:10204000E05D0AE2020E07D0350E005C05E2040EE8
:10205000E05D02E2030EDF6F070E1315006EF80E4F
:102060001317DF0501E11385020EDF5D01E1138324
:10207000030EDF5D02E113851383040EDF5D01E1D2
:102080001381070E1315005C08E0050EDBECEBF086
:102090002D907EEC5EF0F00E8C161200D9ECE4F080
:1020A00021B814D0FE0EDB5015ECF1F0016EFE0EDF
:1020B000DB50040F15ECF1F0026EFF0E015C08E13D
:1020C000FF0E025C05E1199A17B8198A000E09D0B3
:1020D0000150006E17A802D00250006EE1EC9AF099
:1020E000010EDEEFE4F00301916B926B936B946B46
:1020F00091C38DF392C38EF393C38FF394C390F384
:10210000030E016EFF0E015C32E0056A030E026EE3
:10211000FF0E025C22E00250EA6A890FE96E030EAC
:10212000EA22EF504C6E4D6A0150EA6A850FE96E63
:10213000030EEA22EF50F5ECE5F00AECEBF0EF507D
:1021400091ECF1F0055091ECF1F00AECEBF00FC0DE
:10215000EFFF10C005F00206DBD70150EA6A8D0FD1
:10216000E96E030EEA2205C0EFFF0106CBD712008D
:1021700000AE04D0006C01010E0E146F63ECE9F0A8
:10218000010115510AE114C115F1100E146F165119
:1021900004E115C116F1100E156F130E186F120021
:1021A00095ECF1F069507CECEBF0EFCFDFFF010E26
:1021B000BFC1DBFF020EC0C1DBFF010178B738D021
:1021C000695006E0010EC4C1DBFF020EC5C1DBFF92
:1021D000DFCFE6FF19EC04F0E552E66E33ECEAF0EF
:1021E000E8ECE5F00B0EDF2497ECE5F0E66E6950C5
:1021F000EA6AE60FE96E020EEA22E8ECE5F0DF504B
:1022000011E13AECEAF0010EEF6EDB0404E1500E4E
:1022100071ECE8F007E233ECEAF0020EEF6E3AEC14
:10222000EAF0EF6A33ECEAF0EF50E66E67ECE9F0C3
:10223000030EE15C02E2E16AE552E16EDEEFE4F0FA
:1022400045ECEFF0BFC1DFFF010EC0C1DBFF0101B4
:1022500078B71ED0695005E0C4C1DFFF010EC5C1CB
:10226000DBFF69507CECEBF0EF5012E13AECEAF066
:10227000EF5007E0DF040BE1500E15ECE5F008E24B
:1022800006D0DF0405E1010EDB504F0801E288DFD4
:10229000020EE15C02E2E16AE552E16EDEEFE4F09B
:1022A000030E0C5C03E1030E785C01E0000C010CF2
:1022B000030E0C5C05E1020E785C03E0780401E09B
:1022C000000C010C030E0C5C03E1020E785C01E0D3
:1022D000000C010C030E0C5C08E1785006E10101D2
:1022E000CA51040B01E0020C010C000C030E0C5C43
:1022F0000DE1020E785C04E101013D51010B07E1A3
:10230000780404E101013D51020B01E1000C010CD4
:102310000601F25106E0030E0C5C03E17850000860
:1023200001E3000C010C030E0C5C04E1780403E0F3
:10233000785001E0000C010C030E0C5C06E1020E6B
:10234000785C04E0030E785C01E0000C010C0101F4
:102350003D51080B03E0030E0C5C09E03D51040BFA
:1023600005E00C0404E0020E0C5C01E0000C010C22
:10237000CEEC0CF0ECECE5F0EF9CF8ECEAF007E0CA
:10238000ECECE5F0EF8C0701E26B56C1D5FA1200D8
:102390008DECE5F003E0FCECEAF001E1000C010C4F
:1023A0000C5004E10A01DA51040B01E1000C010CAC
:1023B0000C5003E1F3ECEEF001E1000C010CBAEC7F
:1023C000ECF00CE0CDECE8F009E00301D851ACEC06
:1023D000F4F032ECE9F0E80E0AECE5F01200AFECB4
:1023E000F4F00C5005E1F3ECEEF002E0020EDF6ECB
:1023F000010178B9DF84DFCFE6FFEB0EEEECE4F00D
:102400000C5004E10A01DAB7DA95D9DFE552DEEFC4
:10241000E4F0030E0C5C11E10101CB51040B05E06B
:1024200078040CE0020E785C09E0CA51040B05E068
:10243000785004E0030E785C01E0000C010C0C50B5
:1024400003E1B2ECEAF004E1F7ECEEF001E1000C9C
:10245000010C9EECE9F001E0040C4DECE9F001E028
:10246000080C040E0C5C01E11B0C0C5009E0030E7F
:102470000C5C05E1785004E0030E785C01E0030C8D
:10248000010C9EECE9F001E00A0C4DECE9F001E0F2
:10249000380C040E0C5C01E1640C0C5001E0500C93
:1024A000380CEFDFE66ED5DFE66ED60EE66E0A0E6E
:1024B00000EFE5F037EC56F0190E01240A01D88040
:1024C000D75503E2190E0124D76FBEECECF0D75DAF
:1024D00003E2BEECECF0D76FD46B3488DCEFEFF0A6
:1024E00082ECE6F00DE19EECE9F00AE14DECE9F05A
:1024F00007E1F8ECEAF004E13BECE8F001E1000C64
:10250000010C896A700E8A6E030E8B6E700E8C6ED3
:10251000320E8D6E040E8E6E8F6A800E906E916AF2
:1025200092688F0E936E900E946E956A9D0E966EC5
:102530007B0E976E070E986E300E996E9A68120099
:102540002098268A189A02012B5114E00701EF9B6C
:10255000EF9B33BCEF8BE1EC09F002012B6BF1C672
:1025600000F00C5002E0F3C600F00050E66EE20E00
:10257000EEECE4F02682120060ECF4F007ECEEF0F2
:1025800094ECF4F094ECF4F094ECF4F0C09EF00EC3
:102590008C16020E0F0B05E0D89010320F32E806B1
:1025A000FBE142ECE7F0030E23ECF2F0FDE14A50D0
:1025B0000F5E4B50105A2BAA0DD00A0E3E6E3F6A8A
:1025C000DBC743F0DCC744F096ECF8F03C500F2634
:1025D0003D501022AFEC93F0A8EC04F0300F010155
:1025E000196F0BECE9F001011A6F3A500F6E106A87
:1025F0009FEC04F0300F01011B6F300E3A241C6F6A
:10260000300E195D02E1200E196F1B8F410E1E6FF7
:102610001200D9ECE4F005010151EA6A000FE96EFD
:10262000080E00ECF3F0012B015153ECE5F002E64B
:102630000CECEEF001E3016B002BDEEFE4F0020E98
:102640001EEFE8F005EFF3F094928B9094908EEFEC
:10265000E8F08B9205ECF3F082B0FF0C000CEFDF9A
:10266000EEDF82A2FE0C000C0701080EC96F8B92F0
:1026700005ECF3F082B207D0F2DF000904E0FE0EB1
:10268000F36EF46812000701C89FC847C89182B072
:10269000C881C907EDE1C85111EFE9F0D9CFE6FFD4
:1026A000E1CFD9FF0701080EC96FFE0EDBCFC8F7D7
:1026B0008B9282B206D0D3DF000902E0FF0E17D062
:1026C00011D0C837D8A006D094929480B8DF9482F5
:1026D000B6DF06D094928B909490B1DF9482AFDFF6
:1026E0000701C9070701C951E4E1000E00D0E55216
:1026F000E7CFD9FF12008B9294928B9094908EEC3E
:10270000E8F094801FEF13F08B9094901FEF13F07C
:1027100078ECE6F059EC0FF023EC5FF063EC0FF08F
:102720002DEC5FF031EF9BF0E1EC18F0909C908E77
:1027300030EC2CF00101776B2FEC0BF077EC09F00B
:10274000020EE66EF50E82ECEBF046EC0AF00701A5
:10275000010E066F076B086B096B0A6B0B6B0C6B3A
:102760000D6BF00E0E170F6B106B116B126B600E72
:10277000136F146B156B166B186B18C717F71B6B61
:102780001C6B206B1D6B1E6B1F6B99EC5EF00601C2
:10279000526B52C650F6547113EC51F08A985AECB1
:1027A00098F09AEC97F00601556B55C654F60B6AF3
:1027B0001200F29E9D0E966E8D9CFCD7E6EC26F0E4
:1027C0000701F10504E14C0E005C06E203D05A0E4D
:1027D000005C02E2A9DFEDDF000C46EC0AF0E8EC59
:1027E00018F03488B1EF4BF08B8A010160B18B9AFD
:1027F000C69A8B96F00E8C1407098C6E96EC5EF0E0
:102800008A9AE8EC08F08B860000000000008B96A6
:102810000000F2EC08F000008A8AC68A12001A5002
:10282000800B01E0010E7CECEBF0EF50090801E2B7
:10283000000C010CF00E8C16050E8C12C08EB0EC44
:10284000EFF0C3CF4AF0C4CF4BF005ECE8F005EC55
:10285000E8F0C3CF4CF0C4CF4DF0060ED8904D3207
:102860004C32E804FBE14A504C240701DB6F4B502B
:102870004D20DC6FC09EF00E8C1612008F0ED9EC2E
:10288000E5F0030E0002F3CF0CF20050200801E344
:10289000000C010C0101DD51040B2EE037ECE8F0D7
:1028A0002BE02150200B28E03450400B25E1E6DFDF
:1028B000000922E00A0E64ECE5F0E0DF00091CE00C
:1028C000FA0E64ECE5F0DADF000916E0090E06EC1A
:1028D000E5F012AE04D0129E11ECEEF008D012BC5E
:1028E00006D0128C16ECEEF00201020EBC6F3BEC2F
:1028F00027F04EEC27F0258A1200F00E8C16070EFA
:102900008C12C08EB0ECEFF0C3CF4CF0C4CF4DF0C2
:10291000EBECEEF0EBECEEF04C50C3244A6E4D5075
:10292000C4204B6E4A50C3240F6E4B50C420106E0F
:10293000110E9FECF1F0C09EF00E8C1601015F515C
:102940004C6E4D6A3B0E4C26010E4D220F504C5CD6
:102950004A6E10504D584B6E4AC0DDF70701DD51ED
:1029600054080BE2DD5153ECE5F002E647ECE7F0EA
:1029700004E25CECE6F001E0010C000CC08E870E76
:10298000D9ECE5F007ECEEF0D8900F361036D89081
:102990000F361036E0ECEBF0C09ED9C74AF0DAC72C
:1029A0004BF0030E23ECF2F0FDE14A500701D95F32
:1029B0004B50DA5B0F50D9271050DA231200860EE5
:1029C000010164254C6E4D6A000E4D22D9C74EF0B0
:1029D000DAC74FF0600E436E446A4EC03EF04FC0FF
:1029E0003FF0EBECFCF03EC04EF03FC04FF04E50DD
:1029F0004C5C4A6E4F504D584B6E4A50006E120060
:102A000069ECEFF00EE1F00E0201131507010D6FF6
:102A10000F0E02011315006E0038F00B07010C6F4A
:102A20000DD0F00E020114150701096F0F0E0201FF
:102A30001415006E0038F00B0701086FDEEFE4F0AC
:102A4000C00E016E5CECE6F002E0B00E016E2CA848
:102A500002D0D00E016E01010F5101263CEF4DF066
:102A6000D9ECE4F0B2ECECF002E1FE0EDB066950CA
:102A7000060D43ECE5F0140E4A260A0E4B22FE0E1C
:102A8000DB5009ECF3F0DEEFE4F041ECEFF0A5EC05
:102A90000DF0050E0C5C06E10701E26B0A01D56B37
:102AA000DA931CD0A1ECE7F0EFCFE2F70C50DF6E29
:102AB000D5CA00F0C2ECECF0DF500DECF0F09AEC6F
:102AC000F1F09AECE7F0020E6F5C0CE19A0E0B5CF1
:102AD00009E30B509E0806E300C0D5FAE66AA8ECAD
:102AE00090F003D0DFCFE6FFBBDFE552695003E093
:102AF000D5CAB1F20BD082ECE6F008E00A01D76B40
:102B0000060150850A01DA81C4EC1EF0159C07010C
:102B1000E25101E0158CC30E060150170A01DAA13B
:102B200002D0140E01D0280E060150130A01DAA3B8
:102B300004D0D8CAE7F7D9CAE8F78AEC1EF00C50DF
:102B4000DCECE5F0EFCFEFF7ACEC25F0010EE66E34
:102B5000E66A73ECE6F07DEC95F036EC2CF0E6ECF2
:102B600009F0E552DEEFE4F0C2ECECF09AECF1F0A3
:102B70000C500DECF0F09AEFE7F00C50DCECE5F0C7
:102B800055ECECF0050E0C5C0CE00A01DAA306D063
:102B9000E7C7D8FAE8C7D9FA8AEC1EF0E5DF0EECF1
:102BA000F3F0120041ECEFF0DF6A080EDF5C05E2A3
:102BB00021ECE6F0EF68DF2AF8D7E552DEEFE4F02B
:102BC00041ECEFF0DF6A080EDF5C0CE221ECE6F08E
:102BD000EFCF4AF0FE0EDB504A5C02E1010E03D05B
:102BE000DF2AF1D7000EE552DEEFE4F041ECEFF022
:102BF0000301D95104E0DB2B030ED95D17E37FEC11
:102C0000E5F0DEDFE552000911E1DF6A080EDF5C66
:102C10000DE221ECE6F0EF50FF0806E121ECE6F0D2
:102C2000FE0EDBCFEFFF02D0DF2AF0D7E552DEEF5A
:102C3000E4F041ECEFF0DF6A080EDF5C0BE221EC20
:102C4000E6F0EF50FF0804E021ECE6F0EF5003D08F
:102C5000DF2AF2D7FF0EE552DEEFE4F045ECEFF0AD
:102C6000DF6A080EDF5C10E221ECE6F0010EEFCF28
:102C7000DBFFDB50FF0806E021ECE6F0EF68010E19
:102C8000DB5003D0DF2AEDD7000EB6ECEAF002E20B
:102C9000E16AE552E16E4A50DEEFE4F041ECEFF01C
:102CA000318ACFECF3F0D1ECF1F0D1ECF1F0DF6E42
:102CB000319ADF50E552DEEFE4F041ECEFF007012E
:102CC0008B6B8C6B2EA802D0010E2AD00C0E3DEC23
:102CD000E7F0DF6E07018B2B000E8C23DF5008E03E
:102CE000FF0EDF5C05E0580E8B5D020E8C59EEE3A3
:102CF0008B518D5D8C518E5904E28BC78DF78CC73B
:102D00008EF7580E8B5D020E8C5909E301018C5130
:102D100003E15A0E77ECE5F02E88000E01D0010E8B
:102D2000E552DEEFE4F0D9ECE4F0E1ECEFF0DEEFB9
:102D3000E4F053ECF1F003E2FBECEEF004D0FE0E15
:102D4000DB50F60F410FDEEFE4F0FFECEEF004E0B5
:102D500001013651E82402D001013651E66EC40E5D
:102D6000EEEFE4F041ECEFF0FBEC26F0DF6E0F0E3F
:102D7000E66EDF5007E0030EDF5C04E001018B51DB
:102D8000020B02E1000E01D0010E000905E00A0E5F
:102D900001017B03F35001D0000EE66ED90E0AEC60
:102DA000E5F0E552DEEFE4F065C18EF2FCECEAF00E
:102DB00002E166C18EF2006A02018EA302D0008891
:102DC00007D08E51010B04E08E51800B01E0008C86
:102DD00000507FECEAF002018EA502D05F0E05D014
:102DE0008EA702D04F0E01D05E0E006E0050F1ECA7
:102DF000E4F002018EB508D08E51400B02E04B0E7C
:102E000001D04A0EF1ECE4F007010F9D02018E5152
:102E1000020B05E08E51200B02E007010F8D060129
:102E20005295FFECEEF005E08E51100B02E006012A
:102E30005285258A1200FCECEAF003E18EC266F1AD
:102E400002D08EC265F1D4EF16F0D9ECE4F0325026
:102E5000080B35E10101DD51100B31E10601BA6BC0
:102E6000020EBB6F328601018C5129E1450E58ECF0
:102E7000E5F02A0E58ECE5F0440E58ECE5F0530E60
:102E800058ECE5F0450E58ECE5F0300E692458ECAE
:102E9000E5F03B0E58ECE5F05D0E77ECE5F0FE0E4C
:102EA000DBCF2CF789C72DF788C72EF7010139A989
:102EB00006D02A0E20ECEEF02A0E20ECEEF0DEEF2B
:102EC000E4F041ECEFF02E50100B06E13250100B05
:102ED00003E00701F10502E1000E17D001013951AD
:102EE000100B0AE03150200B07E1695002E0400E60
:102EF00001D0210E20ECEEF007018A6BFE0EDBCF35
:102F000088F77FECE5F019D8E552E552DEEFE4F002
:102F1000D9ECE4F00601B82B000EB923BA51B81968
:102F200009E1BB51B91906E17FECE5F08EDFE5520E
:102F3000010E01D0000EDEEFE4F0D9CFE6FFE1CFC5
:102F4000D9FF020EE1262E50100B03E10701F10517
:102F500002E1000E9AD0FE0EDBCF89F701010101DC
:102F60003951100B19E03150200B16E1FE0EDB3801
:102F70000F0BE66EDEDEE552E66ED5DEE552FE0EA6
:102F8000DB500F0BE66ED5DEE552E66ECCDEE55289
:102F90002E0EE66EC8DEE552695027E10601B86BD9
:102FA000B96B84B007D0E66AB3DFE552000901E0EF
:102FB00001D0F7D78C9A0000FE0EDBCFE6FF13ECB2
:102FC0007AF0E5520000C950DF6E00008C8A0601DD
:102FD000B86BB96B84A008D0010EE66E99DFE5529C
:102FE000000901E001D0F6D731D0010101013851CB
:102FF000080B05E101010101DD51100B27E006017D
:10300000B86BB96B86B008D0020EE66E81DFE55270
:10301000000901E001D0F6D78C9C0000FE0EDBCF4A
:10302000E6FF13EC7AF0E5520000C950DF6E0000B5
:103030008C8C0601B86BB96B86A008D0030EE66EC7
:1030400067DFE552000901E001D0F6D707018A5198
:1030500003E107018A2B14D007018A0511E107015A
:10306000881DDF5C0AE0695003E02550100B05E085
:10307000040E6924E66EE9DEE5520701020E8A6F4E
:10308000010EDFCFDBFFDF5000D04A6E020EE15CA5
:1030900002E2E16AE552E16E4A50E552E7CFD9FF1C
:1030A00012006DECEFF0DEEFE4F06DECEFF0FC0EF3
:1030B000A3ECF1F0DEEFE4F06DECEFF0FC0EA3EC2E
:1030C000F1F0FB0EA3ECF1F0DEEFE4F04CECEFF0EE
:1030D00001013CA904D0010E696ECFECF3F0696ADE
:1030E000CFECF3F054EFEFF04CECEFF001013CA922
:1030F00006D0010E696E7DECEFF013ECF3F0696A17
:103100007DECEFF013ECF3F054EFEFF04CECEFF05C
:1031100001013CA90BD0010E696E22ECF4F06EECBB
:10312000E6F0FA0EDBCFE6FF08DFE552696A22EC33
:10313000F4F06EECE6F0FA0EA3ECF1F054EFEFF0E1
:10314000D9ECE4F0CFECF3F0D2C1E6FF48ECE6F0C6
:10315000D3C1E6FF48ECE6F00FC0E6FF48ECE6F02E
:1031600010C0E6FF48ECE6F0DEEFE4F047ECF4F0E8
:1031700001013CA902D0010E696EF00E8DECF1F058
:1031800054EFEFF047ECF4F001013CA902D0010E3E
:10319000696EF10E8DECF1F054EFEFF0D9CFE6FF50
:1031A000E1CFD9FFFE0EDBCFE6FF13EC7AF0E5525C
:1031B00000008C8E000000008C9EE552E7CFD9FF06
:1031C00012002BB203D0740E4AECE7F02B821200EF
:1031D0002BA203D0760E4AECE7F02B9212002BB212
:1031E00003D0750E4AECE7F02B8212002BA203D01D
:1031F000770E4AECE7F02B921200D9ECE4F032B2F1
:1032000006D0790EF1ECE4F0FE0EDBCF2CF2DEEF0F
:10321000E4F0D9ECE4F002015ABF07D05DECE5F030
:103220005951EE265A51ED2208D0FF0E59154A6E1B
:103230007F0E5A154B6E4AECF2F0FC0EDBCFE6FF28
:1032400041ECEAF04A6E4B6A4ABE4B680A0E50ECFB
:10325000E8F04AECF2F0FB0EDB5069E001010B6B89
:103260000C6B69502DE1FF0E0A01DF5D29E0030EB2
:10327000DE5D03E10101CE0E21D0050EDE5D02E12F
:10328000320E14D0020EDE5D03E101019C0E16D059
:10329000060EDE5D02E1640E09D0DE0503E10101E8
:1032A0006A0E0CD0070EDE5D05E1960E01010B6F74
:1032B0000C6B06D0DE5104E10101380E0B6F0C6976
:1032C000FB0EDB0416E1BAECEAF006E3A7ECF1F042
:1032D000EE26E451ED2205D0A7ECF1F0EE5EE451CC
:1032E000ED5A5DECE5F001010B51EE260C51ED229B
:1032F00015D0BAECEAF006E3A7ECF1F0EE5EE4518B
:10330000ED5A05D0A7ECF1F0EE26E451ED225DEC8C
:10331000E5F001010B51EE5E0C51ED5A66ECF4F054
:10332000FD0EDBCFEEFFFE0EDBCFEDFF06D0FD0E78
:10333000DBCFB4F6FE0EDBCFB5F67FECE5F042EC6A
:10334000E8F0B3ECF4F0DEEFE4F041ECEFF0140E53
:10335000DF6E010178A302D0230EDF6E78A102D0C8
:103360000A0EDF6EDF50E552DEEFE4F00A0E036E68
:103370000C5002E1EADF036E0050320D43ECE5F041
:10338000010E0F0B03E027ECF2F0FDE103500A0DF4
:10339000A8ECE7F001010F50D25D1050D3590BE2B9
:1033A000D2510F5C02015B6F0101D3511058020131
:1033B0005C6FE5ECEBF0120004B007D06DECE9F0C7
:1033C0000101D8ECF0F0110E03D06CECF4F0100E0B
:1033D000F1EFE4F0B0C6B4F6B1C6B5F658ECF1F0D2
:1033E000CBBD06D00F500601B45F1050B55B05D0C1
:1033F0000F500601B4271050B523B5C6E6FFB4C67A
:10340000E6FFB3ECF4F0056A0101CBAD02D0060E85
:1034100005266A0E0524A8EFF0F0FBEC26F0056EF9
:10342000055003E1B2ECEAF003E1F7ECEEF002E064
:10343000060E05266AEC11F0006E005002E0005006
:10344000056ECDECF0F003E14FC101F00ED0A1EC20
:103450000BF0000903E085C101F007D0050E005C08
:1034600002E1016A02D056C101F0040E0524E66EA5
:103470002BEC04F0E552ACECF0F0030E005C10E134
:1034800078040EE1FCECE6F0CBB505D0980ED2271F
:103490003A0ED32305D0980ED880D2573A0ED35780
:1034A000E3ECEEF00CE0000405E10101B40ED26F94
:1034B000460E04D001017C0ED26F2E0ED36FE66A49
:1034C0000150E66ED2C1E6FFD3C1E6FF28ECE6F07C
:1034D0006A0E0524A8EFF0F002015B6B5C6B21AC77
:1034E00002D00101E28996EC04F00101E2990C504E
:1034F00011E12A5173ECE9F039DF0101CBBD06D0AF
:103500006DECE9F0D8ECF0F0130E69D06CECF4F04F
:10351000120E65D0BEECEAF00CE00101F20ED26FA3
:10352000030ED36F23DF04900101CAA50CD00480E1
:103530000AD058ECE7F009E0FCECE6F017DF049065
:103540000101CBB5048038DF4DD0DC0E0F6E050EC7
:10355000106E1CECF1F0780E4A1806E14B5004E1B5
:10356000400E0F26060E1022050E0C5C0BE1010E1C
:10357000E66EE66A980EE66E3A0EE66E4ADECBEC32
:10358000F3F02FD0040E0C5C11E16DECE9F0E66E67
:103590003A0EE66E28ECE6F00101CDA723D0CD511E
:1035A000020B02E0180E1BD0190E19D00C0404E017
:1035B0006AEC11F001080CE16DECE9F00F244A6EA1
:1035C0003A0E1020F6ECF3F028ECE6F0110E07D0DE
:1035D00025ECEEF042ECE7F098ECEFF0100EE66E22
:1035E00070DCE552695004E05BC263F25CC264F2D5
:1035F000120072DF695006E182ECE6F002E0EAEFC9
:1036000019F00BDF1200D9ECE4F00701B451320DD0
:10361000ACECF0F0BAECEAF011E1FE0EDB500EE19A
:103620000C5004E101012A5173ECE9F0BEECEAF020
:1036300005E00101F20ED26F030ED36FDEEFE4F06E
:1036400041ECEFF0695004E02550100B01E1B9D1D5
:10365000CEEC0CF0D6CAB3F707011E0EB46F0C50B7
:1036600005E159ECE8F03FC0B4F710D0030E0C5C54
:103670000DE1030E785C02E1140E07D058ECE7F080
:1036800005E0260E25ECF0F00701B46FD7CA00F074
:103690000701EFAF10D0190E006E0A01D75D06E2E8
:1036A000C6ECECF05DECF1F0005E05D0190ED75DD4
:1036B0005DECF1F00026190E005C05E3190E005CCC
:1036C0000701B42705D0190ED88000540701B45F54
:1036D000040E006E0C5005E138DE5DECF1F0006E7A
:1036E00009D00C0406E0020E0C5C03E0040E0C5C36
:1036F00001E1006A0701B351FE0BE8420024056EA8
:10370000DF6A0550B45D13E2DF2AB351FE0BE842D5
:10371000B425016E01500024FE0BE842B46F005046
:10372000015C02E20050016E0050015CB36FB3C750
:10373000B2F7040E0C5C03E1B351E824B26F050E3E
:103740000C5C05E1320EB36F1F0EB46FB26966EC0C
:10375000F4F0EECFB5F7EDCFB6F7040E0C5C20E237
:10376000DFCFE6FF50DFE552020E0C5C08E06AECAA
:1037700011F0020804E01FEC12F0000909E0010159
:10378000D2510701B5270101D3510701B62308D053
:103790000101D2510701B55F0101D3510701B65BA9
:1037A000CDECE8F001E109D1ECECE5F0EF96070192
:1037B000B251D5ECE5F004E24A500A08000E4B5431
:1037C00003E3ECECE5F0EF8697ECF3F0080B02E096
:1037D000B60E01D0B00E006E3BECE8F002E0B30E86
:1037E000006E0701B751005C09E1BD51B51906E152
:1037F000BE51B61903E1B851B25D1AE000C0B7F787
:10380000B5C7BDF7B6C7BEF7B2C7B8F7B5C7D2F1EF
:10381000B6C7D3F1B251320D69ECE5F0050E0C5C80
:1038200004E1C80E0F6E320E106E005029ECE7F066
:10383000CDECE8F001E1C1D0ECECE5F0EF9AECEC76
:10384000E5F0EF8E4DECE9F018E10701B351020805
:1038500014E301013DAB04D0ECECE5F0EF8A0DD0B0
:103860000701B451D5ECE5F004E24A501E08000E01
:103870004B5403E3ECECE5F0EF9EE3EC23F00C504B
:1038800003E0030E0C5C2EE10701EF51800B03E116
:10389000BAECEAF027E1DF5025E1E7DBE5ECEBF0FD
:1038A0000A01D751190808E2190ED75D6AECE7F052
:1038B0000101D2274B50D323BAECEAF008E2C6EC60
:1038C000ECF06AECE7F00101D25F4B50D35B0101F1
:1038D0000A0ED303F3CFD3F1D203F3CFD2F1F450D6
:1038E000D32704D0DFCFE6FF8EDEE5520701B351C8
:1038F000320D69ECE5F04DECE9F007E001012A51E9
:1039000073ECE9F0960E0F6E106AD8EC09F003081C
:1039100002E10101D38F97ECF3F0200B02E0B70E28
:1039200001D0B10E006E0701B951005C10E1BF512A
:103930000101D2190CE10701C0510101D31907E1BE
:103940000701C1510F1802E1C25110180DE000C06B
:10395000B9F7D2C1BFF7D3C1C0F70FC0C1F710C0CC
:10396000C2F7005029ECE7F04DECE9F024E0CDEC93
:10397000E8F021E00701C3510101D21909E1070173
:10398000C4510101D31904E10701BA51B35D13E039
:10399000D2C1C3F7D3C1C4F7B3C7BAF70701B35154
:1039A000320D69ECE5F0B20E29ECE7F0100EE66E90
:1039B0009DEC17F0E552DFEC11F0CAEC0EF097EC3D
:1039C00068F0E552DEEFE4F0CDECF0F001E112003A
:1039D000CDECE8F047E0040E005C05E3B4C6D2F19C
:1039E000B5C6D3F117D0030E005C07E1780405E1FA
:1039F000B5C7D2F1B6C7D3F10DD0DC0E0F6E050EF0
:103A0000106EE3ECEEF004E0400E0F6E060E106E4A
:103A10005CEC0AF0F00E0F6E0A0E106E000403E06C
:103A2000020E005C0EE101018BA105D08A516E0DE2
:103A300069ECE5F006D0355104E0C80E0F5E000ECB
:103A4000105A040E005C04E1700E0F6E170E106E1B
:103A5000050E005C04E1C80E0F6E320E106ECB0E28
:103A600029ECE7F0CDECE8F03EE00101DC0ED26F8E
:103A7000050ED36FF00E0F6E0A0E106E030E005C73
:103A80000CE1780409E18E51400B06E0FCECE6F015
:103A9000900E0F6E010E106ED38FE3ECEEF014E07B
:103AA00001018A516E0D69ECE5F0E5ECEBF0010ED9
:103AB0000F0B05E0D890D333D233E806FBE1640E58
:103AC0000101D227000ED323050E0C5C09E1010190
:103AD0000E0ED26F060ED36FC40E0F6E090E106E4F
:103AE000CF0E29ECE7F01200530E006EE66A00508C
:103AF00018ECF3F0695003E15C0EF1ECE4F05B0EBE
:103B0000F1ECE4F0A70E016E026A2FECEEF0C20EAB
:103B10000AECE5F05D0EF1ECE4F0D6EFEBF001011C
:103B20003CA905D0570EE66E66EC18F004D0570E8F
:103B3000E66E61EC17F0E552120045ECEFF08DEC0B
:103B4000E5F02BE0F1ECE5F028E10701875125E1F4
:103B500001013C51800B03E1050E0C5C1EE14C0E93
:103B60003DECE7F0DF6E050E0C5C11E10101DE9F1C
:103B7000DFA8DE8F3CA90BD0010E696E4C0E3DEC28
:103B8000E7F084ECEAF0696A3398DBA83388010136
:103B90003CAF03D0010EDF1401D0000EB6ECEAF00A
:103BA00002E2E16AE552E16E4A50DEEFE4F0010123
:103BB0003C51800B06E08DECE5F003E0F1ECE5F024
:103BC00001E0000C010CF3DF000902E0510E01D00E
:103BD000500EF1EFE4F06FC1E6FFD00EEEECE4F032
:103BE00054C1E6FFD10EEEECE4F070C1E6FFD30E57
:103BF000EEECE4F0E3EF1DF001013CA905D0560E18
:103C0000E66E66EC18F004D0560EE66E61EC17F026
:103C1000E552120001013851100B02E0140E01D0E0
:103C2000050EE66EAC0EEEEFE4F02150400B06E020
:103C30000101DF51040B02E1DF8501D8120041ECE4
:103C4000EFF055C1DFFFFCECEAF003E159C1DFFF03
:103C500009D00101E051020B05E09751040B02E08D
:103C600098C1DFFF040EDF02F350E66EC70EEEECE4
:103C7000E4F001019751080B03E0DF51040B02E06F
:103C8000000E01D0010E000902E06F0E01D06E0E91
:103C9000F1ECE4F00201FB51E824E66ED40EEEEC08
:103CA000E4F0E552DEEFE4F0020EE66EBC0E18EC36
:103CB000F3F07C0EF1ECE4F0070EE66E6C0E18ECFF
:103CC000F3F07D0EF1ECE4F0BC0E0F6E020E6EEC24
:103CD000F0F07E0EF1ECE4F06C0E0F6E070E6EEC61
:103CE000F0F07F0EF1ECE4F0D6ECEBF046C1E6FF2D
:103CF000C10EEEEFE4F0620E006E07010E9D0101B1
:103D000058AD03D0002A07010E8D0050F1ECE4F00D
:103D1000258A12000701E7510C0803E3E8510C085B
:103D200005E2E76B0C0EE86F0A01DA931200016AF4
:103D30000D0E015C07E051ECE9F002E001501200C9
:103D4000012AF6D7000C0C0E016E015007E051EC71
:103D5000E9F002E0015012000106F7D7000C07015C
:103D6000E56BE66BD7DFE7C701F00701E851D880C4
:103D7000015409E38AEC04F0F3500701E513F45011
:103D8000E613012AF2D71200016A9EECE9F00BE07B
:103D9000E7ECEFF006E24A500508000E4B5401E252
:103DA000012A1D0E0DD04DECE9F011E0E7ECEFF02B
:103DB00006E24A501408000E4B5401E2012A1F0E7D
:103DC0005FECEBF0F3CFE5F7F4CFE6F71200E7ECAA
:103DD000EFF016E24A504608000E4B5411E23BEC5D
:103DE000E8F00EE10701F80EE56FE669050E0C5CE0
:103DF00001E1C7D0E76B0C0EE86F0A01DA83C1D08E
:103E0000006A0A01D751D5ECE5F006E24A500D08E8
:103E1000000E4B5401E2002AD751D5ECE5F006E242
:103E20004A501308000E4B5401E2002AD7511808DB
:103E300001E2002AD751190801E2002AD751D5EC36
:103E4000E5F006E24A501F08000E4B5401E2002A3A
:103E5000D751D5ECE5F006E24A502508000E4B5448
:103E600001E2002A3BECE8F007E0020E006E0101DF
:103E7000CDA302D0040E006E0C5003E0030E0C5CC8
:103E80001CE1E7ECEFF006E24A500508000E4B5447
:103E900001E2012AB6ECF4F006E24A500A08000EEC
:103EA0004B5401E2012AB6ECF4F022E24A50130826
:103EB000000E4B541DE2012A1BD0E7ECEFF006E2A6
:103EC0004A501E08000E4B5401E2012AB6ECF4F0F1
:103ED00006E24A502808000E4B5401E2012AB6ECD3
:103EE000F4F006E24A503208000E4B5401E2012A77
:103EF0009A0E4D6EEE0E4E6E010E4F6E0050506ECD
:103F0000516A526A030ED890503651365236E8063E
:103F1000FAE14D5050244A6E4E5051204B6E4F5096
:103F200052204C6E0150536E546A556AD8905336E5
:103F3000543655364A505324F36E4B505420F46E89
:103F40004C505520D6ECEFF00900F5CFE5F70A000C
:103F5000F5CFE6F7BAECECF005E00701E587E68976
:103F6000E59FE69B030E0A01D45D02E0D45109E10E
:103F7000DEDE0701E76FE7DE0701E86F0A01DA839B
:103F8000C9DE0A01D40514E10701E805056E0A0E31
:103F9000E85D01E20506CBDE0701E76F0550D8803A
:103FA000E75502E205C0E7F7DADE0A01DA8312001C
:103FB000020ED45D12E10701E729056EE751020800
:103FC00001E2052AC0DE0701E86F0550E85D02E264
:103FD00005C0E8F7C4DE0A01DA8312001E0E006E87
:103FE0000C5004E159ECE8F03F500BD0BEECEAF085
:103FF00002E0140E06D058ECE7F004E0260E25ECA3
:10400000F0F0006E0A01D651FE0BE842056E120078
:10401000170E73ECE5F0050E0A01D803F350006E9D
:104020000101012BA1EC96F00101200E1C6F1E8FE7
:1040300012001A0E73ECE5F00A01D951ACECF4F061
:104040005DECECF01E8F1200ACECF1F0F4EC7EF0C5
:104050002AEC2EF0300E01011C5D02E1200E1C6FD7
:104060001E8F016B700EB1EFE8F00C5003E10101FF
:104070002A510BD0030E0C5C10E1030E785C02E1B8
:10408000650E03D0785004E1960E0F6E106A120090
:104090002A0E25ECF0F00F6E106A12009FDF070168
:1040A000EFAF15D0B1ECF0F0E0DF0A01D7511908FD
:1040B00007E2190ED75D6AECE7F00F264B5010228D
:1040C000190ED75D17E2C6ECECF063EFF1F00A01D0
:1040D000D751190803E2190ED75D0026190ED75DD6
:1040E00003E2C6ECECF0005EB1ECF0F0190ED75D27
:1040F00001E1BBDF12003BECE8F00AE00101CD93E7
:104100000A01D751190802E20101CD830A01D76BD8
:1041100012003BECE8F009E00A0E06ECE5F00101C4
:10412000CDA32BD00B0E06EFE5F0AB0E73ECE5F054
:10413000B5DFBAECECF00BE00101410E196F500E47
:104140001A6F0301D851106AE8307F0B0F6E5DECD7
:10415000ECF0BAECECF009E00101460E1B6F2A51BD
:10416000E8240301D85D07E103D0BAECEAF003E1EB
:1041700001012A0E1C6F01011E8F1200D9ECE4F020
:10418000070EE12629EC12F00A01D65D04E229ECC3
:1041900012F00A01D66F41EC12F00A01D880D65510
:1041A00004E241EC12F00A01D66F70EC12F0000943
:1041B00003E00A01190ED76F11DFBAECEAF004E34D
:1041C000190ED75D002603D0C6ECECF0052605508D
:1041D000005C03E30550005E0AD0006AD40507E1E5
:1041E000DC51D75D04E2DCCAD7FADDCAD6FA00C0DA
:1041F000D8FAF4DE05500026BAECEAF004E3190E12
:10420000D75D002609D0C6ECECF0056E0550D880CD
:10421000005402E20550005E35ECF0F00BE24A502B
:104220005408000E4B5406E2540E006EDCCAD7FA56
:10423000DDCAD6FA00C0D9FA190ED75D03E3190E0C
:10424000D75D03D0190ED880D7550701E36FE46B13
:10425000EFAF02D00A0E01D0320EE403F3CFE4F741
:10426000E303F3CFE3F7F450E427695002E0D7CA41
:1042700060F282ECE6F004E0060150850A01DA8182
:10428000FE0EDB5014E02150800B11E10A01D451E5
:1042900002E1DADE0AD0D40502E1BADE06D0020E6F
:1042A000D45D02E1C6DE01D034DF960E096E3550D2
:1042B000040B13E10A01DA51020B0FE082ECE6F085
:1042C0000CE19EECE9F009E14DECE9F006E1BAEC15
:1042D000ECF003E13BECE8F003E056DD359401D06F
:1042E0003EDDF4EC7EF0040E0C5C04E1010E34ECD7
:1042F000EEF0FDE10C500AE10E0ED8800F54010ED5
:10430000105404E20E0E0F6E010E106EFD0EDB5007
:1043100001E195D01950020B01E091D0050E0C5C23
:1043200001E18DD0F8ECEAF001E089D0D5CADFFFD9
:10433000026802C0D5FA050EDB68060EDB68D950AC
:10434000030FE96EDACFEAFFEE68ED68016A050E49
:10435000015C5DE2010E01C0E7FFE75204E0E846C0
:10436000FE0BE706FCE10701E1154FE069500EEC9A
:10437000F4F001500F01BFECE5F0EF50050DDE52F7
:10438000F3CFDEFFF4CFDDFFDD52B9ECE9F01FE241
:10439000010EDB500F5C4C6E020EDB5010584D6E60
:1043A000050EDBCF4EF0060EFFECECF010E2010E36
:1043B000DB500F5C4A6E020EDB5010584B6E050E40
:1043C0004AC0DBFF060E4BC0DBFF0150026EB9ECAA
:1043D000E9F01BE313ECEBF04C6E10503F584D6EC0
:1043E000030EDBCF4EF0040EFFECECF00EE213EC0C
:1043F000EBF04A6E10503F584B6E030E4AC0DBFF85
:10440000040E4BC0DBFF01C0D5FA012AA0D7FF0E76
:104410000A01D55D07E1FF0E025C02E1D56B02D017
:1044200002C0D5FA695002E0D5CAB1F2DF50D55DBD
:1044300006E07DEC95F088ECEBF089ECEAF0B1EC6D
:104440004BF0070EE15C02E2E16AE552E16EDEEF5D
:10445000E4F0006A800E066E056E05500502F3500A
:10446000015CF4500258D8B008D000C005F00642F4
:104470000650051206BE09D0F0D705C000F006426E
:104480000650051206BE01D0E8D700D01200D9ECC4
:10449000E4F02B8420EC15F049C102F05CECE6F06E
:1044A00004E094EC05F0940F026E00504C6E4D6ADF
:1044B0000250F5ECE5F00F50016E10C002F0C9DFBC
:1044C000036AFBEC26F0016E1D50040B2FE0010483
:1044D00003E0020E015C2AE13550400B27E1FE0E9D
:1044E000DB5024E010C202F0025020E0025053ECF6
:1044F000E5F002E647ECE7F019E20250FE0BE84275
:10450000D880005413E20250E824005C0FE2FE0E53
:10451000DB0406E1320E02010F27000E102305D046
:10452000320E02010F5F000E105B032A03500EE1F2
:1045300002010F6B35ECF0F007E24A507108000EF3
:104540004B5402E2710E006E00C010F22550020BB7
:1045500006E12350400B03E03250800B0AE0036A6F
:10456000006A32AE06D0000E0201116F126B0F6F9F
:10457000106B035007E10050E66EE66AC80E0AECC5
:10458000E5F002D0E7EC0BF0DEEFE4F032ECE9F01E
:10459000C20E0AEFE5F0D9ECE4F058ECF1F0F6DFEA
:1045A0001D8EFE0EDB5005E0695003E1680EF1EC54
:1045B000E4F0DEEFE4F041ECEFF035C1DFFF0101A4
:1045C000355108E02150400B05E01C50020B02E081
:1045D000010EDF6EFBEC26F0026E036ADF5006E090
:1045E000030E025C03E0050E025C02E1010E036EA5
:1045F0008C0E006E035001E000683C0E03ECEFF0FF
:10460000C50E0AECE5F0C60E016EDF50006E040E1A
:10461000025C04E1100E0026D80E016E035006E085
:10462000006A040E025C02E1100E006E0050E66E9D
:104630000150EEECE4F0046A035001E0048E0450F3
:10464000E66ECE0EEEECE4F0E552DEEFE4F006ECC2
:10465000EDF003E00101355106E00201DE5105E114
:104660000101355102E0E4EC1CF02B841200016AD8
:1046700054ECE7F001E1012A006A3290015011EC9C
:10468000E6F0EAECEBF0EF50800B06E0015011ECA5
:10469000E6F0EF50006E3280E66A0050E66EDF0E04
:1046A0000AEFE5F0D9ECE4F0695014E1040E0101E1
:1046B0002903F350006EFE0EDB5002E0005001D0E3
:1046C000000EE66EC30EEEECE4F00050E66EAD0EAA
:1046D000EEECE4F0DEEFE4F01CECF3F04D0E0A6ECD
:1046E000695003E0DE52800EDD6E010EDB509CEC63
:1046F000E5F0FF0E005C14E0BC0EF1ECE4F0DF6AC4
:10470000DF5053ECE5F002E647ECE7F009E2010E7A
:10471000DB5061ECF0F000502BECF2F0DF2AF0D728
:104720000A6A020EE15C02E2E16AE552E16EDEEF46
:10473000E4F0D9ECE4F0016A080E015C10E2FE0E30
:10474000DB5001243EECEEF0026E100E025C040D14
:10475000F350006E00502BECF2F0012AEDD7DEEFA3
:10476000E4F0CDECE8F00DE0AB0EF1ECE4F0D8ECC9
:1047700009F0000902E1180E01D0080EE66ED9DF3B
:10478000E5521200CDECE8F00DE0CA0EF1ECE4F0D9
:10479000AAEC0BF0000902E0100E01D0000EE66E4C
:1047A000C8DFE55212004CECEFF00A0E0B5C08E19A
:1047B00025A803D0010E696ED4DF696AD2DF01D06B
:1047C000E1DF54EFEFF0CEEC0CF0ECECE5F0EFCFE6
:1047D0004AF00DECEDF0EF5000014A5C0EE097EC72
:1047E000F3F0E66E0DECEDF0E8ECE5F097ECF3F0AD
:1047F000800AE66EB40EEEECE4F01200AFECF4F0DA
:104800000701F1054EE001013851080B03E1385171
:10481000200B02E0010EDF6E006A0701870507E149
:10482000695002E1008203D0DF5001E000860201FE
:104830008EB3008800507FECEAF0695002E1010E6F
:1048400003D0DF5004E0040E00107FECEAF0010E0C
:1048500052ECE6F000507FECEAF0280E52ECE6F065
:10486000070187051EE0020EF1ECE4F0020EF1EC08
:10487000E4F0006E020E005C08E1695002E1510EA6
:104880000ED0DF500EE0570E0AD0FD0E005C09E09E
:10489000695002E14E0E03D0DF5003E0540E77EC76
:1048A000E5F0E552DEEFE4F00701F10501E1120069
:1048B0002B92E1EC18F0695006E0100EE66EA60EA1
:1048C000EEECE4F00AD0E66AA60EEEECE4F0E66A5E
:1048D000BF0EEEECE4F00AEC1EF0E668A70EEEEC7C
:1048E000E4F0695013E1610EF1ECE4F0620EF1ECDA
:1048F000E4F07BEC1EF0650EFBECF2F0660E0AECC9
:10490000E5F0E66AE66A660E0AECE5F0220EF1ECE6
:10491000E4F0695003E1420EF1ECE4F020EC1BF00E
:10492000FCEC1DF08DEC0CF0695002E14AEC09F052
:1049300013D9C80EE66EB50EEEECE4F0700EF1EC95
:10494000E4F0020EE66EE66AE00E0AECE5F0800E98
:10495000E66EE20EEEECE4F0010163855D95B8ECE5
:1049600011F031DF280EE66E110EE66EE668A90E34
:104970009BECF3F0360EFBECF2F0C00EE66EA40EEC
:104980009BECF3F0695002E172D866D897EC68F0BE
:10499000A3DE695023E1D4EC16F0A5EC16F07CC13F
:1049A000E6FFCC0EEEECE4F054EC1EF03450040BB9
:1049B00002E0530E01D0520EF1ECE4F01FEC1EF0B9
:1049C000E1DEACECE8F0F7DD7DC1E6FFD60EEEEC03
:1049D000E4F0B2EC16F0EBEC1DF049DE74EC1DF0E7
:1049E000010EE66ED8DDE55276ECE9F00601B66B15
:1049F000090EB76FB6DE640EE66EF20EEEEFE4F06F
:104A000001010A0E8C6F88EC13F0248A2A0E9EECAA
:104A1000F3F02E880701010E876F696A010138BB28
:104A2000696EA5EC0DF0EADE696A1200046A010104
:104A300060AF04D012BC048012BE04823DB904846D
:104A40003BECE8F001E004880101E0B50486045085
:104A5000E66EBA0E82EFEBF0695008E10101805179
:104A6000E824E66EA10EEEECE4F0E0DF12006950FF
:104A700018E101013229080DF350E66E050E325D92
:104A800002E2020E01D0010EE66EAA0E0AECE5F07B
:104A900001013C51400B02E0390E01D0380EF1EC1F
:104AA000E4F01200016A0701EFB302D04CC101F03B
:104AB0004DC102F0EF51020B08E00C5004E1060179
:104AC000F051010802E34EC102F00150E66E62C1EE
:104AD000E6FF48C1E6FFA80E9BECF3F002502BEC7A
:104AE000F2F042C100F0CAECF0F004E6F20E4A5CCB
:104AF000000E4B5802E2F20E006E00502BECF2F06A
:104B00003C0E006E0701EFA102D03D0E006E00507A
:104B1000F1ECE4F074C1E6FF73C1E6FF72C1E6FF99
:104B2000A00E9BECF3F071C1E6FFF30EEEECE4F0A7
:104B30000701EFB110D026ECF4F004E076EC68F059
:104B400097EC68F01550100B06E01550200B03E1B0
:104B50001598C4EC6AF0120047ECF4F0A3DF0101F1
:104B60003CA904D0010E696E9DDF696A54EFEFF035
:104B700041ECEFF00C5003E1010EE66E84D0F1EC55
:104B8000E5F001E182D0020E785C67E185EC04F08B
:104B900069ECE5F0AA0E01010F24D26F000E10207F
:104BA000D36F39BD0BD085EC04F0ACECF0F0AA0E5D
:104BB0000101106AD2250F6ED3511022E7DC7D0E61
:104BC000F1ECE4F0680EF1ECE4F043ECEEF0DEDC46
:104BD0007C0EF1ECE4F0690E51ECF2F00101395178
:104BE000400B400A01E0010E4A6ECB51040B040A4F
:104BF00001E0010E4A1805E0550E0F26000E1022A6
:104C000004D0550E0F5E000E105A20ECF1F0010199
:104C10003951400B400A01E0010E4A6ECB51040BA2
:104C2000040A01E0010E4A1805E0AA0E0F5E000E0C
:104C3000105A04D0AA0E0F26000E102232ECE9F012
:104C4000B3ECF4F07F0EF1ECE4F0030EDF6E010143
:104C500097A113D0070EDF6E10D048ECEEF096DC73
:104C60007C0EF1ECE4F0680E51ECF2F020ECF1F087
:104C7000010EDF6E010178BDDF2A69ECF1F005015C
:104C8000040E146FE66A87DCE552E552DEEFE4F0CD
:104C900041ECEFF0CEEC0CF002013F6B0601C26B71
:104CA000C2C6C0F6339E0C5022E1F051010803E366
:104CB0001450010B17E0010E016EF051020802E2E0
:104CC000030E016E040EF05D02E1020E016E015052
:104CD0002EECF2F0E00E0AECE5F0F1C6E6FFEBECAC
:104CE000F1F003D0700EF1ECE4F036DF6AD0030E81
:104CF0000C5C64E1ECECE5F0EF981450010B06E17C
:104D00009EECE9F003E107ECEFF053E058ECE7F03C
:104D100015E02E0E25ECF0F0016E020E026E2D0E47
:104D2000DF6E010197A104D0040E026E4B0EDF6E00
:104D300014A016D00201010E3F6F12D0BEECEAF0B3
:104D40000FE0030E016E010E026E1F0EDF6E0101F9
:104D500078AD06D0040E016E030E026E3F0EDF6EBC
:104D60002FECEEF0E00E0AECE5F0F3C6E6FFEBEC1C
:104D7000F1F09EECE9F003E0ECECE5F0EF880701E0
:104D8000200E7E6F3F0EDF5C02E1100E7E6F640E20
:104D9000DF5C02E10A0E7E6F4B0EDF5C02E10D0E5E
:104DA0007E6F2D0EDF5C02E1160E7E6F7B6B7F6BDC
:104DB00003D0700EF1ECE4F006DD03D0700EF1ECE0
:104DC000E4F03EEC4BF0E552DEEFE4F01C849F0E85
:104DD000D9ECE5F01C940050EFECEEF0005C020121
:104DE0001E6F0050E00BE838E8401E27050E1E2716
:104DF0001EC200F0120020B202D00C5012007D50F2
:104E000012000A0E8DEFF1F014A205D0E2C20FF0ED
:104E1000E3C210F012009A0EDCECF1F00FC0E2F2E7
:104E200010C0E3F212004C6B4D6B4E6B4F6B400E9B
:104E3000506FD89047374637453744374337423766
:104E4000413740374F374E374D374C374B514F5D19
:104E50004A514E5949514D5948514C5909E34B510A
:104E60004F5F4A514E5B49514D5B48514C5B472B5C
:104E7000502FE0D7120012A409D00101CB9912BE25
:104E8000CB89CC9712AC09D0CC8712000101CB970B
:104E900012BECB87CC9912BCCC8912001250040BE5
:104EA00004E00101CB51100B09E11250040B04E1A5
:104EB0000101CB51080B02E1000E01D0010E04905C
:104EC000E8B004801250040B04E00101CC51080B3F
:104ED00009E11250040B04E10101CC51100B02E175
:104EE000000E01D0010E0492E8B00482ECECEAF06E
:104EF00004E00201BB51100B02E1000E01D0010ED3
:104F00000494E8B0048434AC09D0129E0101D7B1F6
:104F1000128E129CD7A308D0128C06D0129E04B019
:104F2000128E129C04B2128C0450040B040A01E08D
:104F3000010E4A6E0450010B4A140496E8B0048630
:104F400007011D9904B61D891D9704A61D8701013F
:104F5000E3B906D007010B9904A218D00B8916D02B
:104F600007010B990450020B06E0020E0201BC156A
:104F700002E007010B8907010B910450020B06E0C8
:104F8000010E0201BC1502E007010B810450040B65
:104F900005E0E6ECE8F002E0000E01D0010E4A6EFA
:104FA0000101D751010B4A140498E8B004880701A5
:104FB0001B9904B81B891B9704A81B87079901013B
:104FC000D7A302D0070107890701109304B4108307
:104FD0000101E39104B6E381E39304B8E38316EFA0
:104FE00025F00701109B12A4108BF4ECEAF049ECB9
:104FF000E9F005E0E6ECE8F002E0DAEC0CF011ECA8
:10500000EEF016EFEEF041ECEFF058ECF2F0200E7F
:1050100061ECF0F00050026E0F0E61ECF0F0010157
:105020002C51005C19E1250E025C16E1050E26EC00
:10503000F1F00101CAA903D063ECE6F0076A050E9E
:105040000C5C07E1030EE66E100EDF24E66EF3EC57
:10505000F1F00A6A010E02D00A6A000EE552DEEF94
:10506000E4F0D9ECE4F0CAECECF03B812C8C2D8A16
:10507000AFECE7F05DECE5F0EE50ED1011E0010172
:10508000452B640E455D03E2BEDF00091BE1010113
:10509000450703E0B8DF0009FAE10101452B12D012
:1050A00001014507FF0E455D03E0ADDF00090AE1A0
:1050B0000101452B640E455D03E2A5DF0009F8E11F
:1050C00001014507DEEFE4F02A50800B0DE00101FD
:1050D0003851400B09E02C50100B06E12B50010B0E
:1050E00003E1100E2C5D01E3000C010C0BECEFF062
:1050F00004E00FECEFF001E2010C000C0701E06BA3
:10510000070E1315006E400E136F005013130101AC
:10511000389D2BAA38D0020E3A5D02E107011387B1
:1051200001013A51020807E2070E3A5D04E2020E5D
:105130003A5D0701E06F2AAE26D0070E01013A5D05
:105140000BE12C50100B08E14951780803E26C0E7A
:10515000495D496F80EC56F0080E01013A5D13E39A
:10516000388D4951780804E207011387139B139D7A
:1051700001013A51080807E20D0E3A5D04E2080EFB
:105180003A5D0701E06F07011291129312895CECFE
:10519000E6F011E0070112811283129954ECE7F056
:1051A00003E17851800B05E02C0505E16051400BCF
:1051B00002E10701128921AC02D09BEC0FF0B3ECA5
:1051C0002CF0258A120069ECEFF04B6ADA0F4A6E78
:1051D000060E93ECEFF0006E009EFE0EDB5004080E
:1051E00006E1FD0EDB504F0802E2020E006EDEEF1C
:1051F000E4F00101E351200B03E04451040803E310
:105200004451040801E2446B040E445D02E1190EAE
:1052100004D0160E442597ECE5F0006E0050E66EC3
:10522000E66A3C0EE66E31ECFAF0CBECF3F005ECFE
:105230000CF0258A12000201320E346F395102E05F
:10524000140E346FC80E496F640E506F1EAC2A984E
:105250001E50400B03E02B50800B02E1E1EC18F0F4
:105260000201906BFC6B1200D9ECE4F0FE0EDB50F7
:105270000EE02AA006D0FE0EDB50030B02E1CBECC1
:1052800007F0280E33ECE7F0FE0EDB06EFD7DEEF7B
:10529000E4F001C502F50501006B289C0101DE91D7
:1052A00012007CECE9F0F5DFF1ECE5F002E0080E2D
:1052B000086E12000850220A01E167D1030A01E1D9
:1052C00046D1010A01E1C7D03F0A17E0010A01E017
:1052D00075D1288C07ECEFF007E0200E06014A5D3F
:1052E00003E0200E43ECE6F01E901F0E086E020154
:1052F0003D5101E164D1086A17D00501005101E177
:1053000081D0F1ECE5F014E00501115107E1020E46
:10531000145D0EE18AEC0FF000090AE102013D5133
:1053200001E13D2B080E086E01011F0EA76F120050
:10533000050100070251EA6A000FE96E080EEA2231
:10534000EFCF02F7022B025153ECE5F002E60CEC32
:10535000EEF001E3026BF1ECE5F006E002C7E6FFD8
:10536000F8EC4FF0E5524BD03C0E0701025D04E132
:105370002582248C239C12003E0E025D04E12592BE
:10538000249C238C1200740E025D64E00601F0512F
:1053900007E02A8A02C7E6FF42EC8AF0E5522A9A21
:1053A000800E0701025D10E2C00E02254A6E4B6AB4
:1053B000000E4B22200E4A5E000E4B5A3EECE5F0EA
:1053C00024ECE7F00701026F800E025D03E10201A9
:1053D000040E676F07010251800805E2800E025D2E
:1053E000FD0F0201676F800E0701025D06E3220ECA
:1053F000086E05011F0E056F120002512BE0200EF2
:10540000086E1200EDECEBF007E007010251800896
:1054100003E3200E43ECE6F044DFF1ECE5F006E0B8
:10542000289C080E086E0101100EA76F2850200B53
:1054300001E1C5D002016A5101E1C1D0199A6ABFE8
:10544000198A2A6B010EE66E7F0E6A1518ECE7F0DA
:1054500002016A6B12001750800B09E11E50040B09
:1054600006E01E50080B03E08150080B4CE1285069
:10547000200B09E01750800B06E03DECECF003E058
:10548000250E675C1FE151EC80F00BDF2194F1ECFD
:10549000E5F003E00201010E3D6F28AA90D0020161
:1054A0006A6B6AC22AF20601F05101E188D0070155
:1054B0000251800801E283D03088200EE66E42EC73
:1054C0008AF01DD0350E675C09E1010EE66EABEC8B
:1054D0000FF0E552F2ECEBF0179E120070ECB5F015
:1054E00000090FE00D50006E020E20ECF3F00D509D
:1054F000026E00500D6E0250E66E16EC8FF0E55213
:105500001200BFEFB8F0F1ECE5F006E0080E086E0F
:1055100001011F0EA76F1200FE0E070102150EE01B
:10552000238E010E016F02A102D0030E016F0291C2
:105530000243210E086E0501200E07D00201020E63
:10554000676F220E086E05011F0E056F120007011E
:10555000015114E00107248004EC80F0086A1EA0C9
:1055600007D0020E086EF0ECEAF002E137ECE9F049
:105570000101210EA76F1E80239E12000201010E61
:10558000676F238E220E086E12000201675113E02E
:105590002490670704EC80F0030E086E1EB005D05F
:1055A000070E086E006A37EC91F00101220EA76F1A
:1055B000239E1E90120005C508F0120072DE120034
:1055C00086C206F1EDECE8F00AE2100E2C5D09EC63
:1055D000E6F0060E09ECF0F0EFCF06F104D02CA8AF
:1055E00002D0960E066F0651D880495502E206C1D8
:1055F00049F11200DACFE4FFE2CFDAFFE9CFE4FFAE
:10560000EACFE4FFE652FC0EB36EF30EB26E020177
:1056100025070201255105E10201320E256F010126
:1056200024811E961E94010158A105D081B41E84C8
:1056300081B21E8604D081B21E8481B41E8602010E
:1056400026070201265137E10201050E266F0101EE
:10565000AB5116E00101AB07020102016651020BDA
:1056600005E01E50040B02E1020166810201020105
:105670006651080B05E01E50080B02E10201668529
:105680000101AC5106E0FF0E0101AC5D02E0010139
:10569000AC2B20AE04D00601E42B000EE52307015D
:1056A0007D5109E007017D0707017D5104E17EC7B7
:1056B0007DF7010124830101AA5102E00101AA073B
:1056C00002010D2B0101279701012795010127A157
:1056D00002D001012785010127A302D001012787FC
:1056E000010127930101279188A202D0010127819E
:1056F00088A002D0010127830F0E010127150101A7
:10570000266F01012651EA6AC90FE96E060EEA22E8
:10571000EFCF25F1010125A12BD02050080B08E087
:10572000010101013C51010B03E02850010B20E075
:105730002E50400B03E03050200B1AE02150200B7C
:1057400017E0010125AF02D0790601D0792A0101C5
:105750000101CA51100B0CE02050080B09E02C503D
:10576000200B06E1010125AF02D0070601D0072A70
:105770000101289701012895010128A102D001010A
:105780002885010128A302D001012887010128935F
:105790000101289188A802D00101288188AA02D09D
:1057A000010128830F0E010128150101266F010157
:1057B0002651EA6AC90FE96E060EEA22EFCF25F1FB
:1057C000010125A124D0010101013C51200B16E16A
:1057D0002050080B13E02E50400B08E1010101019D
:1057E0003C51020B0BE02850010B08E12E50400BFE
:1057F0000EE0010101013C51010B09E12150200B98
:1058000006E0010125AF02D0070601D0072A9EAAB3
:105810001CD0ABA209D0AB98000000000000000033
:1058200000000000AB8811D00701C72B0701C6514B
:10583000C62BEA6A000FE96E0C0EEA22AECFEFFF2C
:105840000701C75102E1C6C7C5F7A1920701520778
:10585000E552E5CFEAFFE5CFE9FFE5CFDAFF11003A
:1058600001013CAB02D03C9B248A12000701EFB13E
:1058700003D0129A129812001298EFA31288129A6B
:10588000EFB3128A12000701EF81E1EC09F0F7EFA4
:10589000EBF019A602D0199612002CA806D001012F
:1058A000E0A523D0560E06EFE5F04B0E0A6E200E53
:1058B000016E12A002D0600E016E01504BECF4F0AC
:1058C000005013E0FF0E005C10E026840101B06B75
:1058D00045C11FF2FC0E456F12B0452B72ECE7F08C
:1058E000B5ECE8F026941FC245F11200220E93EFAA
:1058F000F3F001018BAD09D0D9752C51615D0CE13C
:10590000CD95D9A509D0CD8507D0D9792C51615D28
:1059100003E1CD99D9B9CD8985EC0CF038EF0DF0C4
:1059200034AC02D079EF2CF02CA61BD0127012925E
:1059300012A012820101CB9F12B0CB8F0701169FDC
:1059400012B0168FB8EC09F0E66ACCECC6F0E5525E
:105950008DECC5F00201906B258A17859ADFACEFBC
:105960000CF076EF2CF08DECE5F003E0F1ECE5F0D7
:1059700006E01494010157A306D0148404D01494B3
:1059800001013CB51484149614A414861498145080
:10599000040B04E15CECE6F001E0148812004CEC2E
:1059A000EFF0006A0301C95111E0CCC359F2CDC335
:1059B0005AF2800ECD151DE0CCC359F2CDC35AF278
:1059C0000201596D5A1F000E5A2311D014ECEDF04C
:1059D000595F7A0E5A5B0101A00E505D7A0E515943
:1059E00008E214ECEDF0D88059577A0E5A57800E21
:1059F000006E060E436E446A59C23EF05AC23FF032
:105A0000EBECFCF03EC059F23FC05AF200500201EC
:105A10005A13010178A717D0BAEC3EF0C1EC96F00A
:105A200002C101F003C102F004C103F005C107F196
:105A3000696A560E3AECE9F0010E696E560E3AECC0
:105A4000E9F0DF50696EE552DEEFE4F0D9ECE4F006
:105A5000FB0EDBCFE9FFFC0EDBCFEAFFEECF4AF017
:105A6000EECF4BF0EECF4CF0EECF4DF0EFCF4EF04F
:105A700075ECE8F04AC0EEFF4BC0EEFF4CC0EEFF05
:105A80004DC0EEFF4EC0EEFFDEEFE4F0EDECF3F0C4
:105A9000CAECE6F09F0EE66E010E15ECE9F0CCECD8
:105AA0003AF0D850010B06E0FF0E01019A5D02E0CA
:105AB000010E01D0000EDEEFE4F045ECEFF00050F7
:105AC000FAECF1F04DECFDF048ECFDF00009FCE1E2
:105AD000C450006E1C50040B32E0CAECF0F004E637
:105AE000F90E4A5C000E4B582AE20201F2514B6A51
:105AF000E8307F0B4A6EC80E15ECF0F01CECF1F0AC
:105B0000CFECE7F0A1ECEFF0EECF3EF0EDCF3FF0C1
:105B100096ECF8F03CC0EEFF3DC0EDFFCFECE7F0B7
:105B2000FA0E436E446AEECF3EF0EDCF3FF0EBEC61
:105B3000FCF03EC0EEFF3FC0EDFFEF50006E020EE6
:105B4000E15C02E2E16AE552E16EDEEFE4F041EC95
:105B5000EFF00050DF6EA70E4A6EE90E4B6E010E9D
:105B60002CECF1F00150006E009E0FEC97F001AEAE
:105B7000F2D7E552DEEFE4F041ECEFF00050DF6EDB
:105B80002450100B12E10050E66E8DEC04F0E5524B
:105B9000800B0BE00101450E196F520E1B6F1BC1EC
:105BA0001AF1200E1C6F040E016F2B8824A808D058
:105BB000A30E4A6EEB0E4B6E010E2CECF1F007D0EB
:105BC000DFCFE6FF8DEC04F0E552016EDF2A2BA853
:105BD00002D0019E2B980150006E009E3AEC97F087
:105BE00001AEE4D72498E552DEEFE4F053ECF1F097
:105BF00003E2FBECEEF004D0FE0EDB50410FF60F9B
:105C0000006E0FEC97F0DEEFE4F0F9ECF3F0DB3828
:105C10000F0BE66EEBDFE552FE0EDB500F0BE66E70
:105C2000E5DFE552DEEFE4F0D9ECE4F01BECEDF05B
:105C3000020E0101002784EC96F0DF50006E050E85
:105C40000101005F84EC96F0030E0101005FE55254
:105C5000DEEFE4F0D9ECE4F01BECEDF082ECE9F0DF
:105C6000DF50006E0101020E016FA1EC96F0E552CB
:105C7000DEEFE4F000C06FF2A3EC93F0FF0E005CE7
:105C800001E065DF1888120000C070F2AFEC93F0FD
:105C9000FF0E005C01E070DF188A1200A3EC93F0A5
:105CA000FF0E005C01E053DF188C640E096E259630
:105CB0001200AFEC93F0FF0E005C01E05DDF188E88
:105CC000640E096E25961200D9ECE4F072ECE7F050
:105CD000C6ECEAF090ECE6F0DEEFE4F0D9ECE4F0AC
:105CE00072ECE7F0DFEFF0F0D9ECE4F0F6EC89F0DD
:105CF0000101190EA96FFC0EDBCFADF1FD0EDBCF5C
:105D0000AEF1FE0EDBCFAFF1DEEFE4F0830E0A6EF4
:105D1000E00E4BECF4F0800E005C08E2F6EC89F04B
:105D20000101190EA96F0201E00EDF6F1200F9ECFC
:105D3000F3F0DBCF4BF0800E4B1407E022ECEDF0DC
:105D40004A6C4B1E000E4B2202D022ECEDF0EDEC23
:105D5000F2F0DEEFE4F0016A040E015C0DE20128CE
:105D600056ECF0F0EA228EECEAF0015056ECF0F03E
:105D70008EECEBF0012AF0D7EA0E3DECE7F00301E0
:105D8000C46F318AD1ECF1F00301C56F319A010182
:105D9000DE870480016A040E015C22E2015056ECA9
:105DA000F0F0EA22EECF4CF0EFCF4DF0012856ECA8
:105DB000F0F0EA22EE504C5C4A6EEE504D58F6EC94
:105DC000F3F05EECF2F0010E57ECE6F007E204901F
:105DD000050E57ECE6F002E20101DE97012ADBD75F
:105DE0000450010B48E001018F51080B03E102014F
:105DF000515141E01850020B3EE1020150513BE18C
:105E0000BCC3E6FFBDC3E6FF5EECF2F00F5010101E
:105E100032E0F40E0F5C010E10582DE20401440E26
:105E2000BB6F0301800EBD1503E00401550EBB6F6F
:105E300000ECEBF0040E57ECE6F002E2310E026FDC
:105E4000140E57ECE6F002E2330E026F3C0E57ECF4
:105E5000E6F002E2390E026FDC0E57ECE6F002E2E9
:105E6000340E026F020E13ECEFF003E20201320E69
:105E7000506F0EECCFF01200F9ECF3F0DBAE08D06F
:105E8000DB50FF0DFE0EF3CFDBFF1CECEBF007D079
:105E90001CECEBF0DB50FF0DFE0EF3CFDBFFDB5015
:105EA000DEEFE4F041ECEFF00701875101E045D16E
:105EB000F10501E142D13350040B01E13DD10C5019
:105EC00004E18650020B01E137D1E30E3DECE7F02F
:105ED0000601C16F58ECE7F001E094D0140E060102
:105EE000E76EC119E8AE02D0C13503D0E750D880C3
:105EF000C15502E2140EC16FEC0EE76EC119E8AE97
:105F000002D0E73402D0E750C15D02E2EC0EC16F6F
:105F1000C051E76EC119E8AE02D0C13503D0E750D9
:105F2000D880C15502E2C02B0BD0C051E76EC11919
:105F3000E8AE02D0E73402D0E750C15D03E2C0070B
:105F4000C0C6C1F6080E4A6E4B6AC5C63EF0C6C64C
:105F50003FF029ECEDF03EC0C4F6C4C64AF04B6AEF
:105F60004ABE4B684A500601C55F4B50C65BC1C66E
:105F70004AF04B6A4ABE4B684A50C5274B50C6236D
:105F8000C4C6E6FF79DFE552016E010EE66E0E0E25
:105F900001241EECE7F002012B5101E1CDD01A9E45
:105FA000D1ECE8F002E0000E01D0010E4A6E0C5078
:105FB00003E1B2ECEAF008E00C5004E00101CA5140
:105FC000040B02E0000E01D0010E4A1804E00601A5
:105FD000C151792603D00601C151795EAAECEAF0DD
:105FE00005E02050020B02E17950076E0601C15115
:105FF00001E0A2D002012B51320801E39DD0320E04
:106000002B6F9AD0E40E3DECE7F00601C36F026AF5
:10601000016AC151E76EC319E8AE02D0C33503D09F
:10602000E750D880C35505E2C151C35DC4ECE9F027
:10603000026E0601C351E76EC119E8AE02D0C13548
:1060400003D0E750D880C15505E2C351C15DC4EC0F
:10605000E9F0016E0601C251D880025402E202C08A
:10606000C2F6C051D880015402E201C0C0F6000E51
:10607000E76EC219E8AE02D0C23503D0E750D8802F
:10608000C25505E2010EE66E0D0E1EECE7F0010EA4
:106090000601E76EC219E8AE02D0C23503D0E75060
:1060A000D880C25505E2010EE66E0C0E1EECE7F03C
:1060B000020E0601E76EC219E8AE02D0C23503D067
:1060C000E750D880C25505E2010EE66E0B0E1EECBD
:1060D000E7F0000E0601E76EC019E8AE02D0C03549
:1060E00003D0E750D880C05505E2010EE66E0F0ED2
:1060F0001EECE7F0010E0601E76EC019E8AE02D013
:10610000C03503D0E750D880C05505E2010EE66ED9
:10611000100E1EECE7F0020E0601E76EC019E8AEA5
:1061200002D0C03503D0E750D880C05505E2010E3B
:10613000E66E110E1EECE7F03394E552DEEFE4F06C
:1061400041ECEFF00701F10504E1FD0EDB6AFE0E04
:10615000DB6AFC0EDB504DE102013A514AE104904A
:10616000FE0EDB50140804E2140ED4ECE7F00480B9
:10617000FE0EDBCF4AF06B51D8804A5403E2FE0E8C
:10618000DBCF6BF201012B51100B03E0050E0C5C11
:1061900005E10450010B02E0FE0EDB2ADF6A150E5A
:1061A000DF5C1AE2006AFE0EDB5004E0FE0EDB50FC
:1061B000DF5C0BE301012B51100B09E0050E0C5CB9
:1061C00006E002016B51DF5C02E1010E006E00503F
:1061D0001BECE9F0DF2AE3D71450010B6AE002015F
:1061E000315167E10C5003E0030E0C5C62E1338433
:1061F00060D0FC0EDB0431E102013A5106E0FD0EF5
:10620000DB5003E12350400B57E1FE0EDB50080842
:1062100003E2080ED4ECE7F0FD0EDB500C0805E2BB
:106220000C0EF36EFD0EF3CFDBFFD8ECE8F0150E8D
:10623000DF5C3FE2FE0EDB5004E0FE0EDB50DF5C75
:1062400007E3090EDF5C07E3FD0EDB50DF5C03E2D2
:10625000010E1BECE9F0DF2AEAD7FC0EDB50020846
:1062600028E1FE0EDB50080803E2080ED4ECE7F04C
:10627000FD0EDB500C0805E20B0EF36EFD0EF3CFA6
:10628000DBFFD8ECE8F0150EDF5C13E2FE0EDB500E
:1062900004E0FE0EDB50DF5C07E3090EDF5C07E382
:1062A000FD0EDB50DF5C03E2010E1BECE9F0DF2AA0
:1062B000EAD7FE0EDBCF1DF2E552DEEFE4F07D50B3
:1062C00022ECE9F072ECF4F00150080D4A50F3248E
:1062D0000A01E26F4B50F420E36F12000101C45138
:1062E000BF5D0CE1C551C05D09E1C651C15D06E16C
:1062F000C751C25D03E1C851C35D01E0000C010C50
:106300007D500C5C01E0000C0C500BE1B2ECEAF0AB
:1063100001E0010E4A6ED751400B01E0010E4A5CCC
:106320002DE0030E0C5C24E10101D6512DECE6F0CA
:10633000785C1EE158ECE7F00CE00101CB51040B56
:1063400001E0010E4B6ED751040B01E0010E4B5CD6
:1063500015E058ECE7F00CE10101CA51040B01E033
:10636000010E4C6ED651040B01E0010E4C5C06E0B0
:106370000C5003E0030E0C5C01E1000C010CAEDFDD
:10638000000903E0BDDF000901E1000C010CF7DFAB
:1063900000092FE0050E0C5C01E1010C7D5022ECA0
:1063A000E9F0C2ECECF07D506EECF1F0015013EC32
:1063B000F4F00C50100DF3CF50F0F4CF51F02A0E42
:1063C00050260A0E51220701E251080D5050F324C5
:1063D0004E6E5150F4204F6E4EC0E6FF4FC0E6FFA8
:1063E00074ECF9F0526E060EE15E5250000901E1C4
:1063F000010C000C2CC161F10FC110F11BB202D0D5
:1064000063ECE6F00C507D6E2E50400B03E13550EE
:10641000200B17E0010139A306D0D893CCB3D88361
:10642000D895CCB5D885D79DCBBDD78DD795CBB5D5
:10643000D785D695CAB5D685A1ECF3F01DECF0F062
:106440001BD07D5004E10101D79DCBBDD78D030E3C
:106450007D5C12E10101A1ECF3F01DECF0F058ECD1
:10646000E7F006E00101D795CBA506D0D78504D08B
:106470000101D695CAB5D6852E50400B03E13550A3
:10648000200B0CE0500EE66EE66AA4ECF3F0E66E2C
:106490007A0EE66E0A0EB6ECE6F00CD0050E0C5C39
:1064A00009E0CEECECF077ECF0F07D506EECF1F022
:1064B00064ECF2F0050E7D5C08E07D50EA6ACF0FD7
:1064C000E96E0A0EEA22E2C7EFFF120061C12CF169
:1064D00010C10FF1CFECE9F07D500C6E2E50400B47
:1064E00003E13550200B07E065ECECF0A4ECF3F091
:1064F000B6ECE6F00DD0050E0C5C0AE081ECF0F095
:106500000C50100D38ECE7F01BECEEF064ECF2F000
:10651000050E0C5C02E00EECF3F01200D9ECE4F096
:1065200036DF00090FE1BDEC15F0FE0EDB5002E195
:1065300061DF01D0CBDFFBECEBF0258ACAECECF09D
:106540003B833B81DEEFE4F02D50100B12E049EC71
:10655000E9F00FE0BDEC15F04DDF010E696E198218
:10656000A5EC0DF045EC15F0D2ECECF045EC15F097
:10657000199212002E8C60ECEEF051EC0AF01B9494
:106580005CECEEF0696A01013CA90DD0348C010E7F
:10659000E66E1FD9E552A5EC0DF03EEC4BF0F4ECA5
:1065A000EAF085EC0CF045EC15F04CEF05F0D9EC79
:1065B000E4F05CECEEF0A2ECE9F012E1CB91D7B1A3
:1065C000CB81CB93D7B3CB83CD95D9B5CD85CD99A1
:1065D000D9B9CD89CD91D9B1CD81CD9FD9BFCD8F3D
:1065E0002E9C18983CA906D0349CE66AF2D8E55255
:1065F000A5EC0DF045EC15F0FE0EDB5002E03EEC94
:106600004BF0E4EC1CF0F4ECEAF04CEC05F0DEEFBF
:10661000E4F0BDEC15F0A2ECE9F011E078ECE6F066
:10662000358A17D8359A45EC15F01D8A78ECE6F0D6
:106630001D9A19842EECE7F0199494EFEBF03CA925
:1066400003D063ECEEF0696A04D845EC15F0D0EFA6
:1066500010F061C102F010C103F0C4C1CFF2C5C196
:10666000D0F2C6C1D1F2C7C1D2F2C8C1D3F27D50B7
:10667000006E67ECEEF0D8C1DCF12E50400B03E168
:106680003550200B08E065ECECF0580EE66E060E77
:10669000B6ECE6F009D0050E005C06E081ECF0F007
:1066A00025ECF3F02CECEDF0016A050E005C03E044
:1066B000005022ECE9F09EDE02C02CF103C00FF185
:1066C000CFC2BFF1D0C2C0F1D1C2C1F1D2C2C2F1BA
:1066D000D3C2C3F100500C6E2E50400B03E1355075
:1066E000200B1EE0010139A30ED0CC93DCB3CC8388
:1066F000CC95DCB5CC851396CCB313861394CCB56E
:10670000138408ECC0F00101CB9DDBBDCB8DCB9594
:10671000DBB5CB85CA95DAB5CA85EEECEFF019D0BA
:106720000C5004E10101CB9DDBBDCB8D030E0C5C55
:1067300010E10101EEECEFF058ECE7F006E00101AA
:10674000CB95DBA506D0CB8504D00101CA95DAB57F
:10675000CA852E50400B03E13550200B0AE0500E45
:10676000E66EE66A25ECF3F0A4ECF3F0B6ECE6F0A6
:106770000BD0050E005C08E0CEECECF025ECF3F05D
:1067800077ECF0F02CECEDF001C0E2F7050E0C5CBC
:1067900004E0A1ECE7F001C0EFFF049001013CB17F
:1067A00004803C913CB33C813C9304B03C83139CFB
:1067B0003CB1138C139E3CB3138E2EBC03D0FBEC68
:1067C000EBF0258AF0EC38F0CAECECF0BF0E3B6F32
:1067D000120069ECEFF00AE0696A01016395E3ECED
:1067E00023F0010E696E01015D8509D0010E696E0D
:1067F00001015D95E3EC23F0696A01016385E3EC37
:1068000023F0DEEFE4F045ECEFF00E0E0101305D19
:10681000DF6E060E312584ECEAF00601F45126E025
:1068200007ECEEF0060ED89010320F32E804FBE1D0
:10683000040EDF02F35063ECF1F0200E6CECEEF08E
:1068400002E20F6A106A010EDB504C6E4D6A42EC98
:10685000E7F0070E50ECE8F04AECE8F0FF0E57ECDA
:10686000E6F002E20F68106A0FC0F5F6DF50005E36
:1068700035ECF0F006E24A50C808000E4B5401E235
:10688000006A010EDB504C6E4D6A0050060D43EC61
:10689000E5F04AECE8F00F50006E0050150802E2F7
:1068A000150E006E020EE15C02E2E16AE552E16E55
:1068B000DEEFE4F041ECEFF00201315105E121504F
:1068C000010B02E1345102E0000E1DD0AF0ED9ECF5
:1068D000E5F099DF0050DF6E00C0D4F7090E016EBD
:1068E00001012BB901061450010B06E00150D880BC
:1068F000005402E20150006EE66AE66A0050E66E5D
:1069000093ECE8F0DF50E552DEEFE4F0D9ECE4F090
:10691000016A0A0E015C19E2FE0EDB50010B06E073
:10692000270E01246EECE5F0675C0AE0FE0EDB50FA
:10693000020B09E0310E01246EECE5F0675C03E127
:1069400001500D6E02D0012AE4D7DEEFE4F0D9EC5D
:10695000E4F0800E0D6E17AE17D0179E1750010B86
:1069600003E11750100B10E0100E0D6E7FECE5F0F8
:10697000CDDFE5522A0E675C02E1200E0D6E2B0E74
:10698000675C02E1400E0D6EDEEFE4F0D9ECE4F05E
:10699000DAECE9F07FECE5F0F7EC0BF0E5522AECED
:1069A000F3F00101A46FA451640D69ECE5F0010E50
:1069B000EB50680F32ECF2F02FECF3F033ECEDF02B
:1069C00000504C6E4D6A01014C504A5CD26F4D50E4
:1069D0004B58D36F2AA60BD09A5133ECEDF001013E
:1069E000D2514A5C0F6ED3514B58106E06D09A515B
:1069F000106AD2250F6ED3511022D7ECEEF088EC3E
:106A0000EFF03EC0A4F13AC09AF1DEEFE4F0D9EC29
:106A1000E4F0DAECE9F0DB5009ECE6F0030E09EC07
:106A2000F0F0EF500101A45D02E0000E11D0FE0E67
:106A3000DB5009ECE6F0EAECEBF0EF509A5D006E0B
:106A400000BE006C040E005C02E2010E01D0000EDC
:106A5000DEEFE4F0A8ECF3F0920E4A1810E14B5090
:106A60000EE1006A3AEC2EF0BD0E006E44EC2EF002
:106A7000096A228602018D6B7E6B299E082AA8EC8A
:106A8000F3F0930E4A1845E14B5043E1010EE66ED8
:106A90005EDFE5520A0E0D5C25E202018D5105080C
:106AA00026E37E51020823E38D2B29BE7E2B010EA7
:106AB000016E070E015C13E20128B3ECE5F0EF5024
:106AC000006E060E015C05E1800E010118150D1027
:106AD000006E36ECF2F000C0EFFF012AEAD70101A8
:106AE000189F17D0200E0D5C08E129AE02D0268E2B
:106AF00010D0298E0101188F0CD0400E0D5C04E1DE
:106B0000980E086E1B8805D0100E0D5C02E19A0EDF
:106B1000086EA8ECF3F0980E4A1801E07DD04B50B7
:106B200001E07AD0010E016E070E015C0DE236EC39
:106B3000F2F0EF9E36ECF2F0EF500E0803E136EC87
:106B4000F2F0EF6A012AF0D712C1A4F10A0E010196
:106B50001303F35014259A6F0A0E1503F3501625EC
:106B60009B6F0A0E1703F3CF9CF19E6B9EC19DF1A4
:106B7000040E02018D5D0DE27E510BE115C1A4F101
:106B80000A0E01011603F35017259A6F9C6B9CC1E6
:106B90009BF102017E0508E114C1A4F19BC19AF1A9
:106BA0009CC19BF101019C6B020E02017E5D0EE116
:106BB00013C1A4F10A0E01011403F35015259A6FB5
:106BC0000A0E1603F35017259B6F9C6B9A0E086EE6
:106BD000D7EC0DF0006E005013E10101A45103E168
:106BE0009A51370802E2268E12005FECE8F00A0E96
:106BF000005C06E10101DD51010B02E03CEF09F010
:106C000000C02CF12EECE7F09DEC04F058EC0BF0FA
:106C1000FBECEDF0AFECE7F0A8ECF3F09A0E4A18BD
:106C200007E14B5005E1189A189853DA0C0E086EDC
:106C300012008C9804902EB00480695003E00490F8
:106C40002FBC04803F0E07013715006E04A002D050
:106C5000008C01D0008E01018EA102D0300EC66ED4
:106C60000050E66E13EC7AF0E55236C7E6FF13ECFF
:106C70007AF0E55239C700F0040E0002F3CF00F0BD
:106C8000070138BF0082070138BD008038C701F016
:106C9000040E0102F3CF01F0070137BF01820701A3
:106CA00037BD018004A002D0008C01D0008E0050BE
:106CB000E66E13EC7AF0E5520150E66E13EC7AF0D2
:106CC000E5520470200E006E04A002D0280E006E63
:106CD0000050E66E13EC7AF0E552080EE66E13EC07
:106CE0007AF0E5528C880000310EC66E695004E1DE
:106CF0002E9004B02E8003D02F9C04B02F8C120055
:106D0000010178B71FD024EC7AF0080E69244A6E8E
:106D1000F00E8C144A108C6E96EC5EF08A9A00008D
:106D2000E8EC08F0210EE66E13EC7AF0E552080E5E
:106D3000E66E13EC7AF0E5527CDF8A8AF00E8C1650
:106D400020EC7AF01200010178B71BD002010D6B24
:106D500024EC7AF0080E69244A6EF00E8C144A1066
:106D60008C6E96EC5EF08A9A000063DF37C73AF7C4
:106D700038C73BF78A8AF00E8C1620EC7AF00DC2E9
:106D80000EF212006950020DF3CF5BF7F4CF5CF7FF
:106D9000530E07015B27070E5C236950020DF3CFEA
:106DA00065F7F4CF66F75D0E6527070E66230101D0
:106DB0009A51C80D43ECE5F09B51020D4A50F32463
:106DC0000F6E4B50F420106E9C51310803E20F2AD5
:106DD000000E1022CC0E0F5E060E105AD8EC09F0F1
:106DE000006E005012E000501FECF2F0400B03E187
:106DF0002850040B0AE00050E66E5AEC0EF0E55203
:106E00000050310802E2AFECE7F0010EE66E8DECC7
:106E100098F0E552320E4B6E4BC044F09CC13FF0EF
:106E20002FECFDF03BC04AF00A0E4C6E4CC044F013
:106E30004AC03FF0D1ECF0F0056E23ECE8F0EE50E4
:106E4000ED103CE00150055C44E30F2A000E1022D7
:106E50000201C8510F1812E1C95110180FE123ECBB
:106E6000E8F0CAC2EEFFCBC2EDFF4FECE7F0CCC2B8
:106E7000EEFFCDC2EDFFCEC201F01AD0E66A8DEC76
:106E800098F0E5520201A007000EA15B23ECE8F0A8
:106E9000EECFCAF2EDCFCBF24FECE7F0EECFCCF273
:106EA000EDCFCDF201C0CEF20FC0C8F210C0C9F2D2
:106EB00023ECE8F0EE50ED100CE109D005504A6EDD
:106EC0004B6A4FECE7F04A50EE264B50ED22FCECBB
:106ED00098F02E9A19ECF1F0570EE926070EEA22E7
:106EE0008EECEAF023ECE8F0EECF4CF0EFCF4DF073
:106EF0004C504A1819E14D504B1816E119ECF1F0BD
:106F0000610EE926070EEA22EECF4EF0EFCF4FF0EA
:106F10004FECE7F0EECF50F0EFCF51F050504E185D
:106F200002E151504F181AE02E8A23ECE8F08EEC63
:106F3000EAF019ECF1F0570EE926070E8EECEBF0B3
:106F40004FECE7F08EECEAF019ECF1F0610EE92677
:106F5000070E8EECEBF0040EDBECEBF012000C0EE7
:106F600069244A6EF00E8C144A108C6E96EC5EF01A
:106F70008A9A00006950E96EEA6AD890E936EA36E2
:106F8000530EE926070EEA22EECF0FF0EDCF10F0F8
:106F9000E8EC08F0E66A13EC7AF0E55200011050D4
:106FA000040DF350006E060E0FC0E7FF070B04E060
:106FB000E742E79EE806FCE1E7500010E66E13ECBE
:106FC0007AF0E55200010F50040DF350E66E13EC19
:106FD0007AF0E552F2EC08F06950E96EEA6AD8906E
:106FE000E936EA365D0EE926070EEA22EECF0FF00B
:106FF000EDCF10F0E8EC08F010C0E6FF13EC7AF0EB
:10700000E5520FC0E6FF13EC7AF0E552010EE66E92
:1070100013EC7AF0E552F2EC08F08A8A00000000E6
:10702000F00E8C161200D9CFE6FFE1CFD9FF010197
:1070300078B74BD0FE0EDB5001E0A4DEFD0EDBCFB7
:107040008FF20C0E69244A6EF00E8C144A108C6E6E
:1070500096EC5EF08A9A0000E8EC08F0FD0EDB404A
:107060007F0B4A6EFD0EDB50040DF3504A10E66EA6
:1070700013EC7AF0E552FD0EDB40E8403F0B800D4B
:10708000F350006E0050E66E13EC7AF0E552070103
:107090005139F00B006EFE0EDB5003E0030E0012C0
:1070A00001D000820050E66E13EC7AF0E552F2EC6B
:1070B00008F0FE0EDB5002E052DF07D000000000B7
:1070C0008A8A00000000F00E8C16E552E7CFD9FF47
:1070D000120086D8CEEC3EF02682248A120053C2DB
:1070E000A3F154C2A2F155C2A1F10101A06B9F6BA3
:1070F00020A402D0A8EF3AF0CCEF3AF013C201F08E
:1071000014C202F015C203F068EC44F002011351FE
:10711000015C06E11451025C03E11551035C04E0DB
:10712000B5EC45F099EC5EF01200AFECF4F0010123
:107130008EA715D0FE0EDB5008E0FD0EDB5005E1FA
:10714000DF68CAA102D0010EDF6EFE0EDB5007E140
:10715000FD0EDB5004E0010EDF6ECAB1DF68DF50C8
:107160001FE0A3ECE5F0A36BA3C1A0F1A3C19FF1C5
:107170006AECF2F0D1ECE8F002E0000E01D0010E72
:107180004A6EDF0402E0000E01D0010E4A1802E050
:10719000DFD901D001DA9DEC04F0CAECECF03B81C0
:1071A000E552DEEFE4F00101A36BA26BA16B0201DB
:1071B000B351E8244A6E640EAFECE6F03BC0A0F198
:1071C000320E38ECF0F0B3C23FF02FECFDF03FC0D0
:1071D0009FF10201B4A102D0A8EF3AF0CCEF3AF04F
:1071E00008AE6ED02C50400B03E02D50200B31E048
:1071F000800E0101BF1507E1BF510EE10301E3510C
:107200000101C05D09E2BF6BE3C3C0F1C36BC3C141
:10721000C2F1C3C1C1F11DD0100E2C5D1AE2360EB1
:10722000BF5D03E3360EBF6F0DD01E0EBF5D11E3D1
:107230002C0EBF5D0EE2250EBF5D02E21E0E01D0D8
:107240002C0EBF6FC36BC3C1C2F1C3C1C1F1C3C1B7
:10725000C0F12C50400B03E02D50200B31E1800E8B
:107260000101C41507E1C4510EE10301E35101011D
:10727000C55D09E2C46BE3C3C5F1C86BC8C1C7F102
:10728000C8C1C6F11DD0100E615D1AE2360EC45D94
:1072900003E3360EC46F0DD01E0EC45D11E32C0E39
:1072A000C45D0EE2250EC45D02E21E0E01D02C0E5E
:1072B000C46FC86BC8C1C7F1C8C1C6F1C8C1C5F1A8
:1072C000EDECE8F023E2E051040B20E0BF511D0893
:1072D00009E2DE51200B03E0DE51400B0FE0DE8BB4
:1072E000230E08D0DE51200B03E1DE51400B06E0F7
:1072F000DE9B110EE66ED2EC08F0E55249ECE9F0A7
:1073000005E02C51615D02E1BFC1C4F12C50400B7E
:1073100003E02D50200B23E02150400B09E11350D6
:10732000080B06E02E50400B12E0CA51100B0FE183
:107330002150400B12E02050020B03E11350040BCC
:1073400006E12050020B09E01350080B06E0A3EC05
:10735000E5F0C5DEE5ECE9F002D0F0ECE9F02C5008
:10736000400B03E02D50200B25E12150400B03E0A2
:107370001950400B09E01350080B06E02E50400B4B
:1073800009E1AAECEAF006E12050020B11E01350EB
:10739000040B0EE079ECE7F0A2DE9AC1BAF19BC1D2
:1073A000BBF19CC1BCF19DC1BDF19EC1BEF102D03B
:1073B000FBECE9F001017851040B09E0800E0814A0
:1073C00006E0100E2C5D03E20301280EE76F20504B
:1073D000020B19E10201B451010B03E1B451020B9C
:1073E00012E0050E0C5C07E02150800B0CE0050E4E
:1073F0000101995D08E12150400B05E084ECE7F0C4
:10740000D2DEE5ECE9F02E50400B01E0A0D02C508C
:10741000400B04E1C9ECE8F001E199D02CC100F087
:107420002C50400B05E02D50200B02E161C100F013
:10743000800E081401E18BD0100E005C01E387D0B0
:1074400020EC11F02DBA0DD006ECEAF0C4C19FF18A
:10745000C5C1A0F1C6C1A1F1C7C1A2F1C8C1A3F1C4
:107460000CD084ECE7F0BFC19FF1C0C1A0F1C1C155
:10747000A1F1C2C1A2F1C3C1A3F15FECE8F0010127
:10748000E951200B54E10B0E005C51E22D50200B12
:1074900003E000502C5D06E12D50200B48E1005028
:1074A000615D45E02DAA0BD000C00FF100C02CF1AA
:1074B00060B70FD000C010F100C061F10AD000C069
:1074C00010F100C061F160B704D000C00FF100C03E
:1074D0002CF12CC1CEF159EC0FF02CC1E6FFE6687F
:1074E000FBEC46F0E552E552056E010160B70FD0A6
:1074F0002DAA06D0050EE66E05243FECE9F005D076
:10750000050EE66E055093ECEAF00FECE5F00E0E7A
:1075100005249CECE5F00101CD9B00BACD8B0A6AF5
:10752000B2EC46F021820201010E346F12002050AD
:10753000010B03E02D50200B09E13150020B07E055
:107540002D50200B04E13C51100B01E0D7DD12005F
:107550000101A3519E279E51090803E20A0E9E5F76
:107560009D2BA2519D279D51090803E20A0E9D5FA4
:107570009C2BA1519C279C51630803E2640E9C5FE5
:107580009B2BA0519B279B51630803E2640E9B5FDA
:107590009A2B9F519A2712000101A3519E5F9E5181
:1075A0000A0803E20A0E9E279D07A2519D5F9D5186
:1075B0000A0803E20A0E9D279C07A1519C5F9C517B
:1075C000640803E2640E9C279B07A0519B5F9B51BC
:1075D000640803E2640E9B279A079F519A5F12008A
:1075E000F00E8C140F098C6E96EC5EF08A9A0000F7
:1075F00018C7E6FF13EC7AF0E552E8EC08F0F2EC7D
:1076000008F08A8A12002D9069500701196F1A6BD1
:10761000170E07011927070E07011A23470E4A6E96
:1076200019C7E9FF1AC7EAFF4A50EF126950EA6A20
:107630002F0FE96E070EEA22EFCF33F7070133A1D0
:1076400005D019C7E9FF1AC7EAFFEF94070133A372
:1076500005D019C7E9FF1AC7EAFFEF92070133A562
:1076600005D019C7E9FF1AC7EAFFEF90070133AD4C
:1076700005D019C7E9FF1AC7EAFFEF9C0E0E69246F
:107680004A6EF00E8C144A108C6E96EC5EF08A9A5C
:1076900000006950EA6A170FE96E070EEA22EF5000
:1076A000E66E13EC7AF0E552E8EC08F0F2EC08F044
:1076B00082A82D808A8A1200A6DF050E64EFE5F00D
:1076C000D9ECE4F0010178B73ED0B6ECE7F0EFCFAB
:1076D00033F7FE0EDB5006E1470E11ECEAF0470BE4
:1076E0004A5C01E090DFFE0EDB5006E1380E11EC43
:1076F000EAF0380B4A5C21E069500701196F1A6BF8
:10770000170E1927070E1A23570E4A6EFFECEBF0DF
:107710004A50EF1633A703D0FFECEBF0EF8633A906
:1077200003D0FFECEBF0EF8E33BB03D0FFECEBF0BC
:10773000EF8AC2DF010E52ECE6F070ECF2F033C7D4
:10774000EFFFF00E8C16DEEFE4F00701040E506F31
:10775000D890403341334233433344334533463387
:107760004733502FF6D71200010178B7120019ECF9
:10777000F1F0530EE926070EEA22EECF67F7EDCFC0
:1077800068F719ECF1F05D0EE926070EEA22EECF5C
:1077900069F7EDCF6AF7030E07013C156B6F6C6B51
:1077A000020ED8903F333E333D333C33E806F9E1D7
:1077B00067C74AF068C74BF09AECE6F073ECFAF052
:1077C0003BC0EDFF3AC0EDFF39C0EDFF38C0EFFF21
:1077D00069C74AF06AC74BF09AECE6F096ECFBF00A
:1077E0003FC0EDFF3EC0EDFF3DC0EDFF3CC0EFFFF1
:1077F00038C06DF739C06EF7020E0701D8903C37DC
:107800003D373E373F37E806F9E1020E0F0B07011F
:1078100005E0D89068336733E806FBE1020E0F0BF2
:10782000070105E0D8906A336933E806FBE16BC7CE
:107830003EF06CC73FF067C743F068C744F096EC72
:10784000F8F03C5007016D254A6E3D506E214B6E9D
:10785000060E50ECE8F0B4ECF0F069C743F06AC7EC
:1078600044F0C9ECEFF00701020E486FF10E496FCA
:107870000301C95107E009ECE8F0D5C14AF7D4C1CA
:107880004BF704D051C14AF750C14BF73FC740F7FF
:107890003EC741F73DC742F73CC743F70701476B77
:1078A00047C746F747C745F747C744F74EDF13ECCE
:1078B00027F044C739F745C738F746C737F747C7F2
:1078C00036F700010F50070136270001105007015D
:1078D0003723000E382339231200B0ECEFF00050AC
:1078E000016E020E64ECE5F0B0ECEFF00050026EB9
:1078F000010E64ECE5F0B0ECEFF0040EE66E2FEC58
:10790000EEF0D1ECE6F009E0040E03ECEFF00250EB
:10791000E66ED1ECE6F001E0010C000CAFECF4F007
:10792000F00E8C1669288C121C84B0ECEFF0070165
:107930003551005C15E23451005C12E322A20CD0F8
:107940002292CBDF000902E0DF2A0AD03C0E64EC71
:10795000E5F0C3DF000903E0010EDF6E01D0DF6A4E
:107960001C94F00E8C16DF50E552DEEFE4F0695007
:10797000E8247F0F10240A6E0F50016E1200D9EC1C
:10798000E4F0090EE1260F6A106A770E0F5C010E13
:10799000105808E2ECDF0068FDEC4CF00F2A000EF6
:1079A0001022F3D7E66A67ECE9F00701336B335135
:1079B00053ECE5F002E647ECE7F001E339D1B6EC31
:1079C000E7F033C7EFFF9AECEBF00C0E52ECE6F069
:1079D0001F0E17ECEFF075ECE7F033C700F084EC06
:1079E00096F01AA802D0FFEC04F069EC95F033C7CA
:1079F00000F0620EDE6EDD6A560E3EECE6F0030E1F
:107A0000DB6A400E005C63E2DC0E3AECEDF0005005
:107A10002F0803E2AA0E3AECEDF0200E005C09E21A
:107A2000CC0ED0ECEAF00050070803E27C0ED0EC5C
:107A3000EAF0080E00C0DBFF800E00244A6E4B6A9D
:107A4000000E93ECEFF00A0D020EF3CFDBFF030EF6
:107A5000F4CFDBFF080EDB50006E3C0E4CECE6F082
:107A6000090E005C03E2500E4CECE6F000501808E2
:107A700008E2210E005C05E2020EDBCFDEFFDBCF69
:107A8000DDFF0050240803E2280E4CECE6F0CFECBA
:107A9000E7F0CC0ED880EE54010EED5404E2CC0E8B
:107AA000DE6E010EDD6E040EDBCF4AF0050EDBCF7D
:107AB0004BF0DECF4CF0DDCF4DF04C504A5C4D50DA
:107AC0004B5805E2040EDBCFDEFFDBCFDDFFCFEC52
:107AD000E7F0060EEECFDBFF070EEDCFDBFF4CEC41
:107AE000EAF0020EDBCF4CF0030EDBCF4DF04A5034
:107AF0004C5C4B504D5801E398D0180E0701335D94
:107B000012E1D950060FE96EDACFEAFFDE0ED88017
:107B1000EE54000EED5407E24CECEAF0E30EACEC50
:107B2000F3F001E27BD00A0E4A6E4B6A060EDBCF01
:107B30003EF0070EDBCF3FF089ECE5F03EC09AF156
:107B40003AC09BF10A0E01019B03F3CF9BF19E6BA0
:107B50009EC19DF19EC19CF1C2EC36F0AFEC37F0B6
:107B6000060EDBCF3CF7070EDBCF3DF707013E6B80
:107B70003F6BA00E416E860E426E010E436E446A4C
:107B80003CC73CF03DC73DF03EC73EF03FC73FF02D
:107B900073ECFAF038C03CF739C03DF73AC03EF715
:107BA0003BC03FF7E1DDA3EC36F0040E52ECE6F00B
:107BB0000701C80E356F250E346F4CECEAF0620EEB
:107BC000ACECF3F002E21C0E346F1AA803D0060EE0
:107BD000355F34272282A2DE00091BE0060EDBCFD0
:107BE0000FF0070EDBCF10F041ECEDF033C700F0E3
:107BF000FDEC4CF0D950060FE96EDACFEAFFCC0E5F
:107C0000EE180CE1010EED1809E1012AFDEC4CF033
:107C100005D007013451D880005407E2060EDB0678
:107C2000070E01E35CD7DB065AD70701332BBFD61B
:107C30000C0E346FDD0E356F760E0F6E010E106E6A
:107C4000040E57ECE6F023E292DE3CEC4DF080ECC3
:107C500098F0FF0E005C07E1420E77ECE5F00FC0F4
:107C600029F710C02AF7450E0F180DE110500BE14F
:107C7000280E005C03E300502A0805E2450E77EC6D
:107C8000E5F000C02BF70F06000E105AD9D7D0EC44
:107C900010F00201800E8A6F69EC38F0090EE15C89
:107CA00002E2E16AE552E16EDEEFE4F0B6C101F016
:107CB000B7C102F00101000E0D6F0D0E0E6F0A012B
:107CC000D751040DF3500C10036EBDEC0CF0066E92
:107CD0000C5004E1B2ECEAF001E00686030E0C5C05
:107CE00004E17850080DF350061212000A01040E48
:107CF000DE6FDF69695005E10C50030802E3E051D3
:107D000001E1000CD3DF0A01DF6BE051DF5D30E2FF
:107D100029ECF0F0EF50015C23E10101BEECE6F04C
:107D2000EF50025C1AE1BEECE6F0EF50035C12E1AA
:107D3000BEECE6F0EF50006E1F0E0014065C07E18B
:107D40000050E00BE838E8400A01DE6F010C0D0737
:107D5000000E0E5B0D07000E0E5B0D07000E0E5B96
:107D6000040E01010D27000E0E230A01DF2BCDD7D3
:107D7000DF69000C0301C95107E009ECE8F0D4C148
:107D800020F1D5C121F104D050C120F151C121F120
:107D90000101F10E226F020E236F12004CECEFF086
:107DA00034BC39D02CBC1AD0696A38D82550100B95
:107DB00004E10101E351400B0CE0800E081403E0E4
:107DC0003050800B03E01950400B03E0010E696E48
:107DD00025D8309E21BC20D0199C1ED02DAA08D0B9
:107DE0002150400B03E02050020B16E1696A13D0CA
:107DF0002150400B09E149ECE9F003E1E351400B6C
:107E000003E0010E696E0AD82150400B05E02050B6
:107E1000020B02E0696A02D854EFEFF04CECEFF08D
:107E20000101080E9A6F150E9B6FF40E0F6E010E76
:107E3000106E2150400B06E082ECE6F003E0B0C289
:107E400001F003D0BDEC0CF0016E0150E66E41EC88
:107E5000EAF04A6E4B6A4ABE4B684A500001DFECBA
:107E6000EEF09FEC04F001019C6F3AC09DF19E6B17
:107E7000A36BA3C1A2F1A3C1A1F1A3C1A0F1A3C1AE
:107E80009FF12150400B04E082ECE6F001E1FAD0D2
:107E9000695017E03450400B14E10CC05DF2CBC1C7
:107EA0005EF2D7CA5FF25BC261F25CC262F27D50E1
:107EB0000C6ED7C1CBF160C2D7FA63C25BF264C269
:107EC0005CF20C5005E0030E0C5C30E178502EE0C3
:107ED000D7ECEEF05BC23EF05CC23FF089ECE5F01F
:107EE0003EC0A1F17CECE5F03AC03FF02FECFDF094
:107EF0003FC0A2F15BC24AF05CC24BF00A0E77ECC5
:107F0000F2F04AC0A3F11FEC12F0000903E1CCEC3F
:107F10003AF002D0A8EC3AF058ECE7F023E047EC56
:107F2000EDF01FEC12F0000918E01AD0040E0C5C02
:107F300019E296EC04F001010F0EA16F1CECF1F0B8
:107F4000780E4A1804E14B5002E1100EA1270C04F0
:107F500004E06AEC11F0010803E1CCEC3AF002D045
:107F6000A8EC3AF069500EE1C1DE000902E01C8A7B
:107F700003D01CAA07D01C9A6CEC1AF0E66A5EECDF
:107F80004BF0E552BAECEAF005E11C50200B3FE063
:107F900069503DE1D751DE25FC0FE16F190EE15D1F
:107FA000056E190EE15D04E2190ED880E155056EEB
:107FB0000701EFAF07D07CECE5F005C03FF045ECE2
:107FC000EAF00AD00550FE0BE8420101A16FA26B56
:107FD00005A002D0050EA26F0C040BE00C5003E1CB
:107FE000B2ECEAF006E0030E0C5C08E1F7ECEEF010
:107FF00005E10A01E151190808E304D00A01E15141
:10800000190803E2A8EC3AF002D0CCEC3AF069503F
:1080100023E034BC0AD05DC20CF05EC2CBF15FC27B
:10802000D7FA61C25BF262C25CF20101E39702011E
:10803000D55101019B5D0FE10201D65101019C5D0B
:108040000AE10201D75101019D5D05E10201D8510C
:1080500001019E5D01E0E387695045E1020129517C
:1080600006E0D65101019C5D02E005013B859AC105
:10807000D4F29BC1D5F29CC1D6F29DC1D7F29EC16C
:10808000D8F231D0FBEC26F0016E6AEC11F0026EF2
:10809000010405E0020E015C02E0025014E002500F
:1080A00002E00250016E01010F0EA16FE3ECEEF051
:1080B00003E0100E0101A12735AC02D06AECF2F00A
:1080C00001040CE00ED0030E015C0DE158ECE7F06A
:1080D00002E047ECEDF0F7ECEEF003E1CCEC3AF027
:1080E00002D0A8EC3AF02CC100F0695005E0345001
:1080F000400B02E161C100F000500A0801E3A8D082
:10810000100E005C19ECE8F043ECF4F001E185D0CE
:10811000B9ECF4F001E181D02DDEA00E0101205D6B
:108120007A0E2159F10E2259020E235918E2A00E9F
:108130004E6E7A0E4F6EF10E506E020E516E205141
:108140004E5C4A6E21514F584B6E2251505823516C
:1081500051584AC0D2F14BC0D3F1006A15D020C1AA
:108160004AF021C14BF022C14CF023C14DF0A00ECA
:108170004A5E7A0E4B5AF10E4C5A020E4D5A4AC0C4
:10818000D2F14BC0D3F10068590E0F6E020E106E83
:10819000DEAB04D0640E0F6E020E106E0FC04EF0F8
:1081A00010C04FF0506A516A2AECEEF04C6A4D6AEA
:1081B00033ECF1F04EC041F04FC042F050C043F0FC
:1081C00051C044F073ECFAF038C020F139C021F10D
:1081D0003AC022F13BC023F1010121C120F122C1AB
:1081E00021F123C122F1236BC1EC96F00101A06BB8
:1081F000A0C19FF104C13CF504C1A1F105390F0BE9
:1082000005013D6F0101A26F0F0E051505013E6FBF
:108210000101A36F00C03FF514D087EC08F0010105
:10822000A06BA0C19FF1F6ECF2F0A16F050EEB5030
:10823000A26FA36B006AEF50010B01E0006887ECAE
:1082400008F0005003E0CCEC3AF002D0A8EC3AF091
:108250009AC19FF19BC1A0F19CC1A1F19DC1A2F166
:108260009EC1A3F1695007E12050020B0AE02150A2
:10827000400B0AE106D03450400B03E1C9ECE8F0B2
:1082800003E084ECE7F002D006ECEAF00101DE51F5
:10829000200B07E0695003E02C51615D02E1020E02
:1082A0009A5FE3BD27D01A9E695004E02E50400B20
:1082B00001E11A8ED1ECE8F003E0A8EC3AF002D02C
:1082C000CCEC3AF0695016E001013851080B12E08D
:1082D0003C51100B0FE10A0E9A6F330E9B6F1E0E6E
:1082E0009C6F9E6B9EC19DF178A704D0050E9A6F7E
:1082F000370E9B6F01017851080B2CE02150400B89
:1083000029E1016A3851080B0BE03C51100B08E0E1
:108310008B51400B05E0E351080B02E1020E016EA8
:10832000696A430E3AECE9F0010E016E49ECE9F09E
:1083300003E1E351400B07E08B51400B03E0E351B5
:10834000080B01E0016A010E696E430E3AECE9F098
:10835000DF50696E010178A71DD09AC1E6FF46EC97
:10836000E8F0016E9BC1E6FF46ECE8F0026E9CC1AE
:10837000E6FF46ECE8F0036E0A0E01019D03F350A0
:108380009E25E66E46ECE8F00101076F460EE66EAC
:10839000D5D8D0D09B514A6E4B6A0A0E98ECF4F0B7
:1083A00001019A510A0DA8ECE7F0010E0F26000E0C
:1083B000102241ECEDF03CEC4DF00A6A270E005C17
:1083C00006E1460E0F1803E1105001E1002AB6EC59
:1083D000E7F0EF50005C0AE02A50040B07E1040EBE
:1083E000DBECEBF0B6ECE7F000C0EFFF2A94C2EC58
:1083F00036F02EAA09D008AE03D0AFEC37F004D087
:10840000E6C2E6FFBDECE7F09AC14AF04B6A4C6A5F
:108410004D6A400E416E420E426E0F0E436E5CEC92
:10842000E7F09BC14EF04F6A506A516A100E416EE0
:10843000270E426E436A446A4EC03CF04FC03DF086
:1084400050C03EF051C03FF073ECFAF038C04EF02F
:1084500039C04FF03AC050F03BC051F025ECEBF082
:108460009CC152F0536A546A556A640E416E426A66
:10847000436A446A52C03CF053C03DF054C03EF0E1
:1084800055C03FF073ECFAF038C052F039C053F0E9
:108490003AC054F03BC055F052504A2653504B223C
:1084A00054504C2255504D229DC156F0576A586A7F
:1084B000596A0A0E416E426A436A446A56C03CF0E9
:1084C00057C03DF058C03EF059C03FF073ECFAF091
:1084D00038C056F039C057F03AC058F03BC059F098
:1084E00056504A2657504B2258504C2259504D2234
:1084F0009EC15AF05B6A5C6A5D6A4A505A24070161
:108500003C6F4B505B203D6F4C505C203E6F4D509C
:108510005D203F6FB4EC3BF0A3EC36F002018A51D2
:1085200009ECECF008E14B5006E125BC04D0E66A0A
:1085300060EC3BF0E552E552DEEFE4F0D9CFE6FF28
:10854000E1CFD9FF02010D6B24EC7AF001010101AA
:108550008E51010B07E001010101E351040B02E11F
:10856000300EC66E0C0E69244A6EF00E8C144A1042
:108570008C6E96EC5EF08A9AE8EC08F0FE0EDBCF8B
:10858000E6FF13EC7AF0E552FE0EDB50006EFE0EB5
:10859000DB50530807E00150E66E13EC7AF0E55229
:1085A00001500026FE0EDB50460804E0FE0EDB50B4
:1085B000560815E10250E66E13EC7AF0E5520350CE
:1085C000E66E13EC7AF0E55207C1E6FF13EC7AF0A1
:1085D000E55200500224032401010725006EFF0E1E
:1085E0000002F350E66E13EC7AF0E552FE0EDB501B
:1085F000530806E1C950006EE66A13EC7AF0E552C2
:108600008C880000000000000000310EC66E8A8ACF
:10861000F00E8C1620EC7AF0E552E7CFD9FF12006D
:10862000D9CFE6FFE1CFD9FFB5C19AF1B6C19BF131
:10863000B7C19CF1B8C19DF1B9C19EF10101A46B14
:10864000FE0EDB500A0807E22A96FE0EDBCFE6FF9D
:10865000C6EC34F0E5520101006B800E01011615E5
:10866000036E800E01011315026E010EEA6E9A511F
:1086700005D89B5103D89C5101D814D0076B066FC5
:108680000A0E065DD8A003D0066F072BF9D700515C
:10869000110FE96E0751EF6EE92A0651EF6E002BBC
:1086A000002B000C04D8E552E7CFD9FF12009DC182
:1086B00017F19EC118F10101A45105E10A0E9A5D5E
:1086C00002E2100E116F0701EFBB03D00101100E83
:1086D000186F0701EFAD05D00101100E176F17C11C
:1086E00018F11EBC03D00101138F03D00250010109
:1086F000131361EC0BF0000903E10101168F03D0A5
:10870000035001011613A45109081AE2020149514C
:1087100017E0A3EC93F00101020E006F9AC100F084
:1087200084EC96F0A4C100F00101006B84EC96F09B
:10873000010EE66EE66A84EC09F0E552E55212009D
:108740000101A45118E00701EF51200B14E1298C1D
:1087500017C118F116C117F115C116F114C115F1A1
:1087600013C114F112C113F111C112F17EECF2F038
:108770003BC011F11200299C1200D9CFE6FFE1CFD6
:10878000D9FF020EE126010EA4C1DBFF2EAC0FD0F3
:108790002CC1DFFFEFC7F0F7B5C19AF1B6C19BF16D
:1087A000B7C19CF1B8C19DF1B9C19EF114D061C1AE
:1087B000DFFF7D50EA6AE90FE96E070EEA22EFCF8C
:1087C000F0F7BAC19AF1BBC19BF1BCC19CF1BDC12C
:1087D0009DF1BEC19EF10101A46BDF500A0806E2C3
:1087E0002A96DFCFE6FFC6EC34F0E5520101016BBB
:1087F000800E01011E15026E010EEA6E9A5105D817
:108800009B5103D89C5101D816D0076B066F0A0EF6
:10881000065DD8A003D0066F072BF9D70151190FB9
:10882000E96E0751300FEF6EE92A0651300FEF6EF7
:10883000012B012B000C010EDBCFE6FF0BD8E5521C
:10884000020EE15C02E2E16AE552E16EE552E7CF39
:10885000D9FF1200D9ECE4F0300E01019D251F6F05
:10886000A45105E10A0E9A5D02E2200E196F07017C
:10887000F0AD03D00101200E1F6F01011B8F6FECC3
:108880000BF0000903E101011E8F03D0025001012A
:108890001E13A45116E00701F051200B12E11EC176
:1088A0001FF11DC11EF11CC11DF11BC11CF11AC11C
:1088B0001BF119C11AF17EECF2F03B50300F0101AF
:1088C000196FA4C1A5F1FE0EDBCFA4F1DEEFE4F039
:1088D000E66A08D8E55231A204D0010EE66E02D84D
:1088E000E5521200D9ECE4F0050EE126FE0EDB5055
:1088F0000CE1BFC1DFFF010EC0C1DBFF049020B05F
:108900000480040E2CC1DBFF0ED0C4C1DFFF010EBA
:10891000C5C1DBFF049031B20480030E15C2DBFF3A
:10892000040E61C1DBFF020EDB6A0450010B01E1A2
:1089300004D11C0EDF5C01E300D1100EF36E040EB7
:10894000DBCFF4FFF350F45C01E3F7D00E0EDF5CF5
:1089500001E383D0070EDF5C48E2030EDF5C16E222
:10896000020EDF5C0DE2DF5005E0460E15ECE5F08F
:1089700001E3E3D0800E3EECE6F00201400EBCD0F5
:10898000010EDB500A0801E3D8D00BD0050EDF5CE6
:1089900015E2030EDF5C0BE11E0E15ECE5F001E3C2
:1089A000CCD0C00E3EECE6F00201800EA5D0010E48
:1089B000DB50140801E3C1D0100E23D00201080ED1
:1089C000156F050EDF5C0AE1190E15ECE5F00BE3FF
:1089D000010EDB50320801E3B0D005D05A0E15EC81
:1089E000E5F001E3AAD0100EA6D0090EDF5C16E276
:1089F000070EDF5C09E1010EDB50280801E39DD082
:108A0000300E3EECE6F007D0300E3EECE6F0280EDD
:108A100015ECE5F032E20201080E6ED00201200EE4
:108A2000156F090EDF5C07E1550E15ECE5F001E36B
:108A300084D0300E80D00D0EDF5C09E20A0EDF5CC0
:108A40000AE1010EDB50140801E377D004D03C0E9C
:108A500015ECE5F072E2080E6ED0160EDF5C37E220
:108A6000120EDF5C18E20E0EDF5C0AE1010EDB5035
:108A70003C0863E20C0E3EECE6F00201200E3CD016
:108A8000110EDF5C04E3460E15ECE5F056E20C0E29
:108A90003EECE6F029D00201100E156F120EDF5CDD
:108AA00005E1010EDB50280848E20FD0130EDF5C11
:108AB0000CE0140EDF5C05E15A0E15ECE5F03DE22A
:108AC00004D0010EDB50320838E2010E34D0180E0B
:108AD000DF5C14E2160EDF5C0AE1010E3EECE6F00C
:108AE0000A0E15ECE5F006E20201100E05D0030EA9
:108AF0003EECE6F00201040E156F1FD00201040ED9
:108B0000156F180EDF5C05E1320E15ECE5F015E28D
:108B10000BD0190EDF5C05E1010EDB5032080DE2CF
:108B200003D01A0EDF5C02E1030E05D0460E15ECF1
:108B3000E5F003E2030E3EECE6F0FE0EDB50EA6ADF
:108B4000130FE96E020EEA22020EDBCFEFFFFE0EDC
:108B5000DB5003E0030EDBCF15F2050EE15C02E211
:108B6000E16AE552E16EDEEFE4F007010A6B1F0EE9
:108B70000B17116B0D6B0DC70CF7030E06171F0EAD
:108B80000717096B09C708F72CC100F0EDECE8F0F6
:108B900002E20FC100F00201135103E02050010B6B
:108BA00047E100500A0A3FE0030A39E0010A35E0D4
:108BB0000F0A2DE0010A27E0030A20E0010A1BE06A
:108BC000060A14E0010A0FE0020A08E0010A36E191
:108BD0000701118D11830A890B8B30D00701118F8A
:108BE00011830A892BD007010B8D02D00701118355
:108BF00011870A8B23D007010B8D11830701118385
:108C0000118B0A8D1BD007011189118304D0070134
:108C1000118311890B8F0A8F11D007010B8F070168
:108C200011850A870BD00701118311850A8506D0AB
:108C3000E66A00EC15F0E55215C211F72CC100F000
:108C400000500A0802E20FC100F0010160A707D03E
:108C500061C100F000500A0802E210C100F00201F8
:108C6000145103E03150020B35E100500A0A2FE0A5
:108C7000030A2AE0010A26E00E0A21E0010A1DE0AB
:108C8000020A18E0010A14E0060A0FE0010A0BE0EC
:108C9000020A06E0010A23E107010689078B1FD0BB
:108CA000070106891CD00701078D0701068B17D025
:108CB0000701078D0701068D12D00701078F0701F5
:108CC000068F0DD00701078F0701068708D007011F
:108CD000068505D0010EE66E00EC15F0E5520101A7
:108CE0003CB905D0FC0E07010613E00E071305EF93
:108CF0000CF032EC0EF02C50040B08E0005009ECA4
:108D0000E6F0EF50020B02E125EC0EF0258A12008E
:108D100041ECEFF0830E0A6E0A0EE66E01010F03BE
:108D2000F350E66E740EE66E020E0FECE5F0DE0E0A
:108D30009CECE5F00050DF6EFE0E4BECF4F0010110
:108D4000DF9D2F9EB90E005C05E1FF0E0201745DF0
:108D500001E02F8EA30EDF5C02E10101DF8DE55201
:108D6000DEEFE4F04CECEFF0695034E11950010B08
:108D700031E1CEDF01015751080B03E12C51090805
:108D80000EE228EC05F0FF0805E1800EE66E3AECF5
:108D900005F0E55228EC05F00101496F08D0FF0EFF
:108DA0008D5D03E1320E8D6F02D08DC149F134EC3F
:108DB000F3F02B847EEC28F037EC23F02CA60AD0BD
:108DC000E66ACCECC6F0E5520701169F12B0168F8A
:108DD0008DECC5F0FBECEBF025A808D038EC0DF0DD
:108DE00025A804D0010E696ED0EC10F0696AD0ECB1
:108DF00010F054EFEFF041ECEFF0FD0EDB50100DF2
:108E0000F350DF6E010E0A6E0201680EC26FFD0E96
:108E1000DB500A080AE2020E0A6E690EC26FFD0EEE
:108E2000DB50F00F100DF350DF6E1AECEFF002E0A4
:108E3000E9ECF0F0DF50E552DEEFE4F00201B25170
:108E400003E0B251330802E20D0EB26FB351D5EC1C
:108E5000E5F005E228ECE8F002E21E0EB36FB4BFC5
:108E6000B46B120045ECEFF01AECEFF01BE0E9EC0C
:108E7000F0F00F0E61ECF0F00A0E005C07E101016A
:108E8000DD51010B03E00A6A000E5DD200C02CF137
:108E900001018B51100B06E00A0E48ECE5F002E2EE
:108EA000FE0EDB682CC10FF10101E0A506D0DE9BB0
:108EB000450EE66ED2EC08F0E55202018B6B010123
:108EC000E09532EC0EF0EDECE8F022E2100E2C5DB5
:108ED00038ECF3F079EC05F02EECF0F011E0B9ECA1
:108EE000F0F001010F6FEF380F0B02018B6FAEEC4A
:108EF000E5F0800B03E00101E085DE8DFADE08D0AD
:108F0000FE0EDB680101090E0F6F0FC12CF1268EDA
:108F1000D0ECEFF0100E26ECF1F00F0E0101C915A8
:108F20000C6EC9390F0B7D6E7D50060802E20C50A5
:108F30007D6E0C0401E1CA91020E0C5C01E1CA8154
:108F4000A1ECF3F0786E60B704D02CC161F10FC1D1
:108F500010F161C110F161510A0817E2100E615D54
:108F600038ECF3F02EECF0F005E0B9ECF0F0010194
:108F7000106F08D0FE0EDB680101090E106F10C1E2
:108F800061F1268E61C100F002D02EECEBF00050B2
:108F90000101615D03E12C51615D0FE073ECF1F0C3
:108FA000050EE66EDF243FECE9F00FECE5F00A0E6B
:108FB00061ECF0F000380F0B7D6E040E71ECEEF0FA
:108FC000D60EE66E010E0FECE5F0D0ECEFF01AECE9
:108FD000EFF003E1C2C20AF002D0100EDF26100E3D
:108FE0004FECF4F0F3ECF1F01AECEFF05CE02CC194
:108FF000E6FFE66894ECE6F00B0E61ECF0F0030E91
:109000000C5C09E01F0E0101CA17E00E0014CA1320
:10901000A1ECF3F0786E0050046E0101CA97045081
:10902000080B01E0CA870C0E61ECF0F0440E010160
:10903000CB17BB0E0014CB131EECEFF0070E010193
:10904000CC17F80E0014CC131EECEFF00A0E010141
:10905000CD17F50E0014CD13C2C20AF00D0EE66E48
:10906000030EDF24E66EB50EE66E020E0FECE5F0A1
:1090700073ECF1F00C0E61ECF0F0440E0101D71727
:10908000BB0E0014D7131EECEFF0070E0101D8172A
:10909000F80E0014D8131EECEFF00A0E0101D917D8
:1090A000F50E0014D9130201BBBFBB6B0A6ABFC126
:1090B00007F5C0C108F5C1C109F5C2C10AF5C3C1B0
:1090C0000BF5C4C10CF5C5C10DF5C6C10EF5C7C180
:1090D0000FF5C8C110F519B42DD013941396139A37
:1090E000209201013951020B1CE082ECE6F019E1FB
:1090F0000101CC51010B04E0FDECB8F0000911E1D5
:109100000101CC51010B05E02C51615D02E1138A94
:1091100020821396CCB313861394CCA509D0138464
:1091200007D0F8ECECF00101D895D893CC95CC930E
:1091300008ECC0F0EDECE8F01AE2680E0F2532EC16
:10914000F2F000500101BF5D016E01AE03D0BF51CE
:10915000005C016E015003080AE2050E21ECEFF0FD
:10916000BF0EE66E010ED0ECE5F000C0BFF10101CC
:1091700061510A081AE2680E102532ECF2F0005034
:109180000101C45D026E02AE03D0C451005C026EE8
:10919000025003080AE2050E21ECEFF0C40EE66E61
:1091A000010ED0ECE5F000C0C4F1320E4AECE7F05D
:1091B000300E4AECE7F0F7ECEBF0B3EC2CF053ECAC
:1091C0000EF0139C01013CB1138C139E3CB3138E23
:1091D00084EC7FF0139801013CB913882CA4CC9F38
:1091E0001294CCBF12840701109B12A4108B0201B1
:1091F000BC51030802E3BC5102E1020EBC6F4EEC0D
:1092000027F02CB602D00101CB9F12900101CBBFF9
:1092100012801292CBAF1282B8EC09F001015851C2
:10922000800B05E02C50040B02E025EC0EF0660EDE
:109230000A6E080E01012C03F3289CECE5F000C037
:1092400042F5FF0E005C02E10501426B01063CECB9
:109250004DF0FF0E005C01E1006A7F0E0014050175
:10926000406F01015851100B04E1DD51200B01E169
:10927000CB9B080E6103F350050F9CECE5F000C09A
:1092800043F5FF0E005C02E10501436B01063CEC77
:109290004DF0FF0E005C01E1006A7F0E0014050135
:1092A000416F01015851100B0AE1DD51200B07E11C
:1092B0006051080B03E01C50080B01E0D9910A6AC9
:1092C000010E69CFDBFF3CA905D0696EFDEC68F0AB
:1092D00097EC68F0696AFDEC68F097EC68F015A40B
:1092E00003D00501FA0E446F010EDB50696E6A0E61
:1092F00001010F250A6EF00E9CECE5F0FF0E005CFC
:1093000001E1006A00C0E0FA040E0002F350E66ECC
:10931000E66A000EE66E0D0E0FECE5F00A6A22DD3D
:10932000ACEC0CF0F0ECE9F0FBECE9F0796A1EBC77
:1093300009D00701D36B030E016E2CC100F05DDB79
:109340004EECEDF0010EB6ECEAF002E2E16AE55215
:10935000E16E4A50DEEFE4F041ECEFF00B0E01015C
:109360002C5D0BE2C0C1E6FFBFC1E6FF3CECF3F0B1
:10937000005001012C5D01E0B7D00B0E615D07E2EA
:109380002EECEBF000500101615D01E0ADD00A0E62
:109390002C5D02E249C18DF1D0ECEFF03BEC27F0FF
:1093A0000101CB9F12B0CB8FCC9F12B4CC8F39A3CD
:1093B0000DD0F80ECC17CC9120B2CC81CC9313B643
:1093C000CC83CC9513B4CC8587EC55F02CC1CEF171
:1093D000F2ECF0F0050E93ECEAF04FECF4F039EC1F
:1093E000E5F00A0EDF24016E7D38F00B0C10D5EC91
:1093F000E8F0050EE66ECA0EE66E010E71ECEEF0B8
:1094000039ECE5F0A2ECE9F01BE073ECF1F00A0EA8
:1094100061ECF0F00F0E00160A0EDF24016E7D38AD
:10942000F00B0010D5ECE8F0A2ECE9F009E0040E36
:10943000E66ED60EE66E010E71ECEEF039ECE5F05C
:10944000050E3FECE9F0E66E050EDF2432ECF0F09D
:109450001DBA45D0D0ECEFF001015751080B03E1E4
:109460002C51090805E249C1E6FF3AEC05F0E55246
:10947000E9ECC4F00101CB51800B01E0010E76EC68
:10948000EBF03BC1EFFF1AECEFF003E1C2C20AF0D0
:1094900002D0100EDF2654ECEDF0DFCFE6FF39EC02
:1094A000E5F00A6ABDEC15F0660E0A6E080E0101C1
:1094B0002C03F350016E40C500F09FDA012A42C52B
:1094C00000F09BDA080E01016103F350040F016EF6
:1094D00041C500F092DA012A43C500F08EDA0A6A2B
:1094E0004EECEDF00201306BE552DEEFE4F041ECC2
:1094F000EFF07F0EDF6E3BECE8F007E02D50400B05
:1095000004E12D50800B01E1DF060F0E06010D175F
:10951000DF1C0E17E552DEEFE4F006010D910E9F01
:109520000F99EE0E10171217139914911200F9ECFF
:10953000F3F0DBCFE6FF0FEC14F0E552E71803E0A1
:1095400006010D8F02D006010D8D01013DA502D04F
:1095500006010E8101018BA102D006010E87DEEF0C
:10956000E4F01A9E0050050A01E173D0010A5BE0A5
:10957000070A2AE0010A23E0030A1FE0010A01E0CA
:10958000120006010D8BD1ECE8F002E0000E01D0D4
:10959000010E4A6EB2ECEAF001E0010E4A1802E058
:1095A00006010D890601F051010801E20E83010157
:1095B0008FAD63D006010E871200E66A02D0010E5D
:1095C000E66EB5DFE552120006010E89D1ECE8F037
:1095D00002E0000E01D0010EDAECEAF002E0060132
:1095E0000D89785003E0030E785C02E106010D79E5
:1095F00007ECEFF002E006010E8333A00ED0D1ECB1
:10960000E8F002E0000E01D0010EDAECEAF003E02F
:1096100006010D8D02D006010D8F01013DA72DD051
:1096200006010E81120006010E8B0101CDA725D087
:10963000CDA303D006010D8D02D006010D8F0101CF
:109640008F51080B03E10201515117E006010E830F
:10965000120006010E8D0201B451040B04E04D51BD
:1096600002E106010E830201B4A102D006010E87B9
:109670000201B4A302D006010E851200800E081468
:1096800005E02150010B02E10C5002D0FBEC26F06A
:10969000006E2DDFB1EF4AF0060150510A01DA9158
:1096A000040B01E0DA818DECE5F007E00601525190
:1096B00001015799800B01E057891200D9ECE4F0C1
:1096C0000C50006EFBEC26F0056E6AEC11F0046E97
:1096D000045006E00450006E21BE02D00450056E16
:1096E0001B0E00246EECE5F0016E210E05246EECDD
:1096F000E5F0026E005005E1B2ECEAF002E0220E65
:10970000016E055005E1B2ECEAF002E0420E026E95
:10971000030E005C09E1045007E1F7ECEEF004E011
:10972000200E016E400E026E0150F1ECE4F0695023
:1097300006E1FE0EDB5003E00250F1ECE4F0040E13
:10974000005C0DE10101CDA707D0CD51020B02E075
:10975000270E03D0280E01D0240EF1ECE4F0DEEF4A
:10976000E4F041ECEFF034B886D0695002E1B8EC97
:1097700011F00A01DA5106015099010B01E05089FC
:109780000A01DA5106015095010B01E050850A01EA
:10979000DA510601010B02E0509B01D0508B0A0107
:1097A000DA510601010B02E0509701D05087CDEC51
:1097B000F0F006E10601508D528F5291509F21D05A
:1097C000030E005C0EE10601508D509F93EC11F0EA
:1097D000000903E00601509D508F0601528F5291FF
:1097E00010D00601509D508F529F010157A902D001
:1097F0000601528F06015291010157B902D00601AC
:1098000052812150800B14E11550100B11E01550BE
:10981000200B0EE10C5009E0030E0C5C06E0050E77
:109820000C5C03E03BECE8F003E01598C4EC6AF054
:10983000030E0C5C03E0050E0C5C02E176EC68F0B4
:1098400014900C5004E1149001018BB51480030EA8
:109850000C5C04E1149001018FB51480149A14A0DB
:10986000148A54EC0DF0695004E184EC7FF0E3ECD1
:109870001DF0B3EC2CF03450100B18E101018F51A6
:10988000400B14E02150800B11E169500FE1FBEC1B
:1098900026F0010804E0FBEC26F0020807E10C507A
:1098A000DF6E0C6A0DEC1AF0DF500C6EF9EC1AF05A
:1098B0002682CEEC3EF0010EE66E00DFE55220EC93
:1098C0001BF0B1EC23F034B848D0FCEC1DF0C4EC34
:1098D0006AF0EFEC11F048EC26F01D98359001018C
:1098E000E2BB02D025EC09F0050E0C5C03E0050E8E
:1098F0007D5C02E18DEC0CF016EC25F069502DE159
:10990000B8EC25F0DBEC22F01FEC1EF0D4EC16F0E6
:109910008DECE5F002E0C2EC23F0B2EC16F034A4DA
:1099200002D054EC1EF06EECE7F056C1E6FFE66A9A
:1099300041ECF3F0016E01016081005006E0030E7E
:10994000005C04E17850010801E26091F4EC13F04E
:10995000050E005C02E14AEC09F03498E552DEEFB6
:10996000E4F08E9400000000030EE66E13EC7AF033
:10997000E552040E0A5CE66E13EC7AF0E5520150F3
:10998000E66E13EC7AF0E552A7ECFCF0006E0000F6
:109990008E841200D9CFE6FFE1CFD9FF8E9400006C
:1099A0000000060EE66E13EC7AF0E5528E8400009D
:1099B000000000008E9400000000020EE66E13EC22
:1099C0007AF0E552040E0A5CE66E13EC7AF0E5528A
:1099D0000150E66E13EC7AF0E552FE0EDBCFE6FFA7
:1099E00013EC7AF0E5528E84040EE66E79ECFCF00E
:1099F000E552E552E7CFD9FF120045ECEFF00050F9
:109A0000DF6E010EDB6A38D8DF50005C2DE0040EFB
:109A10000A5C16E2F29EA1980A50AA6E0150A96E45
:109A2000DF50A86EA69EA69CA684550EA76EAA0E11
:109A3000A76EA682F28E040E52ECE6F0A69414D025
:109A40008D8A010EDB2ADFCFE6FFA4DFE55289DF36
:109A5000DF50005C02E040EC0EF0DF50005C04E000
:109A6000050E15ECE5F0EDE3020EE15C02E2E16AC1
:109A7000E552E16EDEEFE4F01CECF3F0040E0A5C5C
:109A80000AE20A50AA6E0150A96EA69EA69CA68064
:109A9000A850006E13D08D8A010EDB2A62DF0050C1
:109AA000DF6E5FDF0050DF5C02E040EC0EF0005044
:109AB000DF5C04E0050E15ECE5F0EEE3020EE15C80
:109AC00002E2E16AE552E16EDEEFE4F0D9ECE4F0A7
:109AD0005BECEDF011E0FC0EF6ECEDF09CECE5F04B
:109AE000FD0EDBCFE9FFDB2AFE0EDBCFEAFF01E351
:109AF000DB2A00C0EFFFECD7DEEFE4F0D9ECE4F0B6
:109B00005BECEDF011E0FE0EF6ECEDF0016EFC0EFC
:109B1000DBCFE9FFDB2AFD0EDBCFEAFF01E3DB2A27
:109B2000EF50D5ECE8F0ECD7DEEFE4F0D9CFE6FF6C
:109B3000E1CFD9FFE6528E848D9A00000000060E18
:109B4000E66E13EC7AF0E5528D8A0000000000000A
:109B50008D9A00000000D80EE66E13EC7AF0E55204
:109B6000D7C7E6FF13EC7AF0E552E66A13EC7AF019
:109B7000E552E66A13EC7AF0E5528D8ADF6A1E0E32
:109B8000DF5C07E2640EE66E34EC29F0E552DF2A72
:109B9000F6D7E552E552E7CFD9FF1200D9CFE6FF5D
:109BA000E1CFD9FF35AE33D08E848D9A000000000E
:109BB000030EE66E13EC7AF0E552D7C7E6FF13EC1E
:109BC0007AF0E552FC0EDBCFE6FF13EC7AF0E552BB
:109BD000FB0EDBCFE6FF13EC7AF0E552FA0EDBCF9B
:109BE000F3FFDB06F35000090FE0A7ECFCF0006E7A
:109BF000FD0EDBCFE9FFDB2AFE0EDBCFEAFF01E340
:109C0000DB2A00C0EFFFEAD700008D8AC69EE5522E
:109C1000E7CFD9FF120045ECEFF0DF6A0101E99BC5
:109C2000DF2AFA0EDBCFE6FF22ECF4F053ECEAF089
:109C3000FA0EDBCFE6FFCAECE6F0AC0EE66E030EE2
:109C4000E66E53ECEAF0010EDB6AFA0EDB5015EC1F
:109C5000E5F017E2010EDB50E76E75ECE8F0E75037
:109C600009ECF0F0EFCF4AF0010EDB50EA6AAC0FDE
:109C7000E96E030EEA22EF504A5C03E1010EDB2A93
:109C8000E4D762ECEDF002E040EC0EF062ECEDF0B7
:109C900003E0140EDF5CC4E3140EDF5C02E2010E8D
:109CA00003D00101E98B000EB6ECEAF002E2E16AB2
:109CB000E552E16E4A50DEEFE4F0D9CFE6FFE1CFA6
:109CC000D9FF35AE46D08E848D9A00000000060E76
:109CD000E66E13EC7AF0E5528D8A00000000000079
:109CE0008D9A00000000020EE66E13EC7AF0E55249
:109CF000D7C7E6FF13EC7AF0E552FE0EDBCFE6FFA6
:109D000013EC7AF0E552FD0EDBCFE6FF13EC7AF0B0
:109D1000E552FA0EDBCFF3FFDB06F350000911E04A
:109D2000FB0EDBCFE9FFDB2AFC0EDBCFEAFF01E312
:109D3000DB2AEF50006E0050E66E13EC7AF0E5522D
:109D4000E8D700008D8AC69E050EE66E34EC29F039
:109D5000E552E552E7CFD9FF12000701D76B020E9B
:109D6000E66EE66AE668D20EE66E010EDDECE7F01E
:109D70000101D21D01E1D31D02E043ECEEF012001F
:109D800045ECEFF0358E0701D76BDF6ADF2A84ECF4
:109D9000F2F0DDECE7F084ECEAF0DB5005E00901DD
:109DA000001D09E1011D07E1010EDB6A40EC0EF028
:109DB000010E52ECE6F0010EDB5003E1050EDF5C14
:109DC000E5E3DF50040802E2010E6DD00901001D39
:109DD00004E1011D02E1020E66D0025104250F6E5E
:109DE00003510521106E000E0F5C400E105802E268
:109DF000030E59D006C9D2F107C9D3F10101000EF3
:109E0000D25D380ED35902E2050E4DD0400E02014C
:109E10000F24AC6F000E1020AD6FAC510101D225A4
:109E20000F6E0201AD510101D321106E08C9D2F1AC
:109E300009C9D3F1800ED25D030ED35902E2060E9A
:109E400032D00FC0AEF210C0AFF20201AE5101012C
:109E5000D2250F6E0201AF510101D321106E0AC944
:109E6000D2F10BC9D3F1BC0ED880D255020ED35516
:109E70000FE20FC0A5F310C0A6F30301A551010125
:109E8000D2250301A76FA6510101D3210301A86FB9
:109E90000EC9D2F10FC9D3F10101D251D31102E1A0
:109EA000040E01D0000EB6ECEAF002E2E16AE552DF
:109EB000E16E4A50DEEFE4F0D9ECE4F01F0E05014C
:109EC000115D0DE2112B1351EA6A150FE96E050EB3
:109ED00000ECF3F0132B13511F0801E2136BDEEFBC
:109EE000E4F0D9ECE4F0030E785C5BE10F6A106AF1
:109EF000FE0EDB500D0803E11F0E0F6E106AFE0E02
:109F0000DB500A0803E11D0E0F6E106AFE0EDB50D7
:109F1000090803E1EF0E0F6E106AFE0EDB50080811
:109F200003E10F68020E106EFE0EDB507F0804E1A5
:109F3000B50E0F6E030E106EFE0EDB501F0827E2EB
:109F40007F0E48ECE5F023E2410E48ECE5F00EE32D
:109F5000FE0EDB505A080AE3200E4A6EFE0EDBCFDF
:109F6000E7FF4A50E726FE0EE7CFDBFF020EE66E64
:109F70007A0E0301A7254C6E010EA8214D6EFE0E30
:109F8000DB50E00FE8245EECEFF018ECEAF00F5045
:109F900010102CE010C0E6FF8FDFE5520FC0E6FF87
:109FA00023D0FE0EDB504B6A7A0F4A6E060E93ECFE
:109FB000EFF0046E2450040B09E10450800B06E01E
:109FC0006F0EE66E79DFE55224840BD02450040B2B
:109FD00008E00450800B05E17F0EE66E6DDFE55270
:109FE0002494049E0450E66E67DFE552DEEFE4F051
:109FF00041ECEFF0800E48ECE5F003E3200ED4ECEA
:10A00000E7F00201050E3D6FFE0EDB50740811E112
:10A01000010E3D6F030E785C08E105011151FC0B48
:10A02000E842E842020F02013D6F0501006B1E820B
:10A030002BD0FE0EDB5028E0DF6A150EDF5C11E24C
:10A040008BECF2F00BE1DF2AE9ECE7F076ECEEF0D6
:10A05000DF2AE9ECE7F076ECEEF003D0030EDF2622
:10A06000ECD7150EDF5C04E17FECE5F03ADFE5525A
:10A07000200E48ECE5F003E2200ED4ECE7F07FEC94
:10A08000E5F042EC8AF0E552E552DEEFE4F045EC13
:10A09000EFF024A012D01EB009D00201685D1CE3CD
:10A0A0000701016B026B68C269F216D00201682BCE
:10A0B000685180081BE2800E18D01EA010D0070E39
:10A0C0000701015D09E2012B02910243020E020128
:10A0D000685D02E30701028F0201010E06D0020152
:10A0E000682B6851800802E2800E686F1E9024B0D1
:10A0F0001E802450010B03E1020E685D04E01E5037
:10A10000020B01E187D01EA204D00701CC0E026F22
:10A110000FD0070102910243028F070ED88001552C
:10A12000016E01500106000903E002910243F9D7D4
:10A1300000C70AF00201695107081DE269513F0892
:10A1400002E23F0E696FEDECEBF006E0200E43EC0F
:10A15000E6F0200E76ECEEF01850080B0CE007014C
:10A16000035109E0800E02016925006E03C701F06A
:10A170000701030742DC780E0701025D18E22A8A14
:10A1800002C7E6FF67EC04F0E552DF6EDF500EE039
:10A19000EDECEBF00BE03D5104E0DFCFE6FF28DF14
:10A1A00004D0DFCFE6FF42EC8AF0E5522A9A18A6E7
:10A1B00031D00701035105E002C700F003C701F0E9
:10A1C0001CDC0701035106E01E50020B03E11C0ECC
:10A1D000025D1DE103510BE01C0E025D08E1CC0E97
:10A1E000006E030703C701F0FDEC4CF01E821896C9
:10A1F00051EC80F0350E675C03E1410E06ECE5F0B2
:10A20000259224BC25820201010E3D6F01D0030777
:10A210000701026B0A6A020EE15C02E2E16AE552A2
:10A22000E16EDEEFE4F006015051545D03E152515E
:10A23000555D1DE050C654F652C655F6020E6F5CD1
:10A2400009E1050E0B5C06E1E66813EC7AF0E552D5
:10A25000E66807D052C6E6FF13EC7AF0E55250C626
:10A26000E6FF13EC7AF0E5528E8E8E8E8E9E28508D
:10A27000020B2AE02A50010B27E106015051515DE3
:10A2800003E15251535D20E0510E58ECE5F0060118
:10A290005051515D09E050C651F6310E58ECE5F0D1
:10A2A00050C600F074EC98F006015251535D09E07D
:10A2B00052C653F6320E58ECE5F052C600F074EC7C
:10A2C00098F03B0E58ECE5F0120000001200060179
:10A2D000DE6BF00E8C14060904ECEBF084AE02D0B9
:10A2E0000601DE81F00E8C14040904ECEBF084AE60
:10A2F00002D00601DE83F00E8C14070904ECEBF0AB
:10A3000084AE02D00601DE85F00E8C14050904EC43
:10A31000EBF084AE02D00601DE87F00E8C14020949
:10A3200004ECEBF084AE02D00601DE89F00E8C1452
:10A33000010904ECEBF084AE02D00601DE8BF00ED6
:10A340008C14030904ECEBF084AE02D00601DE8D20
:10A35000F00E8C1404ECEBF084AE02D00601DE8F1C
:10A36000F00E8C16120046ECF3F048ECE5F008E332
:10A37000FE0EDBCFE6FFFD0E6DECECF00AE207D03F
:10A38000FD0EDBCFE6FFFE0E6DECECF002E2010EFF
:10A3900001D0000EDEEFE4F045ECEFF02FB26CD010
:10A3A000DF6A080EDF5C36E2F00E8C14DF108C6E74
:10A3B000B70ED9ECE5F000C06FF707016F5119082F
:10A3C00027E2FE0EDB5004E1F00E8C16010E57D092
:10A3D000B70ED9ECE5F000C070F70701705119080D
:10A3E00017E2B70ED9ECE5F000C071F7030EE66E88
:10A3F00070C7E6FF6FC7E6FFD1ECE6F009E0030E99
:10A40000E66E71C7E6FF70C7E6FFD1ECE6F002E149
:10A41000DF2AC7D7F00E8C16080EDF5C2AE2DE5268
:10A42000010EDD6E080E15ECE5F010E2070EE66E8B
:10A43000010EDB503B0F6EECE5F0E66E70C7E6FFF9
:10A44000D1ECE6F003E1010EDB2AECD7080E15ECA7
:10A45000E5F00FE26FC772F770C773F771C774F753
:10A46000010EDB50080DF350DF100701756F7551B9
:10A4700006D0080EDF5C02E1000E01D0800EB6ECC3
:10A48000EAF002E2E16AE552E16E4A50DEEFE4F002
:10A49000D9ECE4F01F981F9EFE0EDB50005C01E03B
:10A4A0001F8E1F9CFE0EDB50D880005401E21F8CD3
:10A4B000020E016E2DA204D01F88FE0E00C0DBFF2D
:10A4C0001FAE8FD01F50200B01E0010E4A6E1F50AF
:10A4D000400B01E0010E4A5C01E080D01FAC0DD0C2
:10A4E0000150D880005414E20150005EFE0EDB5093
:10A4F000D88000540DE21F880BD00128E86C005C66
:10A5000007E201500026FE0EDB50005C01E21F88CE
:10A51000010157A50FD00050036EDF0ED9ECE5F016
:10A52000CAECF0F002E6FFECEDF002E21F9859D021
:10A530000350006E1FA852D0FE0E00C0DBFF049433
:10A54000020E6F5C04E1C90E0B5C01E1048404504F
:10A55000040B11E115EC6EF0000903E025ECEFF0BF
:10A560003DE0FD0EDB50FF0839E00201415136E1CC
:10A570002150200B33E072ECE7F00101010E016F76
:10A5800004A403D0FE0EDB5011D0FD0EDB50006E94
:10A59000BCEC2DF0500E096EFE0EDB40E840E840AA
:10A5A0001F0B006E00501E0802E21E0E006EA1EC92
:10A5B00096F004B413D0030E0101015D016E015049
:10A5C000012A83ECE5F0200EEF6EB0ECF3F0EF50D3
:10A5D000300804E1B0ECF3F0200EEF6E1F9A1FBCC0
:10A5E0001F8AFE0EDB50DEEFE4F01350040B07E190
:10A5F00015EC6EF0000903E025ECEFF02EE072ECB4
:10A60000E7F001012D0E1A6F20A402D02B0E1A6F55
:10A610000201555107E1545105E1535103E1010194
:10A62000200E1A6F7CECE5F055C23FF0D1ECF0F053
:10A63000300F01011B6F300E3B241C6F300E0201E6
:10A64000542501011D6F0701EFAB05D0300E02014B
:10A65000532501011E6F01011C8F12001DECF4F047
:10A66000DCECE5F0EFCFDFFF01019F6BA06BA16B8E
:10A67000A26BA36B1EAE03D0050EA16F3ED0CFEC34
:10A68000E7F0EF50400B03E12850040B1DE07FEC96
:10A69000E5F05AEC0EF0E55200C0A1F1005063085D
:10A6A00027E20101A16BA02B7D0E005C02E1190ED7
:10A6B000A16F1CECF1F0FA0E4A181AE14B5018E1A8
:10A6C000A02B320EA16F14D0CFECE7F0EF50200B8F
:10A6D00002E0A32B0DD0CFECE7F0EF50100B07E01A
:10A6E000020EA26F58A704D0050EA26F01D0A22BB4
:10A6F0002BAE03D0020E64ECE5F0E552DEEFE4F0A1
:10A70000B10E006E02018EA502D0B50E006E005093
:10A71000EAECE8F036C100F002018EA502D07CC15F
:10A7200000F0A1EC96F0300E01011D5D05E17BEC1F
:10A73000EEF002E1200E1E6F1200D9ECE4F0050EDF
:10A740004C6E4CC044F0FE0EA0ECEBF04B6A3D0F9B
:10A750004A6E070E93ECEFF0006EA3EC93F001014C
:10A7600069ECEDF00C0E48ECE5F003E20E0E126F12
:10A770000ED00E0E136FFE0EDB50630802E2100EB9
:10A78000136F0F0E48ECE5F002E2090E146F140E81
:10A79000176F120E186FDEEFE4F0D9ECE4F0AFECB7
:10A7A00093F00101012BFE0EDB50006EA1EC96F040
:10A7B0002C50100B07E1640E48ECE5F003E20101B8
:10A7C000200E1A6F2CA807D001014D0E1E6F570ED8
:10A7D0001F6F1B8F18D0FD0EDB5003E101011C8F92
:10A7E00007D00A0E48ECE5F003E20101200E1B6FD2
:10A7F0000101570E1E6FE151010B05E05751080B87
:10A8000002E02A0E1F6FDEEFE4F0B3EC2CF072ECE6
:10A81000E7F05CECE6F007E0010EE66E94EC05F084
:10A82000940FE66E03D0E66A49C1E6FFB6DFE55253
:10A83000E5522CA806D0D5ECECF049C1E6FF7DDF4F
:10A84000E552120041ECEFF0B90EEAECE8F035C148
:10A85000DFFFFCECEAF003E0E7ECEEF001E1DF6A99
:10A86000DF50006EA1EC96F0640EDF5C03E20101A4
:10A87000200E1D6F0A0EDF5C03E20101200E1E6F29
:10A88000E552DEEFE4F072ECE7F04AC100F0A1EC33
:10A8900096F0640E01014A5D02E2200E196F0A0E65
:10A8A0004A5D02E2200E1A6F930E006EBCEF2DF08F
:10A8B000020E0201955D04E10C0E06ECE5F00AD0F3
:10A8C0000D0E06ECE5F0030E0201955D03E10101BA
:10A8D000320E1E6F500E096E1200F00E006E8DECDF
:10A8E000E5F002E0F30E006E44EC2EF033C100F010
:10A8F0008DECE5F002E054C100F082ECE9F00101DA
:10A900001E8F1200D9ECE4F029C100F0FCECEAF053
:10A9100003E159C100F011D08DECE5F00EE055C116
:10A9200000F0FE0EDB5009E001019751020B05E03B
:10A930009751040B02E098C100F0DEEFE4F0D20E74
:10A94000006E8DECE5F00CE0FCECEAF009E00101B2
:10A950009751020B05E09751040B02E0F60E006ED2
:10A9600044EC2EF0010EE66ECDDFE552A1EC96F040
:10A97000300E01011D5D05E17BECEEF002E1200EE1
:10A980001E6F1200D9ECE4F0B3ECF3F0400B03E1DE
:10A990002850040B05E001018F51020B01E18BD01F
:10A9A000B3ECF3F0200B03E02850040B02E00101AC
:10A9B0009E6BB3ECF3F0400B03E12850040B57E01F
:10A9C0000101A0510EE0A1510CE1FE0EDB5005E1AA
:10A9D0009C5102E19D5101E0A06B9C6B9CC19DF1DB
:10A9E0006AD05A0EA15D13E17CECE5F09CC13FF00A
:10A9F00070ECEDF007E1005003E101019D5102E030
:10AA00000101A16B01019D6B00509C5F54D09C51D2
:10AA100002E19D5150E09D514A6E4B6A9C510A0DD6
:10AA2000A8ECE7F0A15173ECE9F0E8ECF3F0D2C147
:10AA300043F0D3C144F0EBECFCF03AC0D0F13BC0A2
:10AA4000D1F10101D051D11136E0D0510F5ED15179
:10AA5000105AFE0EDB5001E1A16B0A0E4A6E4B6AE2
:10AA600088ECEFF03EC09CF13AC09DF124D0B3ECED
:10AA7000F3F0100B20E0B3ECF3F0200B1CE1020E1E
:10AA8000016E010158A702D0050E016E01C0A2F1AE
:10AA900001C044F09DC13FF070ECEDF004E10050C6
:10AAA00002E000C0A2F1FE0EDB5005E0005003E022
:10AAB00000500101A25FDEEFE4F0D9ECE4F07FEC9E
:10AAC000E5F0E66A5FDFE552E5529AC1CFF29BC13D
:10AAD000D0F29CC1D1F29DC1D2F29EC1D3F2CCEC96
:10AAE0003AF001019A510FE10301E35101019B5D2D
:10AAF0000AE2CFC29AF1D0C29BF1D1C29CF1D2C27C
:10AB00009DF1D3C29EF10201842BDEEFE4F0A2ECB2
:10AB1000E9F006E1D893CCB3D883D895CCB5D885E5
:10AB20001200010139A306D0CC9313B6CC83CC9587
:10AB300013B4CC85ECDF04B058DD08ECC0F069EF4D
:10AB400038F02EBC12000A0E02015403F3504C6E72
:10AB50004D6A5551640DF3504C244A6EF4504D200B
:10AB60004B6E535101014A24D46F000E4B20D56F18
:10AB70000A0E006E0701EFAB02D0010E08D0EFA95C
:10AB800007D0140E006E010158A702D0320E006EDD
:10AB900020B403D001010EECECF029AA1AD01CEC71
:10ABA000F1F0100ED8804A56270E4B560101D551B0
:10ABB0004B18E8AE02D04B3404D04A50D45D4B5011
:10ABC000D5591FE200506AECE7F0D4274B50D5234B
:10ABD00018D000504B6AF00F4A6ED80E4B2201017C
:10ABE0004B50D519E8AE02D0D53504D0D4514A5CCB
:10ABF000D5514B5806E200506AECE7F0D45F4B5059
:10AC0000D55B2084800ED51503E020940EECECF08B
:10AC10001CECF1F0D4C13EF0D5C13FF029ECEDF0D1
:10AC20004BAE04D03A6C3B1E000E3B223A50010161
:10AC3000D45F3B50D55BD7ECEEF092ECF2F03EC027
:10AC400055F23A500101D46FD56B0A0E4A6E4B6A29
:10AC500092ECF2F03EC054F23AC053F230EF56F0AC
:10AC60000101CAA9308E198C048091EF55F00A01B8
:10AC7000DA9F54EC0DF0016A0C5011E182ECE6F021
:10AC80002AE10701EFBF11D00A0E016E59ECE8F07E
:10AC90003F50006E0150005C1EE200501BD0030EBE
:10ACA0000C5C12E10701EFAF02D0160E13D0030EB9
:10ACB000785C02E1140E0ED0785002E11E0E0AD02C
:10ACC000260E25ECF0F006D03BECE8F002E0010E99
:10ACD00001D0160E016E0150160802E2160E016E2A
:10ACE00012000A0E01010F5D09E12C50100B06E164
:10ACF0004951500803E2790E495D01E3000C010C53
:10AD0000F0DF000903E00101500E496F1200D9EC99
:10AD1000E4F000AE14D0FF0E0002F3CF84F2840EF4
:10AD2000E96E020EEA6EEFCF3FF0FE0EDBCF44F08D
:10AD30002FECFDF03FC0EFFF0201846D09D000C091
:10AD40003FF0FE0EDBCF44F02FECFDF03FC084F26D
:10AD5000DEEFE4F001018BAD07D02EAC02D0FCEFAA
:10AD600004F002010A0E3C6F12000101E1A503D0BC
:10AD7000E195A4EFEBF00601D951D995010B01E063
:10AD8000D985D951D997020B01E0D987D99188503B
:10AD9000400B01E0D981D9938850800B01E0D98321
:10ADA0000F0ED91519ECE6F000A005D000AE02D0C8
:10ADB000DF0701D0DF2BDA51DA95010B01E0DA85EC
:10ADC000DA51DA97020B01E0DA87DE51DA91020BF1
:10ADD00001E0DA81DE51DA93010B01E0DA830F0E34
:10ADE000DA1519ECE6F000A009D0A4ECEBF000AE07
:10ADF00003D00601E00702D00601E02BDB51DB9512
:10AE0000010B01E0DB85DB51DB97020B01E0DB8707
:10AE1000DE51DB91080B01E0DB81DE51DB93040B9B
:10AE200001E0DB830F0EDB1519ECE6F000A009D082
:10AE3000A4ECEBF000AE03D00601E10702D006015E
:10AE4000E12BDC51DC95010B01E0DC85DC51DC976A
:10AE5000020B01E0DC87DE51DC91200B01E0DC819C
:10AE6000DE51DC93100B01E0DC830F0EDC1519ECD6
:10AE7000E6F000A00AD00201320E3B6F00AE03D014
:10AE80000601E20702D00601E22BDD51DD95010B40
:10AE900001E0DD85DD51DD97020B01E0DD87DE514C
:10AEA000DD91800B01E0DD81DE51DD93400B01E09F
:10AEB000DD830F0EDD1519ECE6F000A00AD00201CB
:10AEC000320E3B6F00AE03D00601E307120006010D
:10AED000E32B12000450010B4A6E0450020B01E0F8
:10AEE000010E4A5C07E06C0EE66EF20EE66E010E95
:10AEF00039EFE6F0E00E0101EC15016E1F0EEC15C6
:10AF0000026EEDC103F0015003E0E00E015C54E17C
:10AF100002506EE00150021203501FE12050080B56
:10AF200006E03C51010B03E02850010B16E02E50C7
:10AF3000400B03E03050200B10E02150200B0DE0BF
:10AF400002507926CA51100B08E02050080B05E08A
:10AF50002C50200B02E102500726030426E13C514D
:10AF6000200B12E12050080B0FE02E50400B06E1A1
:10AF70003C51020B09E02850010B06E12E50400B1A
:10AF800014E03C51010B11E12150200B0EE03C512B
:10AF9000200B09E02050080B06E03C9B289D076A27
:10AFA0000201320EFD6F02500726020E035C20E103
:10AFB00002500601DF271200800E015C11E1100E25
:10AFC000025C16E2070E0214400F676E178E179888
:10AFD000179002A602D0178801D01780DE951200C4
:10AFE000C00E015C05E1030E025C02E202C0EDF15D
:10AFF000120019BE12008A8C81AE03D00101E997BC
:10B0000012008150800B55E10101E951080B51E11B
:10B01000F29E8A9C04900492090E016EEC6B060E5F
:10B0200033ECE7F0270E026E0150010803E2010144
:10B03000EC91EC4381AE09D00150010805E2020613
:10B040000101EC8F047001D004829EAA04D0020E8C
:10B05000025E06ECE7F002501EECE8F00106E2E1C9
:10B06000E00E0101EC15C0081FE1080E016EF9C2E7
:10B0700006F0020E33ECE7F00F0E936E270E026E11
:10B0800006A002D08A8E01D08A9E069006429EAA11
:10B0900004D0020E025E06ECE7F002501EECE8F06F
:10B0A0000106ECE18F0E936E15DF8A8C0101E987B2
:10B0B000F28E120045ECEFF09CDF28A004D05AEC91
:10B0C000CAF08FEF5DF02450800B4AE13150400B05
:10B0D00047E120A61BD075ECECF001012799020195
:10B0E000845102E0010127890101279B020184AFFD
:10B0F00002D00101278B010127A932D01EAC02D05A
:10B10000EEEC0BF00201640E506F2AD07950006E05
:10B1100001012799005001E02789279B00BE278B5A
:10B1200027BB006C020E6F5C0FE1B90E0B5C03E0F5
:10B13000E30E0B5C05E1D8900032D890003207D0C6
:10B140000038E842070B02D000380F0B006E0050A9
:10B1500006E0278D279F27BB278F796A01D0279983
:10B1600001012751100B09E0CA51100B06E12C50C8
:10B17000200B52E01E50400B4FE12050080B1DE009
:10B180003C51200B09E02E50400B06E1CA51100B38
:10B1900014E02751100B11E07DECECF0010128992F
:10B1A0000201845102E0010128890101289B02016A
:10B1B00084AF32D00101288B2FD00750006E289920
:10B1C000005001E02889289B00BE288B289928BBC5
:10B1D000006C31AC05D0D8900032D89000320FD03E
:10B1E0001CA204D00038E8461F0B08D033A004D0BE
:10B1F0000038E842070B02D000380F0B006E0050F9
:10B200000AE00701280ED86F0101288D289F28BB6E
:10B21000288F076A01D028992C50200B03E01E507C
:10B22000400B0DE001012751100B01E00DD3285117
:10B23000100B01E009D32150200B01E105D3D7CA3F
:10B24000DCFAD6CADDFA91DDDFC600F00601D99935
:10B25000005001E0D989D99B00BED98BD9A938D03B
:10B26000D9BB006C29ECEFF033E0DF6B0201640E18
:10B27000506F1350080B0DE11350040B0AE1020E3E
:10B280000101775D0EE13C51200B0BE02E50400B8D
:10B2900008E1298A0601D9BB299A53DCF2ECEBF0CC
:10B2A00017D03851010B14E03C51010B11E1E0C201
:10B2B00079FF0601D9AB04D0E0C279FF0F01796CA8
:10B2C00001012789CAA903D07950076E28892884EB
:10B2D000E0C600F00601DA99005001E0DA89DA9B55
:10B2E00000BEDA8BDAA97CD0DABB006C29ECEFF077
:10B2F00001E176D0E06B010E0E6EDABB0E6837EC22
:10B30000E8F06CE02E50400B03E0C9ECE8F066E199
:10B31000050E0C5C03E1E0EC0BF060D002019551EE
:10B320000EE0030E2EECF4F0950EE66E020E00EC2D
:10B33000E5F058EC54F0178E3A0E676E4FD032BCE1
:10B340004DD0060150A725D0358491DC0E040BE1C9
:10B3500077ECEDF008E2190E0124D75D04E2020E4D
:10B36000D65FD72B11D0800E0E140EE041EC12F0F8
:10B37000FF0F0A01D65D08E2BEECECF0D880D7558D
:10B3800003E2020ED627D7070A01010ED46F3488D4
:10B3900021D050A523D03584BAECECF008E0C80EDB
:10B3A000E66E280EE66ED80EE66E030E0AD05FDC5F
:10B3B000190E0124E66EBEECECF0E66ED70EE66EDA
:10B3C0000A0E00ECE5F00A01030ED46F34887BEC22
:10B3D00020F0010EE66EE66E73ECE6F089ECEAF022
:10B3E000E1C600F00601DB99005001E0DB89DB9B40
:10B3F00000BEDB8BDBA963D0DBBB006C29ECEFF07C
:10B400005EE0E16B010E0E6EDBBB0E68050E0C5CA0
:10B4100003E1E0EC0BF053D037ECE8F050E02E50B5
:10B42000400B03E0C9ECE8F04AE1060150AB27D03D
:10B43000358437EC56F0800E0E140CE077ECEDF00E
:10B4400009E2BEECECF0D880D75504E2020ED65FDC
:10B45000D7070FD00E040DE141EC12F0FF0F0A01E7
:10B46000D65D07E2190E0124D75D03E2020ED6274E
:10B47000D72B0A01020ED46F3488DCECEFF0060102
:10B4800050A91BD0358451EC12F0E7ECEFF007E245
:10B490004A501408000E4B5402E251EC12F0E7EC53
:10B4A000EFF009E24A503D08000E4B5404E251EC23
:10B4B00012F051EC12F05AEC12F089ECEAF0E2C60C
:10B4C00000F00601DC99005001E0DC89DC9B00BE45
:10B4D000DC8BDCA998D0DCBB006C29ECEFF001E13F
:10B4E00092D0E26B010E0E6EDCBB0E682DA418D05C
:10B4F0008DECE5F008E1C80EE66E330EE66E010E47
:10B50000FBECE4F00AD0C80E2EECF4F0540EE66E1C
:10B51000010E00ECE5F0EBEC1DF06DEC54F06FD09B
:10B5200050AD19D0320E006E01018FAD02D0640E05
:10B53000006E0050E66E080EE66E4A0EE66E010ED4
:10B5400000ECE5F043EC54F04AC103F5EAEC7FF07F
:10B550000201178754D050AF52D06EECE7F00101D2
:10B560008EA503D036EC09F04AD03450040B25E008
:10B57000000403E0020E005C20E10E50462746C1A5
:10B58000E6FFC10EEEECE4F00E0E06ECE5F046C16F
:10B5900000F0010146AF04D046C100F00001006C8C
:10B5A00000900042A1EC96F001012B0E1D6F46AFFA
:10B5B00002D02D0E1D6F1F8F22D002018EA50FD03D
:10B5C0003C0EE66E7C0EE66E010EFBECE4F07CC1F8
:10B5D000E6FFCC0EEEECE4F080EC53F00FD015EC6F
:10B5E0001EF03C0EE66E360EE66E010EFBECE4F04D
:10B5F000A5EC16F080EC53F0020119832B842E8EFB
:10B6000002011E0E306FE3C600F00601DD99005006
:10B6100001E0DD89DD9B00BEDD8BDDA915D1DDBB41
:10B62000006C29ECEFF001E10FD1E36B010E0E6E1F
:10B63000DDBB0E682DA62FD08DECE5F00AE13C0EA7
:10B64000E66E290EE66E010EFBECE4F076ECE9F016
:10B650001FD0FCECEAF006E13C0EE66E590EE66EF9
:10B66000010E12D001019751020B09E09751040B12
:10B6700006E03C0EE66E980EE66E010E05D03C0E1E
:10B68000E66E550EE66E010EFBECE4F01FEC1EF0CC
:10B690009FEC54F0D5D052AFAFD001018EB5B1D0F0
:10B6A00034B632D021BE04D08D0E006E4EEC2EF09A
:10B6B000FF0E0E5C0CE102013F0ED8800F55000E0C
:10B6C00010551FE2400E0F5F000E105B1AD086C2AD
:10B6D00001F02C50100B07E102018651780803E2BB
:10B6E0006C0E015C016E01500101CF5D0AE20201A6
:10B6F000480E0F5D710E105904E2400E0F27000E28
:10B700001023E7EC0BF09CD002012D6B780E016E3C
:10B71000026A0BECEFF002E0DA0E016E2CA804D006
:10B72000960E016E0A0E026E0150E66E0250E66E33
:10B73000490EE66E010E00ECE5F02B84E0EC2AF0F9
:10B7400071EC56F000090BE00101500E496F0E0438
:10B7500006E10BECEFF003E00101790E496F05EC17
:10B7600054F0780E016E54ECE7F002E1500E016ED9
:10B770002C50100B10E10E0403E1790E495D06E038
:10B78000800E0E1408E00150495D05E1328E37EC61
:10B79000E8F001E01D946EECE7F03250800B0EE112
:10B7A000020131510BE000500CE0050E005C09E095
:10B7B000030E005C03E1020E785C03E00E5080ECA7
:10B7C000EEF032AE16D0329E010EDB6A1AA006D021
:10B7D000DB682FEC0BF0050E64ECE5F07EEC28F056
:10B7E000A8DA010EDB5002E02AEC0BF00E5080ECE0
:10B7F000EEF00201188B24D052A122D001018EA5B7
:10B8000003D036EC09F01CD035C1DEF215EC1EF089
:10B81000280EE66E350EE66E010EFBECE4F006EC4B
:10B82000EDF003E00101355106E00201DE5105E1D2
:10B830000101355102E0E4EC1CF0020119852B8472
:10B840002E8E02011E0E306F1EAC64D00701EF83F6
:10B85000E1EC09F001013C91139C3C51010B01E02A
:10B86000138C5AEC34F0006E00500F0802E20F0EF9
:10B87000006E100E0002F3CF21F252EC2FF01E9A50
:10B88000050E0701D3250201D880215501E21E8A49
:10B890002B50800B13E1205111E0050E0701D35D01
:10B8A0000201215D03E225EC09F01E881E50100BF9
:10B8B00031E01E50200B2EE0020109D02B50800BEE
:10B8C0000AE11E50800B07E11E50200B04E0FA0E27
:10B8D000206F1E981FD02BBE02D022EC09F02CBA8C
:10B8E00017D00C0EE66E050E93ECEAF0E66EE2EC75
:10B8F000E7F00AE007C5BFF108C5C0F109C5C1F10D
:10B900000AC5C2F10BC5C3F1E0C279FF0101279B53
:10B91000010127891E50800B0AE101012751100BFC
:10B920006FE02050080B6CE02150200B69E0020111
:10B930001E0E306F1EAC02D0140E306F2CAA2FD00A
:10B940001EBC16D001014551630801E2456B800E13
:10B95000791406E0FB0E795C03E2796A000E11D0DF
:10B96000800E79144CE17950030849E2796A08D0D5
:10B97000796A2BAE09D00501065141E1320E066FFE
:10B98000010E7EECEDF03BD00101A851030837E336
:10B99000010E7EECEDF00101140EA86F30D017837C
:10B9A00005013B812C8C2D8AA3ECE5F00C50E66E52
:10B9B0002EEC53F0E55275ECECF01E50800B05E0D8
:10B9C000795003E1A8EC3AF014D0020184AF09D019
:10B9D000EFC7E6FF5DEC55F0E5520201E051792634
:10B9E00008D0845106E0EFC7E6FF23ECEAF0E0510F
:10B9F000795E02018451DFE12E829DEC04F01E9EEF
:10BA000001012851100B5AE02050080B57E021503B
:10BA1000200B54E002011E0E306F1EAC02D0140E3B
:10BA2000306F178305013B832C8C7D50DF6E2E50C9
:10BA3000400B03E1AAECEAF002E00C50DF6E2EAC02
:10BA400004D02D8AA3ECE5F003D02D9A79ECE7F031
:10BA5000DFCFE6FF2EEC53F0E5527DECECF0020177
:10BA600084AF0BD0DF501FECF2F0E66E5DEC55F0CA
:10BA7000E5520201E15107260AD0845108E0DF5067
:10BA80001FECF2F0E66E23ECEAF0E151075E845120
:10BA9000E4E12E822EAC03D09DEC04F002D08FECBA
:10BAA000E7F025A605D0010E096E0701140E826F7E
:10BAB0000101CAA903D00701280ED86F2CAC2BD0E6
:10BAC000AAECEAF00FE02751100B0CE02851100B04
:10BAD00003E12C50200B06E02E50400B03E1050142
:10BAE0003B832C9C01018BAD03D02C9C08AE198CA0
:10BAF000F0EC38F001013CA9308ECEEC3EF02C9CED
:10BB000026822D50200B06E02E50400B03E1AAECBC
:10BB1000EAF001E0248A0101289927992894020E6D
:10BB2000E15C02E2E16AE552E16EDEEFE4F0D9ECBD
:10BB3000E4F0180E07011B171C6BFE0EDB5001E131
:10BB40001C81FE0EDB0401E11C83B2ECECF001E190
:10BB50001B81FE0EDB50030801E11B83FE0EDB5050
:10BB6000040801E11B85DEEFE4F0695005E0D5CA69
:10BB7000E6FFDDDFE5521200180E07011D171E6BF0
:10BB80000A01D55102E107011E810A01D50502E132
:10BB900007011E83020E0A01D55D02E107011D8126
:10BBA000030E0A01D55D02E107011D83040E0A019F
:10BBB000D55D02E107011D851200000000000000B4
:10BBC000E8EC08F0F2EC08F082A82D808A8A1200D6
:10BBD000020E1EECE8F0DDEF5DF0050EE66EFDEC0A
:10BBE00018F0E552F00E8C148C6EA0D88A9A0000E2
:10BBF0001FC700F00101E3A915D00050E66E13EC59
:10BC00007AF0E5521DC704F0049C07011EB1048CB4
:10BC1000049E07011EB3048E0450E66E13EC7AF006
:10BC2000E5521DD0060E00C0E7FF070B04E0E74217
:10BC3000E79EE806FCE1E750E66E13EC7AF0E55289
:10BC40003F0E0014040DF35007011E11E66E13ECB5
:10BC50007AF0E5521DC7E6FF13EC7AF0E552ADDF4E
:10BC6000F00E8C1406098C6E61D88A9A000020C7E9
:10BC700000F00101E9A315D00050E66E13EC7AF054
:10BC8000E5521BC704F0049C07011CB1048C049E00
:10BC900007011CB3048E0450E66E13EC7AF0E552F3
:10BCA0001DD0060E00C0E7FF070B04E0E742E79E49
:10BCB000E806FCE1E750E66E13EC7AF0E5523F0E41
:10BCC0000014040DF35007011C11E66E13EC7AF01A
:10BCD000E5521BC7E6FF13EC7AF0E5526EDF120067
:10BCE000F00E8C1404098C6E21D88A9A000010C7BB
:10BCF000E6FF13EC7AF0E55260DF1200F00E8C14D0
:10BD000002098C6E13D88A9A000013C7E6FF13EC61
:10BD10007AF0E55212C7E6FF13EC7AF0E55211C74C
:10BD2000E6FF13EC7AF0E55253DF1200010E1EEF2E
:10BD3000E8F0050EE66EFDEC18F0E5522D90DEDF22
:10BD40004CDFF4EC13F0F00E8C1405098C6EEEDF72
:10BD5000EDDFECDFEBDF8A9A0DC7E6FF13EC7AF03C
:10BD6000E5520CC7E6FF13EC7AF0E5520BC7E6FF8D
:10BD700013EC7AF0E5520AC7E6FF13EC7AF0E552CD
:10BD800027DFF00E8C1403098C6ED0DF8A9A000036
:10BD90000FC7E6FF13EC7AF0E5520EC7E6FF13EC8F
:10BDA0007AF0E5520ADFF00E8C140A098C6EBEDFC1
:10BDB0008A9A000009C7E6FF13EC7AF0E55208C73B
:10BDC000E6FF13EC7AF0E55207C7E6FF13EC7AF0D2
:10BDD000E55206C7E6FF13EC7AF0E552EEDE80DFAF
:10BDE000F00E8C1401098C6EC682C6909FDF8A9A71
:10BDF000000000000000000016C7E6FF13EC7AF018
:10BE0000E55215C7E6FF13EC7AF0E55214C7E6FFDA
:10BE100013EC7AF0E552DCDEC680C692F00E8C168A
:10BE20001200810E73ECE5F0320E096E308834C1D9
:10BE30002AF21200030E0A6E2A0EE66E000EE66E5D
:10BE40000A0E4DEFF1F0030E0A6EAA0EE66EA4EC98
:10BE5000F3F0E66E300E9CEFF4F032EFF4F0D9EC34
:10BE6000E4F005013B8FB2ECECF00DE101013CB9CF
:10BE700002D08B9D08D03C99E66A43EC90F0E552E5
:10BE800001018B9D34D0FE0EDB5024E0C9ECE8F0BC
:10BE900021E1CA993CB909D03C89010EE66E43EC18
:10BEA00090F0E55201018B8D03D08B8D29EC90F041
:10BEB000198638EC0DF01B82C7ECB8F0EFECB8F047
:10BEC0001B92076A796A5D0EE66EF20EE66E010E4F
:10BED00039ECE6F0FE0EDB5011E1C9ECE8F00EE0C3
:10BEE0008B9D29EC90F038EC0DF069EC38F0640E85
:10BEF000E66EF20EE66E010E39ECE6F0DEEFE4F0EF
:10BF000012001E50400B0CE02B50800B09E1225018
:10BF1000200B06E02B8E130EEAECE8F025EC09F07E
:10BF2000120025A808D0010EE66E99DFE5520F0E2B
:10BF300050ECF3F01B861200010124A180EF67F0A2
:10BF400001012491020122070201225101E0A8D13E
:10BF50000201640E226F0201EC6B0201295102E022
:10BF60000201290701018C5106E001018C07010142
:10BF70008C5101E13296020130510EE02050080B45
:10BF80000BE0020130070201305106E11EAC02D085
:10BF90001E8E02D02EBE2E9E300E0401B75D06E12D
:10BFA0000201176B186B196B1A6B02D085ECCCF081
:10BFB00002012A5126E00501005123E12850400BDF
:10BFC00020E102014A514B111CE102012A07020142
:10BFD0002A5117E10D50006E02016A5108E07F0EF0
:10BFE00002016A15006E199A02016ABF198A010ED0
:10BFF000E66E0050E66E9AEC8FF0E552E5520201D3
:10C000006A6B02016E0702016E511EE10701F10524
:10C010000FE102010F0E6E6F560E02011E5D07E268
:10C02000870E006E248859EC2EF00968268E0CD0FD
:10C030000101525102011E5D07E2870E006E248845
:10C0400059EC2EF00968268E020128514EE00201BB
:10C0500028070201285147E12250200B44E00E0E30
:10C06000675C3AE131ECAFF028702892520EE66E30
:10C07000E1EC07F0E552520EE66EE1EC07F0E55216
:10C0800028B011D0570EE66E6EEC2EF0E55269EC3A
:10C0900038F045EC15F04E0EE66EE1EC07F0E55297
:10C0A000E8EC18F013D0580EE66E6EEC2EF0E55268
:10C0B00069EC95F0E80EE66E79ECFCF0E552E1EC07
:10C0C00018F0520EE66EE1EC07F0E5523B0EE66E1C
:10C0D000E1EC07F0E55207D028A005D04C0EE66E43
:10C0E00029ECCAF0E55280EF67F0B8ECC4F001012A
:10C0F00001013951100B06E11450020B05E01A50F2
:10C10000200B02E1060105772950400B01E0010EEA
:10C11000020F016E2950400B01E0010E050F026E67
:10C1200003681EAC10D00150EA6A110FE96E010ECF
:10C13000EA22EF7E0150EA6A110FE96E010EEA224F
:10C14000EF50800B036E61EC0BF0000923E0FF0E53
:10C15000035C11E10250EA6A110FE96E010EEA2256
:10C16000EF7E0250EA6A110FE96E010EEA22EF50EB
:10C17000800B036E0FD00250EA6A110FE96E010EB8
:10C18000EA22EF9E0250EA6A110FE96E010EEA22DE
:10C190000350EF126FEC0BF000091AE0FF0E035C86
:10C1A00008E10250EA6A190FE96E010EEA22EF7EF9
:10C1B0000FD00250EA6A190FE96E010EEA22EF9ED3
:10C1C0000250EA6A190FE96E010EEA220350EF12DB
:10C1D000DBEC04F0000902E006011A792350040B9D
:10C1E00005E02D50100B02E00601127918EC08F062
:10C1F00000090EE02D50400B0BE12D50800B08E1A3
:10C200000101DEB703D006010E7102D006010E81D6
:10C210000201435105E01450080B02E006010273CD
:10C2200015ECC4F0000903E12F50200B27E02F9AF2
:10C23000E1EC18F0016A030E015C15E2026A040EDB
:10C24000025C0BE2020E006E37EC91F0320EE66EED
:10C2500034EC29F0E552022AF2D7E66834EC29F0F2
:10C26000E552012AE8D7E8EC18F00101609926822E
:10C270002FEC9BF000ECC4F09CECC3F002013D51AC
:10C2800002E002013D070201905105E02350100B2E
:10C2900002E1020190070201455102E00201450757
:10C2A0002850010B28E08150010B03E02150040BC2
:10C2B00022E019EC16F0FF081EE12E50400B1BE1A6
:10C2C0002150200B18E01950800B15E10201245178
:10C2D00002E002012407020124510DE12AA003D04B
:10C2E000CBEC07F0FBD73B0EE66EE1EC07F0E55236
:10C2F0000201280E246F0601F45102E00601F40742
:10C300000201FE5102E00201FE070201FD5107E0B9
:10C310000201FD070201FD5102E101013C8B010117
:10C3200097AD15D10301C6070301C65101E00FD136
:10C33000C69AF00E8C1407098C6EF8DC8A9A0000FD
:10C340000000000000000000000000000000049059
:10C3500082B804808A8AC68AF00E8C160101E0BD7C
:10C3600012D00301010EC66F04A00CD00301060E0B
:10C37000C66F0101E08D0301CA6BCB6B0301C86B73
:10C380000301C76BE4D0D8900301CB33CA33030158
:10C39000C82B04A003D00301CB8F09D00D0E0301DD
:10C3A000C85D05E20301C72B070E0301C717030190
:10C3B000040EC66F0301C8510F0801E3C8D0030182
:10C3C000960EC66F0101E09DCAC30FF0CBC310F0FB
:10C3D00000010F1C01E1101C0BE1020E6F5C07E174
:10C3E000B90E0B5C04E1248A26820601426BAFD0B1
:10C3F0000FC00FF010C010F00F1E101E10C000F084
:10C40000700E001600380F0B006E0301C751005C60
:10C4100001E09DD00F0E00011016000110A603D000
:10C42000F00E000110120FC0D4F110C0D5F10101BF
:10C43000D53504E3D4511708FC0ED55501E387D058
:10C440000101D890D55104E6E90ED45D030ED5590B
:10C4500001E37DD0D0C3CEF3D1C3CFF3D4C1D0F3A9
:10C46000D5C1D1F30A0E0F6E106A030E0301C95D28
:10C4700003E2640E0F6E106A0101D4510301CE5D18
:10C480004C6ECF510101D5554D6E4CC0E6FF4DC0ED
:10C49000E6FF97EC2EF0E552E552F3CF4AF0F4CFE9
:10C4A0004BF00F504A5C10504B584AE2D0C3CCF3CB
:10C4B000D1C3CDF3FF0E0301C95D02E20301C92B15
:10C4C000030E0301C95D22E30101D4510301CE5DD6
:10C4D0004C6ECF510101D5554D6E4CC0E6FF4DC09D
:10C4E000E6FF97EC2EF0E552E552F3CF4AF0F4CF99
:10C4F0004BF0000ED8804A54000E4B540CE202015F
:10C50000345109E1C2EC05F0000905E0CFEC2CF054
:10C510003488B1EC4BF0020E6F5C11E1B90E0B5C8C
:10C5200003E0E60E0B5C0BE1248A2682B90E0B5C5D
:10C5300006E10601080E426F06011E0E436F07D08A
:10C540000301C951020803E20301010EC96F020190
:10C550004A514B1164E01CA020D002014A07000E92
:10C560004B5B02014A514B1117E11A50200B14E0AA
:10C570001CA210D09EEC0AF054EC05F0EFC2D2F1F0
:10C58000F0C2D3F10EEC0BF00201280E4A6F230E1D
:10C590004B6F02D0A4EC0AF042D02150400B3FE098
:10C5A0001A50400B3CE01850080B03E11A50200BC6
:10C5B00036E002014A07000E4B5B1A50200B0CE0DC
:10C5C0009DEC1DF000090AE18150010B05E101011C
:10C5D0000101DE51100B02E1000E01D0010E0490AA
:10C5E000E8B0048002014A514B1103E00450010BF2
:10C5F00016E002014A6B4B6B0101DE9904A006D0E4
:10C6000002012A6B2AC26AF251EC80F0A4EC0AF013
:10C6100018A604D0259224BC2582228E21940201E2
:10C62000505102E0020150070201515102E00201A3
:10C63000510702014F5102E002014F07020146512A
:10C6400002E0020146070201425102E002014207F4
:10C65000020140510FE002014007020140510AE18E
:10C6600008504A6E4B6A820E4A1801E14B5002E0B4
:10C6700053EC0EF02B50200B56E002013B5153E1DE
:10C680000701DE5102E00701DE0701012C51070816
:10C690003AE276EC28F0000936E008AE0ED0070149
:10C6A000DE510AE17DEC14F0D5EC0FF002010F0E23
:10C6B000456F07015F0EDE6F25D00201455122E173
:10C6C000010101013951040B04E10A0E01012C5D45
:10C6D00007E12FEC0BF0060EE66E34EC29F0E55284
:10C6E0000BEC05F0D5EC0FF0010101013951040B01
:10C6F00004E10A0E01012C5D02E12AEC0BF00201BB
:10C700000F0E456F10D0800E081405E101010101E4
:10C710003951040B08E10701DE5105E1D5EC0FF0BA
:10C7200007015F0EDE6F020123070201235146E17C
:10C730000201280E236F1BAC10D077EC4AF00C508E
:10C74000006EB1EC4AF006010F7906010FA904D082
:10C750007D50006EB1EC4AF031D01CA803D0060128
:10C7600012792CD01DA203D00601147927D01A50BB
:10C77000200B07E0010101013951100B02E1060114
:10C7800005772550020B04E1C3EC0DF0000916E01B
:10C790000201405113E108504A6E4B6A820E4A185A
:10C7A00001E14B500BE02650040B06E12D50800BAD
:10C7B00005E12D50400B02E10601107105014451C5
:10C7C00029E0C2EC05F0000925E02250100B22E020
:10C7D00005014407050144514A6E4B6AD8904B50FD
:10C7E00004E6960E4A5C000E4B580CE305014451DA
:10C7F0004A6E4B6A960E4A1801E14B5002E1050160
:10C80000446B08D006011C91140E0501445D02E240
:10C8100006011C8102013B5102E002013B070201BB
:10C820003C5114E0010101018B51400B0FE0C2ECBF
:10C8300005F000090BE002013C0702013C5106E152
:10C840001B82EFECB8F01B92076A796A0701D85196
:10C8500007E00701D8070701D85102E1076A796AA2
:10C8600002013A511EE002013A0702013A5119E170
:10C87000FBEC26F0000903E193EC97F012D00701DE
:10C88000D5510701D6110DE00701D55102E007018E
:10C89000D5070701D65102E00701D6070201020EB3
:10C8A0003A6F020139510CE0020139070201395196
:10C8B00007E1178E170E676E2DAC02D00F0E676E54
:10C8C0000101A95174E00101A9070101A9516FE11A
:10C8D000ADC1F6FFAEC1F7FFAFC1F8FF0800F550DC
:10C8E000006E0201DF5107E0830E0A6EDFC201F025
:10C8F0003CEC4DF00A6A0201AA51AB1120E0010E96
:10C90000E66EAAC2E6FFABC2E6FF060EE66E010EB9
:10C91000E66E0BEC4EF04A6E050EE15E4A50016E7B
:10C9200006C100F00201AA2B000EAB233550800B8C
:10C9300005E0015003E000507F0801E2006A00506A
:10C9400015E00101190EA96F0050E66E42EC8AF065
:10C95000E5520201DF5103E00201DF2B06D00101A5
:10C96000AD2B000EAE23000EAF2321D02950080BB3
:10C9700003E13150080B02E0299619D00201DF5182
:10C9800005E00201DF6BFA0E096E04D0D89009327F
:10C99000D890093224A60BD0B20EE66EEC0EE66EED
:10C9A000010EE66E74EC2EF0E552E552E5520201FE
:10C9B000385106E0020138070201385101E1269E94
:10C9C0000201375109E0020137070201375104E142
:10C9D0000601416941C640F60101A65102E001018C
:10C9E000A6070701825102E00701820702013F51B9
:10C9F0002AE002013F0702013F5125E1000E060136
:10CA0000E76EC019E8AE02D0C03503D0E750D88039
:10CA1000C05503E20601C00702D00601C02B000E7C
:10CA20000601E76EC219E8AE02D0C23503D0E75066
:10CA3000D880C25503E20601C20702D00601C22B0C
:10CA40000201050E3F6F0301E7516AE00201345114
:10CA500067E108BE03D00301E76B62D00301E7077B
:10CA60000301E7515DE120A20BD0BAC19AF1BBC12D
:10CA70009BF1BCC19CF1BDC19DF1BEC19EF10AD02C
:10CA8000B5C19AF1B6C19BF1B7C19CF1B8C19DF196
:10CA9000B9C19EF101019A514C6E4D6AE80E4D02EA
:10CAA000F3CF4DF0030E4C02F3504D26E80E4C022E
:10CAB000F3CF4CF0F4504D2601019B510A0D4C5020
:10CAC000F3244A6E4D50F4204B6E0A0E4E6E4EC04B
:10CAD00044F09CC13FF02FECFDF03F5000014A2490
:10CAE0000F6E000E4B20106E030E0F0B05E0D8905A
:10CAF00010320F32E806FBE10301E8510F1802E1A2
:10CB0000E95110180DE00FC0E8F310C0E9F3400E32
:10CB1000016E0001105001260FC000F0A8EC91F04A
:10CB2000020131512EE00201310721BC25D0010163
:10CB3000DFA106D00201316B0101DF91F1EC27F09A
:10CB40001B50800B19E0800E081416E02150010BD9
:10CB500013E10201316B1B9E0A01DA8F54EC0DF0D8
:10CB6000010EE66EA8EC90F0E5520201020E3C6F59
:10CB70000201178B05013B850201315102E1248A34
:10CB800026820201205109E01E50400B06E00201FE
:10CB900020070201205101E11E8E0501065102E02D
:10CBA000050106070201485107E00201480702019A
:10CBB000485102E146EC0AF009506BE009060950C1
:10CBC00068E1189C189E30980101DE951D921C9812
:10CBD0002682248A289821BA13D0040E0101445DCC
:10CBE00008E1010101018E51100B03E10101E38F06
:10CBF00005D07EC1E6FFBAEC0EF0E55286EC2EF0D1
:10CC0000218A56EC93F081EC5FF001010101E351C0
:10CC1000100B14E02E50400B11E12250200B0EE0BF
:10CC2000180E675C0BE11750100B08E0020E0B6E3C
:10CC30000DEC9BF0E1EC9AF012AC178E02019551CD
:10CC400003E13250400B25E022AA1CD0092A188E9D
:10CC5000020E0201955D15E1020196514A6E4B6A82
:10CC60004B3404E24A509608000E4B5408E2AFECF5
:10CC700093F0100EE66E56EC97F0E55202D00201EA
:10CC8000962B07D0329C0201955103E0178E3A0E85
:10CC9000676E02012D5102E002012D0702012E51A3
:10CCA00002E002012E0702012F5102E002012F07CC
:10CCB0000201475102E0020147070201435102E02D
:10CCC000020143070201445102E00201440701014D
:10CCD000A85102E00101A8070301E25102E00301AB
:10CCE000E20702014C5102E002014C0702014D51E2
:10CCF0001EE02250200B0CE1110E4A6E4AC044F097
:10CD00004DC23FF02FECFDF03B5002E106010E73E7
:10CD100002014D072250200B05E02150400B02E09C
:10CD2000E3EC05F002014D5102E107EC05F00601CC
:10CD300043510EE0060143070601435103E106019A
:10CD40005A0E436F26860F0E0601435D01E22696BA
:10CD50000201325110E00101E9A503D00201010EE8
:10CD6000326F020132070201325102E16CEC84F0B1
:10CD700002011E0E316F02014E5113E0010101014B
:10CD80002751400B0EE102014E0702014E5109E10D
:10CD900045C100F01986358296ECB5F00201010E0E
:10CDA000346F0201345101E177D0020134070201EE
:10CDB000345101E071D068EC44F0B5EC45F099ECE9
:10CDC0005EF04FEC92F021A204D0219269EC38F091
:10CDD00054D02CA602D049EC2CF01AEC90F045EC83
:10CDE00015F0E4EC1CF025AC0DD025A806D0010E02
:10CDF000696EE66A60EC3BF0E552696AE66A60ECEF
:10CE00003BF0E552259C696A01018BAD07D0010119
:10CE10008B9D010EE66E2FEC5FF0E552E8EC18F00A
:10CE2000640EE66E34EC29F0E552010178B71ED0AD
:10CE30000701F1051BE03550020B18E125A80DD0C4
:10CE4000010E696E8EEC3CF0000907E1480E006EA1
:10CE500059EC2EF00101320E1F6F696A8EEC3CF026
:10CE6000000904E1480E006E59EC2EF09CECC3F072
:10CE70001CA603D0BAEC32F01C9619B008D0E0EC36
:10CE80002AF080EC56F0E66A47EC22F0E552199061
:10CE9000020117894CEC05F00201495106E002013C
:10CEA00049070201495101E126820201355102E0A0
:10CEB000020135070201415102E00201410702016E
:10CEC000335102E00201330702012C510AE0020152
:10CED0002C0702012C5105E1780EE66E66EC18F085
:10CEE000E55202012B5107E002012B0702012B053D
:10CEF00002E1A0EC12F002013E5102E002013E0705
:10CF0000120006014F6B4FC64EF64FC64DF64FC688
:10CF10004CF64FC64BF6120045ECEFF0DE52010E18
:10CF2000DD6EFE0EDB5022E158ECF2F0050EE66EEF
:10CF3000200EDF24E66E4B0EE66E060E0FECE5F0DB
:10CF400026A406D0FF0E06014B5D0FE1DADF0DD0FF
:10CF5000050E4FECF4F0B50EE66E010E0FECE5F0A9
:10CF60000F0E61ECF0F00050DF6E0A6A26B44BD071
:10CF70000101B551630807E3B5510FE10301E35126
:10CF80000101B65D0AE23E0E9EECF3F0FE0EDB50B0
:10CF900001E1B7DF010EDB6A22D0FE0EDB501FE19C
:10CFA0002D50800B07E0DF500A0804E20701EF9BD9
:10CFB000E1EC09F0DFCFE6FF10EC43F0E5520101B0
:10CFC0008B51100B0CE00A0E455D09E2A3EC93F0C7
:10CFD00075ECE7F0DFCFE6FFCCECA3F0E552020101
:10CFE000395111E1640E0101455D07E27CECE5F089
:10CFF00045C13FF034ECEBF005D04D0E196F030E38
:10D000004515310F1A6F016A050E015C31E20150BE
:10D01000EA6A4B0FE96E060EEA22EF504B6A120FD6
:10D020004A6E070E93ECEFF0026E2D0E025C05E1E6
:10D030000101B05102E1200E026E0201395116E1E8
:10D04000020E012483ECE5F002C0EFFF26A404D019
:10D050000101610E196F0AD0015008E12C9A2A0EC5
:10D06000025C04E12D50800B01E02C8A012ACCD710
:10D070002650040B05E10201395102E101011B8F29
:10D08000010EDB50B6ECEAF002E2E16AE552E16E35
:10D090004A50DEEFE4F04DECEEF0016E45518AECC3
:10D0A000E6F0050EE66E4B0EE66E060EE66E200E00
:10D0B00001249CEFF4F03450400B04E00101D951FD
:10D0C000800B09E13450400B04E10101CD51400BCC
:10D0D00002E1000E01D0010E11EFE9F034AC03D0F3
:10D0E0000101D98F12000101CD8D120034AC03D0A3
:10D0F0000101D99F12000101CD9D1200D8EC09F069
:10D100000101076F020E075D01E1070785ECEDF0F5
:10D11000EFCF06F106511F0801E2066B0490CDBD6A
:10D120000480695003E00490D9BF04801200CEEC63
:10D130000CF0EEEC1FF0E2DF300E016E0450010B3C
:10D140001AE00701EF51010B16E0030E0C5C13E02F
:10D1500097ECF3F0080B08E0CAECF0F004E61F0EC1
:10D160004A5C000E4B5807E206C1E6FFE90EEEEC02
:10D17000E4F0310E016E0150F1ECE4F09CDFF3506D
:10D180001596E8B015861200AFEC93F0110EBAECCC
:10D19000E8F0B4DF010106510F0802E26D0E1B6FCB
:10D1A0000651EFECEEF0310F1D6F030E0615310F37
:10D1B0001F6F97EF68F0248E2096006844EC2EF0E5
:10D1C000C4EF68F0249E04EC0EF034AC02D060ECA6
:10D1D000EEF012003450400B04E00101D951010B74
:10D1E00009E13450400B04E10101CB51200B02E175
:10D1F000000E01D0010E11EFE9F07CECE8F0EF0435
:10D20000016E98ECEAF001C03FF02FECFDF03B50CE
:10D21000026E98ECEAF001C03FF0D1ECF0F0036E42
:10D2200004900101CBBB0480695003E00490D9B1A4
:10D230000480110EE66E430E02246EECE5F0E66EFD
:10D24000A90E0AECE5F04A0E03246EECE5F02BEC97
:10D25000F2F00450010B02E0012802E1000E01D0BF
:10D26000010E000902E0370E01D0360E2BECF2F071
:10D27000006A02B004D003280E0DF350006E005077
:10D28000E66EA30EEEECE4F0100E4A6E6AECE8F0E7
:10D290004A50EF1622A832D0700E4B6EEE0E4C6E36
:10D2A000010E4D6EC4ECE7F0EF044E6E4F6A506A0B
:10D2B0004B504E24F36E4C504F20F46E4D50502086
:10D2C000D6ECEFF00800F5CF4AF06AECE8F04A50EF
:10D2D000EF120450010B04E0C4ECE7F0EF5002E160
:10D2E000000E01D0010E4A6E6AECE8F03CECEBF067
:10D2F000DF0EEF14F310EF6ECAEC0EF06BDFF3509D
:10D300001594E8B0158404B002D00501446B1200F6
:10D31000A3EC93F0170E60ECE6F07CECE8F0EF5035
:10D3200006E12DECEFF00E0E60ECE6F010D07CEC98
:10D33000E8F098ECF2F03F280101166F0E0E176F1F
:10D3400098ECEAF0D9ECE7F03B280101186FAFEC5C
:10D3500093F0910EB1ECE8F022A823D00101030E66
:10D36000016FC4ECE7F0EF5003E10107A60E17D000
:10D37000C4ECE7F098ECF2F03B50310F01011F6F65
:10D380001F5102E1630E1F6F070E005C02E23E0EAA
:10D3900006D00E0E005C02E2410E01D0440EB1EC4C
:10D3A000E8F013EFECF0308AD7ECE6F0209688EF47
:10D3B00069F0309A04EC0EF034AC02D060ECEEF080
:10D3C0001200A3EC93F0050E0C5C1BE10101030EAF
:10D3D000006F020EE66E710E0301A7254C6E070E5C
:10D3E000A8214D6E0201B251E8245EECEFF018EC7A
:10D3F000EAF014EC2EF0040E55ECF3F00101188F56
:10D4000029D0030E0C5C1AE158ECE7F009E0220E7B
:10D4100025ECF0F060ECE6F0B30E60ECE6F01AD02C
:10D4200048ECEEF00101006F14EC2EF00101100E3B
:10D43000146F15510FE1100E156F0CD0B7ECF3F00F
:10D440002AC100F084EC96F00101155102E1100EA2
:10D45000156F186BAFEC93F0AE0E006E58ECE7F062
:10D4600002E0B40E006E050E0C5C07E1E90E006EE2
:10D470000201B4A502D0E20E006E0050B1EFE8F058
:10D480002580D7ECE6F020969CDF050E0C5C06E0CC
:10D49000E1EC18F0030E006E37EC91F01200050E6F
:10D4A0000C5C03E14AEC09F004D046EC0AF0E8EC2D
:10D4B00018F0259004EC0EF059EF0FF0A3EC93F068
:10D4C00078501DE0030E785C07E11F0E006E01012D
:10D4D00078AD09D03F0E06D02D0E006E010197A148
:10D4E00002D04B0E006E84EC96F00101115102E166
:10D4F000100E116F002BA40E006EA7EC2DF0AFECF8
:10D5000093F09B0E4A6EE90E4B6E010E4C6E7850F6
:10D510004D6E19ECE5F090EFE6F03380D7ECE6F0D5
:10D520002096CCDF3EEF4BF0339004EC0EF0A1EFF1
:10D530006CF0D9ECE4F0CDECE8F01CE0FE0EDB5032
:10D5400002E0350E01D0340EF1ECE4F049ECE9F0E4
:10D5500011E02150200B0EE0010E696ECDECE8F0D9
:10D5600008E0FE0EDB5002E0350E01D0340EF1EC87
:10D57000E4F0696ADEEFE4F0E66A32ECE9F0A50E69
:10D580009BECF3F0D1EFF1F04CECEFF00701BC5164
:10D59000B15D14E11550100B01E0010E4A6E3450DC
:10D5A000010B4A5C0BE11550200B01E0010E4B6EA4
:10D5B0003450020B01E0010E4B5C2EE0696AB1C7EA
:10D5C000BCF7349015B83480349215BA348215A85B
:10D5D0001DD015AA16D0CDECE8F010E00701B1512E
:10D5E000140D69ECE5F0C8DF01013CA907D0010E7C
:10D5F000696ECDECE8F001E0BFDF696A010EE66E0E
:10D6000006D0E66A96DFE552330E04D0E66A91DF73
:10D61000E552320E4AECE7F054EFEFF00701B1515A
:10D62000140D69ECE5F02AEC2EF01CC119F11DC1B6
:10D630001AF11EC11BF11FC11CF10101200E1D6F4B
:10D64000480E1E6F5A0E1F6F300E195D02E1200E3C
:10D65000196FC4EF6AF0318C2096006844EC2EF00C
:10D660000EEF6BF0319C04EF0EF0095004E02550F2
:10D67000080B01E130880D0E005C03E185ECF0F051
:10D6800009D00A0E005C03E190ECF0F003D00050EA
:10D6900043ECE6F0095006E03050100B03E1FA0EBF
:10D6A000096E25861200010E0701D8908337843752
:10D6B000E806FBE122AC02D0070183810D0E0701D1
:10D6C000855D01E2852B1200229C8650020B01E051
:10D6D000228C07017B5111E122AC51D07B2B010E32
:10D6E000836F846B856F3198866F7E51FE0BE842A5
:10D6F0007E257D6F010124931200010124A33FD0F8
:10D70000249307017B053BE122BC2BD031A826D016
:10D710000C0E855D20E2D89084338333000E835D48
:10D72000040E845918E23A0E83254A6E020E8421B3
:10D73000F6ECF3F024ECE7F0006E090E005C03E178
:10D740000DEC8AF008D0005006E0610E005C02E3A8
:10D75000200E005E8ADF07017B6B1200318853EFD9
:10D760006BF0A1DF31A804D00701010E866F06D04F
:10D770000701862B86510C0801E27B6B3198120061
:10D7800008AE05D0229C8650020B01E0228C0701D6
:10D790007B5110E122BC76D00101249307017C6B00
:10D7A00008AE70D0020E7B277E51FE0BE8427E252C
:10D7B0007D6F12007B050BE17B2B7EC77DF701019E
:10D7C000249322AC5FD00701080E7B6F1200010189
:10D7D00024A358D02493070E07017B5D47E17B6BA0
:10D7E00022AC41D0095004E02550080B01E13088FB
:10D7F0007C514D6A3A0F4C6E060E4D227F515EEC05
:10D80000EFF024ECE7F0006E810E005C03E107010D
:10D810007F6B20D0800E005C04E10701200E7F6F3B
:10D8200019D00D0E005C03E185ECF0F013D00A0E68
:10D83000005C03E190ECF0F00DD00B0E005C02E117
:10D840002A0E06D00A0E005C05E0005003E00050EE
:10D8500043ECE6F0095009E03050100B06E1FA0EF7
:10D86000096E25861200080E7B6F1200080E7B5D84
:10D8700004E122AC07D07B6B12007C917C4322BC7C
:10D880007C897B2B1200A3EC93F0810E60ECE6F018
:10D890000C5008E10601F15105E10101002B640E75
:10D8A00060EFE6F0B7ECF3F0F1C600F0030E0C5CAD
:10D8B00002E1F3C600F084EC96F0050EE66E040E6D
:10D8C000EFEFE7F0E0DFAFEC93F0030E0C5C14E158
:10D8D00007ECEFF006E0590E4A6EF20E4B6E010EA9
:10D8E00005D0540E4A6EF20E4B6E010E4C6E3EEC9D
:10D8F000E5F04CC0E6FF0AD08C0E4A6EE90E4B6E86
:10D90000010E4C6EF0C64DF019ECE5F090ECE6F02F
:10D9100048EC26F029EC12F0006E00500A01D65DAA
:10D9200004E200C0D6FAB1ECF1F012003184D7EC79
:10D93000E6F0209662EF6CF0319404EC0EF0A1EF6B
:10D940006CF08CECEDF0A00E32ECF0F0140E016EE9
:10D950003DC100F0FDEF4CF041ECEFF0E6C64AF0BF
:10D96000E7C64BF041ECECF0060185ECEEF00BE382
:10D97000E4C64CF0E5C64DF0EBECEEF0E6514C5C45
:10D98000E7514D581FE2E451E6250F6EE551E721BE
:10D99000106ED89010320F329BECEAF0030E23EC9D
:10D9A000F2F0FDE14A500601E85F4B50E95B42ECC2
:10D9B000E7F0030E23ECF2F0FDE14A500601E82700
:10D9C0004B50E923E4C6E6F6E5C6E7F69BECEAF041
:10D9D00041ECECF041ECECF085ECEEF00BE39BEC71
:10D9E000EAF005ECE8F005ECE8F04A50E45D4B5055
:10D9F000E55902E2DF6A09D0E851E45DE951E559F1
:10DA000002E2010E01D0020EDF6E9BECEAF041EC67
:10DA1000ECF04A50E825EA6F4B50E921EB6FDF50FC
:10DA2000E552DEEFE4F0229C8650020B01E0228CEE
:10DA300022AC03D00201812B02D00201822B825141
:10DA4000BFECE8F001E14B5008E081514C6E4D6AAB
:10DA5000FF0E4C1822E14D5020E18151BFECE8F05F
:10DA60000DE14B500BE1805153ECE5F004E6FF0E65
:10DA70004A5C000E4B5805E2802B03D0805101E038
:10DA800080070601F15105E180C2E6FFE20EEEECEF
:10DA9000E4F00201826B82C281F2209E0601EC5109
:10DAA00009E122AC45D0010EEC6FE46BE56BED6B48
:10DAB000EE6B3ED0EC0515E122BC3AD0020EEC6FC5
:10DAC0004BDF006E00500BE0070E0601EE5D07E233
:10DAD000EE2BED91ED430050010801E2ED8F0601C0
:10DAE00019D0020EEC5D24E122AC17D09BECEAF0D9
:10DAF000030E23ECF2F0FDE106014A50E85D0F6EE3
:10DB00004B50E959106E0F50E45D1050E5590EE28C
:10DB1000010EEC6FE46BE56B0BD0EA51EA254A6E1F
:10DB2000EB51EB214B6E85ECEEF002E2030EEC6F55
:10DB3000030EEC5D68E1ED91ED43ED8F070ED880AB
:10DB4000EE55016E01500106000903E0ED91ED4331
:10DB5000F9D7780EED5D55E2095004E02550080B29
:10DB600001E13088EDC6E6FF67EC04F0E552006E97
:10DB7000200E005C03E300506E0802E22A0E0BD078
:10DB80002A8A005043ECE6F00601E451EA5DE551D3
:10DB9000EB5903E2200E43ECE6F0040E0601F05DC3
:10DBA00026E12AAA0CD0600E3E6E090E3F6EE8C632
:10DBB00043F0E9C644F0EBECFCF03EC0EFF6E5ECD8
:10DBC00089F0000914E00101390E1A6F1AC119F128
:10DBD0006E0E1B6F640E0601EF5D07E27CECE5F054
:10DBE000EFC63FF034ECEBF01A6F01011C8F2A9A5C
:10DBF000095007E03050100B04E12586FA0E096E3B
:10DC000031860601EC6B208E12000101DF830C507F
:10DC100002E109DF07D0209EBEECEAF002E054DD0D
:10DC200001D0AEDD0101DF931200800E081418E070
:10DC30002B50020B15E12150200B12E00201DF51A5
:10DC40000FE10C5004E10601F051010806E3030E58
:10DC50000C5C06E107ECEFF003E02A0E18140DE06F
:10DC6000800E081409E1F1ECE5F006E00601F2513E
:10DC700003E002013D5101E0000C010C02014C5196
:10DC800003E1120E06ECE5F01200D9ECE4F006C256
:10DC900001F007C202F02DA203D0020ED4ECE7F08F
:10DCA00049ECE9F040E03851800B3DE1020ED4EC44
:10DCB000E7F002010A5153ECE5F002E647ECE7F029
:10DCC00015E20A514A6E4B6A800E78ECF1F0036E51
:10DCD00003504E6E4F6A0250FDECE5F0070E0F0B3D
:10DCE00003E027ECF2F0FDE14A50025E02010A5126
:10DCF000D5ECE5F018E24A508008000E4B5413E2D0
:10DD00000A5157ECEAF04A50036E03504E6E4F6AC8
:10DD10000150FDECE5F0070E0F0B03E027ECF2F0ED
:10DD2000FDE14A50015E69CFC7F2696AFE0EDB046D
:10DD300009E00150E66EA60EEEECE4F00201188355
:10DD400035B09CDFFE0EDB5009E00250E66EBF0EE0
:10DD5000EEECE4F0020118851DB890DFC7C269FF40
:10DD6000DEEFE4F035ECF0F004E228ECE8F001E25C
:10DD7000006A35ECF0F007E24A50E308000E4B541D
:10DD800002E2E30E006E00508AECEEF00024006E1A
:10DD900035ECF0F005E228ECE8F002E2FA0E006E55
:10DDA0001200F2ECF0F02C51615D03E178501DECB3
:10DDB000F0F0A1EF6CF0A5EC0DF0B8EC25F0B1ECB3
:10DDC000F1F0E4EC1CF039ECECF02050020B05E033
:10DDD000BEECEAF002E06BECEBF0B1EC4BF04CEF98
:10DDE00005F041ECEFF0DEEC13F09CEC5FF021AAC3
:10DDF00007D00301E65102E0E60702D0EDEC92F015
:10DE000014DF000902E001DF01D0209E2550200B25
:10DE100006E00201345103E199EC5EF0259A37ECFB
:10DE2000E8F012E03450400B0FE10101CB51200B20
:10DE30000DE0050140510AE08450040B07E1445114
:10DE400005E1280E446F02D00501446B02013B51ED
:10DE500002E067EC51F00101B15112E12850010BD1
:10DE60000FE15AEC34F0006E1EAC83EF78F007013E
:10DE7000D351F00BE83AD35D0024D36F83EF78F0F1
:10DE8000B1051FE12850010B1CE185EC8BF052EC31
:10DE90002FF037ECE8F002E183EF78F03BECE8F0AC
:10DEA00002E183EF78F02D50400B02E083EF78F031
:10DEB0002D50800B02E083EF78F0ABEC2EF083EF77
:10DEC00078F0020EB15D09E12850010B06E14AEC41
:10DED00014F0D2EC93F083EF78F0030EB15D07E11C
:10DEE0002FB483EF78F09AEC97F083EF78F0040E7C
:10DEF000B15D01E0B9D00201355102E083EF78F065
:10DF00001750100B03E11750010B02E0000E01D077
:10DF1000010E2390E8B0238022AA4ED087ECE9F0CE
:10DF2000166E23A036D00101A6511EE1165002E163
:10DF3000010E01D0100E8009176E2850010B03E16D
:10DF40000E0E675C05E10201030E286F640E226F5E
:10DF500028A004D0480E8DECEEF03FD0FBEC09F089
:10DF600000093BE01B8439D0165003E00C0E165C10
:10DF700034E1810E176E165001E1229A0201020E61
:10DF8000356F28A003D0540E8DECEEF00201286B03
:10DF900024D0165022E12350010B1FE1229A285071
:10DFA000010B06E00C0E675C03E1520E8DECEEF007
:10DFB0000201020E356F11D032B40FD0E66ACCECFC
:10DFC00051F0E552000909E032840201020E356F7A
:10DFD000640E416FDF6B08AE356B3250040B02E10B
:10DFE00083EF78F00201355102E083EF78F032944C
:10DFF00087ECE9F0166E165002E183EF78F001012C
:10E00000280EA66F2A0E165C05E12150400B02E097
:10E010001E0EA66F0A0E165C09E0090E165C06E0DD
:10E02000120E165C03E0110E165C02E12D0EA66FB7
:10E03000350E165C02E1FA0EA66F0201020E356F74
:10E04000228A176A1650676E28B005D0FBEC09F0DB
:10E05000000901E01B8429B602D00101A96BA5ECDF
:10E060000DF02B8483EF78F0050EB15D0FE12751A1
:10E07000100B05E12851100B02E167EC51F028A0CC
:10E0800083EF78F05AEC58F083EF78F0060EB15D2C
:10E0900007E121AA83EF78F021EC08F083EF78F014
:10E0A000070EB15D01E0B7D12650800B18E00201E8
:10E0B000385115E192ECEEF002011E0E386F269EEB
:10E0C0002850020B0CE02A50010B09E1510E58ECCC
:10E0D000E5F0300E58ECE5F0010E9BECF0F026ACCC
:10E0E00003D037ECE9F0269C26AA03D046EC0AF0D0
:10E0F000269A01013751800B1BE00201485118E1BB
:10E100001BA404D0040E12ECF1F01B941BA604D047
:10E11000070E12ECF1F01B961BA804D0060E12ECB1
:10E12000F1F01B981BAA04D0050E12ECF1F01B9A1B
:10E130002250080B02E083EF78F02B50400B02E0F6
:10E1400083EF78F002010B5139E1D70ED9ECE5F0FD
:10E150001F9A1FB01F8AE66801C2E6FFA0ECEAF032
:10E160000201016F1F901FBA1F801F50100B04E1A6
:10E170000101E151080B22E028A006D001C2E6FF10
:10E18000470E17ECECF019D001C200F00101E1A735
:10E1900003D0DDC300F0E197030E005E35ECF0F034
:10E1A00004E228ECE8F001E2006A00C006F238BFA1
:10E1B00002D000C007F2E66A68DDE55202010B05F5
:10E1C00048E1CF0ED9ECE5F01F9A1FB21F8AE6682E
:10E1D00002C2E6FFA0ECEAF00201026F1F921FBA32
:10E1E0001F821F50100B04E10101E151100B31E0BF
:10E1F00028A006D002C2E6FF480E17ECECF028D0AB
:10E2000002C200F00101E1A903D0DEC300F0E199F0
:10E21000030E005E35ECF0F004E228ECE8F001E2D9
:10E22000006A00C00AF238AF06D00201800E0A6F01
:10E2300000C007F20AD035ECF0F007E24A50E308DC
:10E24000000E4B5402E202010A69010EE66E1DDD6A
:10E25000E552020E02010B5D45E1E70ED9ECE5F057
:10E260001F9A1FB41F8AE66803C2E6FFA0ECEAF01B
:10E270000201036F1F941FBA1F841F50100B04E18B
:10E280000101E151200B2EE028A007D003C2E6FFD8
:10E29000490E17ECECF0E55225D003C200F0010165
:10E2A000E1AB03D0DFC300F0E19B030E005E5ADD5B
:10E2B00000C008F2005065ECE8F0006EAEECEAF049
:10E2C0000AE208C209F20050E66EA70E82ECEBF0FB
:10E2D0000201188905D069CFC7F2696A01ECF2F032
:10E2E00002011887030E02010B5D01E08AD0EF0ED8
:10E2F000D9ECE5F01F9A1FB61F8AAEECEAF009E2EE
:10E300009E0EE66E05C2E6FFA0ECEAF00201056F84
:10E3100007D0E66804C2E6FFA0ECEAF00201046F51
:10E320001F961FBA1F861F50100B04E10101E15117
:10E33000400B67E028A00CD0AEECEAF003E205C287
:10E34000E6FF02D004C2E6FF4A0E17ECECF038D02C
:10E35000AEECEAF037E21CECECF005C200F0010193
:10E36000E1AD03D0E0C300F0E19D030E005C0701C6
:10E37000056F0551D5ECE5F004E228ECE8F001E288
:10E38000056B0539E8461F0B056F05511D0802E2B4
:10E390001D0E056F050E0C5C03E0050E7D5C03E1B0
:10E3A0008DEC0CF02ED02150200B2BE002014151BE
:10E3B00028E1010157BD25D0130EE66E6EEC2EF05C
:10E3C000E5521FD004C200F0E1AD03D0E0C300F07D
:10E3D000E19D030E005EC6DC35ECF0F004E228ECB3
:10E3E000E8F001E2006A00C009F2005065ECE8F0D4
:10E3F000006E69CFC7F2010E696E01ECF2F0020106
:10E400001889030E02010B5D01E12D920B2B030E07
:10E410000B1783EF78F0080EB15D02E0E3EF76F0C2
:10E420002850010B02E0E3EF76F018BC3DD118A8AC
:10E43000E0D021AE0FD0A85101E0F4D02CA805D037
:10E44000CFC1E6FF9DEC53F003D0E66ADEECC5F0E9
:10E45000E552E8D025A03CD027AD7DD016EC09F0E0
:10E460000C500DE1500EE66E1E0EE66E2A0EE66EA4
:10E47000010E00ECE5F0010195ECEEF01CD058EC3B
:10E48000E7F009E0030EE66E2F0EE66E010EE66E73
:10E4900006EC9DF00DD0050E0C5C0DE1330E2EEC5C
:10E4A000F4F0B20EE66E020EE66EFCEC9CF0E55265
:10E4B000E552E552E55240EC6AF0B1ECF1F0E4ECE3
:10E4C0001CF002010A0E3C6F05013B853B8F43D0D7
:10E4D00033A018D027AD13D058ECE7F003E00101CA
:10E4E000977105D0BEECEAF002E00101787DA5EC61
:10E4F0000DF0B8EC25F048EC26F05EEC6AF0010176
:10E50000279D5FD031A416D027AD25D016EC09F099
:10E510000C5006E1060EE66EF10EE66E060E05D014
:10E520001E0EE66EF30EE66E060EFBECE4F062ECF9
:10E530006CF011D030AA11D027AD0DD016EC09F037
:10E54000150EE66E69504B6A420F4A6E050EC2EC1C
:10E55000EFF088EC69F0010134D02D50400B03E15D
:10E560002D50800B30E027AD5DD016EC09F0010195
:10E57000B0511AE1630EE66E450EE66E010EDDEC5B
:10E58000E6F045C11FF202014E6BB5ECE8F0000960
:10E5900017E02D50800B14E001018F51100B10E19A
:10E5A0000201100E4E6F0CD0290EE66EB0054B6ABC
:10E5B0004B0F4A6E060EC2ECEFF09AECEEF0E5520D
:10E5C0000101A86B2FD029A20DD027AD2BD016ECBE
:10E5D00009F0E6686A0EE66E030EFBECE4F051EC1F
:10E5E000C5F020D022B61ED06FC200F03AEC2EF05B
:10E5F00019D018A205D026A215D02692238212D0B7
:10E6000018A010D026A206D026922CC1E6FF10EC4E
:10E6100043F0E5520201315105E11B50400B02E18C
:10E620003EEC4BF019EC16F0006EFF083DE0420E98
:10E63000005C03E0450E005C15E129C70FF02AC716
:10E6400010F0450E005C04E107012B510F6E106ABB
:10E6500000683AEC2EF00101150E116F030E006FE9
:10E6600014EC2EF05D0E005C16E10101150E116F29
:10E67000100E126F020E006F2CC7E6FF05EC2EF095
:10E68000E5522DC7E6FF05EC2EF0E5522EC7E6FF5A
:10E6900005EC2EF0E5527E0E005C06E1A3EC93F053
:10E6A000E80E006E3AEC2EF018BE73D318AAA5D16E
:10E6B0002DA603D09FEC54F054D32DA403D06DECC1
:10E6C00054F04FD331A425D0010128AD17D0010E4D
:10E6D0000E6E28BF0E680C5005E18CECEDF006ECD8
:10E6E0009DF008D0010EE66EF20EE66E060EE66EA6
:10E6F000F6EC9CF0CBECF3F0B1ECF1F02450200BF5
:10E7000005E101012851400B01E184D062EC6CF07D
:10E7100081D033A01ED0010128AD0DD0010E0E6EA8
:10E7200028BF0E6878CF06F1030EA0ECF4F006C106
:10E7300078FFD1EC6EF02450200B04E10101285148
:10E74000400B68E0DBEC6EF05EEC6AF002011981D0
:10E7500061D025A00CD0010128AD46D10201B475CD
:10E760003EEC4BF040EC6AF00101289D3DD130AA0F
:10E770001AD0010128AD0DD0010E0E6E28BF0E6813
:10E78000150EE66E69504B6A400F4A6E050EC2ECDC
:10E79000EFF02450200B04E101012851400B3AE036
:10E7A00088EC69F037D024AE1AD0010128AD0ED024
:10E7B000010E0E6E28BF0E687EEC68F01F0E2AEC6C
:10E7C000F4F0010185ECEDF006C1EFFF2450200BC1
:10E7D00003E12851400B1EE0C4EC68F01BD031ACC3
:10E7E0001DD0010128AD0DD0010E0E6E28BF0E68A0
:10E7F000C40EE66E0A0EE66EB10EE66E070E00EC73
:10E80000E5F02450200B04E101012851400B02E007
:10E810000EEC6BF00101289D249AE6D02D50400BA0
:10E8200003E12D50800B34E024AA04D0249A9AEC02
:10E83000EEF061D0010128AD94D2289D010E0E6E3C
:10E8400028BF0E68006A26B4002A050E03ECEFF01C
:10E85000B00EE66E010E00ECE5F00601030E426F0D
:10E860000101B0510EE0B0294A6E010E4A5204E097
:10E87000E846FE0B4A06FCE10601426F1E0E436F9E
:10E8800002D04BEC68F09AECEEF0E5520101ACD00E
:10E8900029A215D024AA02D0249A0ED0010128ADB5
:10E8A00060D2289D010E0E6E28BF0E68E668690EC4
:10E8B000E66E030EFBECE4F051ECC5F052D221AE53
:10E8C0001CD00101A85101E04CD2CFC101F023A816
:10E8D00002D0DDEC82F0006A2C50100B05E10FEC49
:10E8E000EFF002E2010E006E0050E66E0150E66E9F
:10E8F000CDEC53F0E552E55234D21CA277D0AFEC08
:10E9000093F0140EBAECE8F0AEEC04F05A0ED88096
:10E910000054006E0050036EA1EC96F00101200E31
:10E920001D6F0201F151035C03E201012A0E1D6F0C
:10E93000010128AD58D0289D9EEC0AF0E4EC0AF0C5
:10E94000190E026E0101DFAF02D01A0E026E28BF4F
:10E9500009D06E0E02014A5F000E4B5B025091EC33
:10E96000F1F008D06E0E02014A27000E4B23025030
:10E9700063ECF1F04A514B1106E0280ED8804A555D
:10E98000230E4B5519E2010128BF0AD00201280EBF
:10E990004A6F230E4B6FEFC20FF0F0C210F00CD095
:10E9A0006E0E02014A6F4B6B02506AECE7F0EF5DAE
:10E9B0000F6E4B50F059106E0301D2510F5CD351C2
:10E9C000105804E2D6510F26D75110220F50D45DB3
:10E9D0001050D55904E2D6510F5ED751105AE5ECCC
:10E9E000EBF00EEC0BF00101A86BBBD122B6B9D154
:10E9F00070C200F044EC2EF0B4D118B2B2D118A617
:10EA000016D0AFEC93F00A0E006EBCEC2DF00101B5
:10EA1000040E016F03C700F01AAC02D0AEEC04F094
:10EA2000A1EC96F01AAC9DD10101200E70D125EC1D
:10EA3000EFF001E17ED12E50400B01E07AD1060EBD
:10EA4000006E2BA502D00A0E006E0050D8807755BC
:10EA500001E2776B28AD1FD0289D010E0E6E28BFF6
:10EA60000E680050E66E770EE66E010EFBECE4F0E9
:10EA7000050E0101775D0BE12B50200B03E02B50BD
:10EA8000010B05E028BF02D0772B01D077070201E8
:10EA9000FC6B0101A86BA85101E063D12150200B50
:10EAA00001E15FD10201DF5101E05BD10A0E0101FA
:10EAB000775D3FE1AFEC93F0C2EC18F001012B0E53
:10EAC000196F000110AE0BD001012D0E196FFF0E52
:10EAD000D8800F561056010E0F26000E1022E70E9A
:10EAE0006CECEEF004E2E70E0F6E030E106E0F50AA
:10EAF000101003E10101200E196F42ECE7F0640EE3
:10EB000077ECF2F04A50006E0101012BA1EC96F077
:10EB1000A4EC04F0300F01011A6F300E1A5D02E10F
:10EB2000200E1A6F1C8F640E1D6F420E1E6F560E44
:10EB300055D0090E775D1EE1AFEC93F0B6EC18F0FE
:10EB40002AEC2EF00101410E196F460E1A6F560E77
:10EB50001B6F300E1C5D01E004D1200E1C6F300EC7
:10EB60001D5D01E0FED07BECEEF001E0FAD0200E5E
:10EB70001E6FF7D0050E775D03E0060E775D30E17E
:10EB8000AFEC93F00101500E196F410E1A6F050E94
:10EB9000775D03E1DDC700F006D0460E196F500E19
:10EBA0001A6FDFEC14F000AE04D0006C01012D0EE2
:10EBB0001B6F0101030E016FA1EC96F0300E0101F5
:10EBC0001C5D0BE11BC11CF1200E1B6F300E1D5D87
:10EBD00004E11CC11DF1200E1C6F430E1F6FC1D03C
:10EBE000070E775D04E0080E775D01E077D0AFECAB
:10EBF00093F00101500E196F4C0E1B6F1BC11AF1DF
:10EC0000310E1C6F69CFC7F2070E775D02E1696AAA
:10EC100003D01C2B010E696E8EEC3CF0C7C269FF5D
:10EC2000010178A73BD0AFEC93F04C0EE66EF20EEC
:10EC3000E66E010EE66E90ECE6F0080E0101775DDF
:10EC400001E11C2B69CFC7F2696A080E775D02E10A
:10EC5000010E696E530E3AECE9F0005003E1020137
:10EC6000FC5119E0005006E00201FC51005C02E09A
:10EC700000C0FCF201012A0E1D6F0201FC390F0BCE
:10EC800021ECECF001011E6F0F0E0201FC1521ECCE
:10EC9000ECF001011F6FC7C269FF63D00050150D72
:10ECA00069ECE5F042ECE7F0060E23ECF2F0FDE152
:10ECB0004A50006E0050DF6E0201345152E182EC86
:10ECC000E9F00101200E1D6FDF50480803E3040E38
:10ECD000DF5C02E22A0E1D6F1F8F43D0020E775DAC
:10ECE00005E1F5EC52F0010E096E3BD0030E775DA5
:10ECF00010E1AFEC93F01EC200F0A1EC96F0300EE4
:10ED00000101195D02E1200E196F1B8F560E1D6F58
:10ED100028D0040E775D03E1BCEC12F022D07751CD
:10ED200003E149ECC4F01DD077051BE179ECC4F098
:10ED300018D002012A510AE02850400B12E1140EAB
:10ED4000095C0FE2810E73ECE5F00BD018A009D03E
:10ED500024AA03D0249ABDEC43F02EAC02D03EECA2
:10ED60004BF019EC16F0006EFF0813E07E0E005C0D
:10ED70000CE1006844EC2EF0440EE66EF20EE66EF6
:10ED8000010EE66E90ECE6F004D00050006E44EC0C
:10ED90002EF00101A85101E0B6D1140EA86F0201B6
:10EDA0006B5101E06B07020E6F5C01E0ACD1CD0E40
:10EDB0000B5C07E0B30E0B5C04E0A10E0B5C01E002
:10EDC000A2D12682A0D1090EB15D03E113EC51F06E
:10EDD0009AD10A0EB15D08E12850010B05E189ECDA
:10EDE00095F06CEC95F08FD10B0EB15D01E08BD1FD
:10EDF0002850010B01E087D1B25110E1BEEC14F0B4
:10EE00009050800B01E179D19050400B01E175D118
:10EE1000909C1E0EE66EF6EC15F06ED1B20511E177
:10EE2000800E08140BE13951040B01E066D12C511E
:10EE3000070804E25CECE6F001E05FD10BEC05F0C2
:10EE40005CD1020EB25D4AE11AEC14F00701DC0E4F
:10EE5000D880DB55000EDC5501E34FD15CECE6F0C9
:10EE600001E14BD1DBC70FF0DCC710F0016A030EE4
:10EE7000015C09E21AEC14F00701DB510F26DC51AA
:10EE80001022012AF4D7020E0F0B05E0D8901032A1
:10EE90000F32E806FBE1DC0E57ECE6F001E32DD182
:10EEA0003D0EE66EF20EE66E010E93ECEDF0010EF5
:10EEB000006EF00E57ECE6F002E2050E006E0FEC6D
:10EEC000EFF004E20050495FACECE8F0780E01018D
:10EED000495D01E312D183EC0FF00FD1030EB25D57
:10EEE00003E16CEC0FF009D1040EB25D39E121AC05
:10EEF0000CD03250010B09E002018851070805E2ED
:10EF00001450080B02E0640E436F2150400B01E0E7
:10EF1000F4D002013B5101E0F0D001015751200B28
:10EF200001E0EBD0F00E8C1625AE287E28AE02D084
:10EF3000030E8C1267EC0CF000090DE067EC0CF08E
:10EF4000000909E067EC0CF0000905E0258E150EBC
:10EF500006ECE5F002D025BE259EF00E8C16CDD035
:10EF6000050EB25D34E1060150932550020B12E10B
:10EF70002050020B04E0BFEC31F0000909E013500F
:10EF8000080B03E11350040B05E002ECEEF002E085
:10EF9000060150832550020B01E0AFD0F0ECEAF0FF
:10EFA00001E0ABD00201405101E0A7D0A9ECEBF0A9
:10EFB00001E14B5001E1A1D02D50800B01E09DD02B
:10EFC0002D50400B01E099D00601108196D0060E1D
:10EFD000B25D44E15751040B3FE02050080B3CE088
:10EFE000DF0ED9ECE5F02BBC23D0CAECF0F002E642
:10EFF000FFECEDF001E381D01E0E64ECE5F0DF0ED6
:10F000003FECF4F0016E050E64ECE5F0DF0ED9EC98
:10F01000E5F0030EE66E015003ECEFF0D1ECE6F004
:10F020006CE02B8C47EC0CF002013C0E466F65D077
:10F0300035ECF0F00BE24A50B908000E4B5406E2F2
:10F040002B9C1E0EE66E34EC29F056D00201465180
:10F0500054E147EC0CF051D02B9C4FD0070EB25D21
:10F060004CE137ECE8F049E02150200B46E060EC41
:10F07000F4F0C09EF00E8C160F6A106A01013CB9C4
:10F0800003D0190E0F6E106A42ECE7F0FA0ED8802A
:10F090004A56000E4B56C3504A5CC4504B582DE2A2
:10F0A0000201EC2BEC51030828E2EC6B010158AD96
:10F0B00007D0589D2FEC9BF07BEC1EF0160E19D05C
:10F0C0006950DF6E696A02010691064306C2E6FFD7
:10F0D000A60EEEECE4F001013CA908D00201079174
:10F0E000074307C2E6FFBF0EEEECE4F0DF50696EA7
:10F0F000170EE66E6EEC2EF0E5520101B22BB25106
:10F10000070801E2B26B0101B12BB1510B0801E21A
:10F11000B16BE552DEEFE4F0016A700E015C0EE2C5
:10F12000000E4A6EEE0E4B6E010E4C6E01504D6E8F
:10F1300053ECF4F0D5ECE8F0012AEFD71200026AA4
:10F14000300E025C08E2B00E0224016E0A0ED5EC0D
:10F15000E8F0022AF5D7120041ECEFF07A0EB1EC9C
:10F16000E8F069EC95F0010E0A6EDF6A100EDF5CC4
:10F1700035E2026A100E025C2FE23CECF0F003E094
:10F18000050E025C06E1DF50E824860F6EECE5F028
:10F19000006E020403E0060E025C07E1DF50E82483
:10F1A000860F010F6EECE5F0006E020EDF5C06E3E9
:10F1B000030EDF5C03E00A0EDF5C0AE10A0E025C6C
:10F1C00002E1110E006E0B0E025C02E1240E006ED5
:10F1D000FDEC4CF0022ACED7DF2AC8D7AC0E016E68
:10F1E000580ED5ECE8F0020E0A6EDF6A090EDF5CFD
:10F1F00012E2026A100E025C0CE23CECF0F003E05A
:10F20000050E025C02E11C0E006EFDEC4CF0022AC1
:10F21000F1D7DF2AEBD70A6A7FDFDF6A200EDF5CD7
:10F2200009E2100E006E800EDF24016EFDEC4CF042
:10F23000DF2AF4D7DF6A0B0EDF5C03E280DFDF2A10
:10F24000FAD7DF6A090EDF5C31E2DF28006E003892
:10F25000F00B006E090E0012DFCFE6FFF7EC0BF0AB
:10F26000E5529EECF2F0EE52090E90ECF3F0EAEC6F
:10F27000EBF02C0E90ECF3F0030E09ECF0F0010E25
:10F2800090ECF3F0040EBEECF0F0050EBEECF0F0E6
:10F29000070EBEECF0F0080EBEECF0F0060EBEEC71
:10F2A000F0F0090EA8ECE8F0DF2ACCD718D822D865
:10F2B000DF6A060EDF5C07E2DF50DCECE5F0010EF2
:10F2C000EF6EDF2AF6D732ECF4F0FD0E016EDB0EA6
:10F2D000D5ECE8F0010E186EE552DEEFE4F0020E18
:10F2E0000A6E5A0EE66E000EE66E030EE66EA20E73
:10F2F0009CEFF4F0730EB1ECE8F069EC95F0140EAD
:10F3000021ECEFF0000EE66E0A0ED0ECE5F00A0EEE
:10F3100021ECEFF0CA0EE66E0A0ED0ECE5F00C0E12
:10F32000E66EE66A010EE66E140EE66E0A0ED0EC8C
:10F33000E5F00A0E21ECEFF0200EE66E0A0ED0EC9E
:10F34000E5F00A01D46BDA6BDA81D56B380ED66F33
:10F35000040ED86F3C0ED96F190ED76F016A020EDA
:10F36000015C0CE20150050D59ECF3F0000EE926AA
:10F370000A0EEA22360EEF6E012AF1D70C6A050E4C
:10F380000C5C1AE20701010EE26FFF0EE25D12E073
:10F39000BDEC15F0C2ECECF09AECF1F00C506EEC18
:10F3A000F1F00701E25113ECF4F09AECE7F00701F9
:10F3B000E207EBD70C2AE3D70701E26B0C6A1AECE1
:10F3C0005FF023EC5FF0030E0A6EFE0E016E810EFD
:10F3D000D5ECE8F00A6A1200240E01013F03F35055
:10F3E000E66EE66A14ECFBF0E552E552010141518C
:10F3F000E8240A0FE66EE66A43ECFBF0E552E552BC
:10F400000C0EBD6E006A01013F510AE0020E40255C
:10F410003F03F3504A6E4B6AFF0E78ECF1F0006E3A
:10F420000050BE6E1200D9ECE4F07FECE5F040EC49
:10F43000FCF0E552000902E0C69EF7D7DEEFE4F0EB
:10F44000C79EC698C78C1200C78EC688C78C12008C
:10F4500099EC5EF02DA003D0210E77ECE5F00701CA
:10F460000B8799EC5EF099EC5EF099EC5EF0070189
:10F470000B972DB003D0270E77ECE5F099EC5EF0FA
:10F4800007010B8599EC5EF007010B952DA002D0CA
:10F490000101E38999EC5EF00701128599EC5EF0B9
:10F4A000070112952DB003D0330E77ECE5F099ECFF
:10F4B0005EF007010F8F99EC5EF007010F9F2DB0F2
:10F4C0000DD00F8B99EC5EF007010F9B2DA003D0A0
:10F4D0000101E38B03D0240E77ECE5F099EC5EF0AC
:10F4E00007011F8999EC5EF007011F9922882DB052
:10F4F00003D06C0E77ECE5F099EC5EF001012BA1E6
:10F500001FD00701108799EC5EF0070110972C843B
:10F510002DA004D0010178AB11D00DD0010178AB42
:10F520000AD00701108F99EC5EF00701109F0101CE
:10F53000E2812DB003D0630E77ECE5F099EC5EF03C
:10F5400001012BA70ED007010D8799EC5EF0070192
:10F550000D9720802DB003D02A0E77ECE5F099ECC2
:10F560005EF001013B510EE00701168199EC5EF05F
:10F57000070116912C862DB003D0660E77ECE5F0CE
:10F5800099EC5EF001013A510EE00701138F99ECFE
:10F590005EF00701139F2B8A2DB003D0690E77EC24
:10F5A000E5F099EC5EF0010138A73BD02588070112
:10F5B000078599EC5EF0070107952DB003D02D0E5D
:10F5C00077ECE5F00701068399EC5EF0070107830D
:10F5D00099EC5EF0070107930101E9932DB0E983EF
:10F5E00099EC5EF0010160A50ED00701098799EC46
:10F5F0005EF00701099731822DB003D0300E77EC11
:10F60000E5F099EC5EF00701208999EC5EF00701C6
:10F61000209931802DB003D06F0E77ECE5F099EC96
:10F620005EF099EF5EF095ECF1F0020EDB6A81EC92
:10F6300012F00F0EC16E040E070104270407040721
:10F64000040704078D8C219A34860201800E8A6F8C
:10F65000D2EC15F00601BA6B800EBB6F40EC0EF0D9
:10F660000A6AFB0E9CECE5F000C0F1F707010E6B97
:10F670000F6B126B206B20C71FF7470E186F18C750
:10F6800017F70201A069A1690701010E066F076B58
:10F6900099EC5EF099EC5EF00301310EE36F070127
:10F6A000090E326F32C731F732C730F732C72FF742
:10F6B000070E516F0301A00ED06F0F0ED16FE50E34
:10F6C000E66E1FECFCF0E552E66872ECFBF0E552EA
:10F6D000E668DCECFBF0E552E668BAECFBF0E552DC
:10F6E000050EE66E5EECFCF0E55285ECECF074DEA7
:10F6F000850EE66EFEECFBF0E5520201320E256F40
:10F70000000EA56EA26E9F6EA282D08EE66A040ED7
:10F71000E66E210EE66EABECFAF0CBECF3F0010EE8
:10F72000DB6A100E15ECE5F018E2D20E4A6EEE0E12
:10F730004B6E010E4C6E010EDBCF4DF053ECF4F02E
:10F74000E66E010EDB50EA6AC90FE96E060EEA2288
:10F75000E8ECE5F0010EDB2AE4D70101276B2791E5
:10F760008850010B01E0278127938850020B01E0AC
:10F77000278328918850200B01E028812893885006
:10F78000100B01E02883E987F28E0601526952C608
:10F7900050F613EC51F065EC98F00101A4ECF2F096
:10F7A0000601526B52C650F613EC51F0010E186E62
:10F7B000A3EC93F0AFEC93F0F6EC89F0060117811F
:10F7C000416941C640F6426B148A13801288128246
:10F7D000148614880A01380ED66F010ED76FC4EC58
:10F7E0001EF06CEC95F087ECE9F0166E380E165CA6
:10F7F00006E10101398987ECE9F00009FCE1C80E56
:10F8000052ECE6F00701D76B358E84ECF2F0E66E31
:10F8100053ECEAF0359E40EC0EF00A6AFCECEFF097
:10F82000DF50005C02E0180E09D0830E0A6EFCEC7B
:10F83000EFF00A6ADF50005C04E01B0E77ECE5F0A5
:10F8400033D0FD0E9CECE5F0DB0E005C03E13A0EDC
:10F85000165C05E181DC010E3EECE6F01ED0020EE6
:10F860009CECE5F000C02BF1370E9CECE5F000C0FD
:10F8700060F1110E9CECE5F000C03AF1120E9CEC28
:10F88000E5F000C03BF10F0E9CECE5F000C038F154
:10F890004F0E9CECE5F000C078F1B00E9CECE5F06A
:10F8A0000050800801E24BDC010E696EE66E60ECF0
:10F8B0003BF0E55280EC36F0E5C2E6FFBDECE7F048
:10F8C000696A9AECEBF080EC36F0E4C2E6FFBDEC3E
:10F8D000E7F0010138B711D0E66ACEEC18F0E55236
:10F8E000040E7FECEAF0010E52ECE6F0E66ACEEC94
:10F8F00018F0E552280E52ECE6F032880701580E57
:10F900008F6F020E906FBC69A5EC0DF0FEEC23F03A
:10F91000010138A707D026ECECF0FEEC23F0696A71
:10F92000A5EC0DF099EC5EF0F29EC0EC4EF00201F9
:10F93000006F000910E0C80E52ECE6F0C80E52EC61
:10F94000E6F0C0EC4EF00201006F000904E07E0E0C
:10F9500077ECE5F0358287EC98F00701F10512E0CD
:10F960000301010ED96FDB6B73DD0301DB5103E093
:10F97000C80E52ECE6F00301DB5104E0D92B040E73
:10F98000D95DF1E3D9C3DAF30301D96BF28E2A9E74
:10F990002BBA2A8E0101DD95FD0E926E0A0E64ECE3
:10F9A000E5F092688F0E3FECF4F010080AE20A0EC0
:10F9B00064ECE5F08F0E3FECF4F0100802E2010178
:10F9C000DD850601D9918850800B01E0D981D9935A
:10F9D0008850400B01E0D98367EC51F0208600018C
:10F9E000126A136A146A156A2D82800E086E176AED
:10F9F000229A700EE66EE66A290EE66E010E0FEC94
:10FA0000E5F0020E0A6E5A0EE66EA20EE66E000ECB
:10FA1000E66E030E0FECE5F0030E0A6E2A0EE66E9C
:10FA2000E66A000EE66E0A0E0FECE5F0AA0EE66E30
:10FA3000300EE66EA4ECF3F00FECE5F0FE0E4BECAE
:10FA4000F4F0810E005C01E055DC060EE66EF00E6F
:10FA50004BECF3F00FECE5F0040EE66EA00EE66E54
:10FA6000F00EE66E060E0FECE5F00601F05104080C
:10FA700001E2F06BF251010801E2F26B200EE66E3A
:10FA8000800EE66E910EE66E070E0FECE5F0060EA8
:10FA9000E66EEA0EE66E350EE66E050E0FECE5F04C
:10FAA000830E0A6EF90E9CECE5F000C086F20201AE
:10FAB0008651DA0802E2DA0E866FDF0E9CECE5F082
:10FAC0000101DD91720E005C01E1DD817E0E0A6EA6
:10FAD0000F0EE66EE66AED0EE66E020E0FECE5F036
:10FAE0000A6A020EDB5011E09EEC09F0BB0ED880D2
:10FAF0000F54200E105402E2010178890F0E9EEC83
:10FB0000EEF003E20101040E446F01017897E385F2
:10FB1000530E3AECE9F0001C810B05E0BA0EC95C0B
:10FB200002E1010178870101E3950301DC69D1EC71
:10FB30000DF001018EBB3D9FFF0E0201FB5D02E156
:10FB40001E0EFB6FFF0EFA5D03E1800EF96FFA6B7C
:10FB5000FF0EF25D02E0F25102E1640EF26F01016C
:10FB600038A73C9978A702D0050E5C6F0501355186
:10FB700050080BE2280E386F38C535F5050E396F81
:10FB800039C536F53A6B3AC537F501018C510A088B
:10FB900001E28C6B180EE66EE0EC15F0E552000900
:10FBA00007E10301DA51010805E2040EDA5D02E221
:10FBB00085ECECF0ECEC79F046EC0AF0A3ECEEF01E
:10FBC0000101DD8395ECEEF0010178A703D003017C
:10FBD0000A0EE36FF9EC28F00401300EB76F010153
:10FBE00058AB03D00401310EB76F04013B0EBE6F5A
:10FBF0000501006B00C502F500C501F5800E056F1B
:10FC000007010C0E346FDD0E356F320EB16F7D6A59
:10FC10000C6AE26B5DECE9F00701EF81D2ECECF0ED
:10FC2000E4C2E6FFBDECE7F054EC24F0010138A794
:10FC30000ED026ECECF0E5C2E6FFBDECE7F054ECAC
:10FC400024F0D2ECECF001016385E3EC23F037EC17
:10FC500025F01A940101DF9F2BAD16D004EC27F09C
:10FC60000F5010100EE00F0E0F5C270E105809E217
:10FC70001A84680E0F1808E1105006E10101DF8FA9
:10FC800003D0600E77ECE5F01AB402D0010197952D
:10FC90000301B00ED26F0A0ED36FAD0ED46F120EE9
:10FCA000D56FFE0ED66F070ED76F0101DFAF0DD0F7
:10FCB0000301540ED26F070ED36F910ED46F0F0E47
:10FCC000D56F3E0ED66F080ED76F54EC05F0268028
:10FCD0002EECE7F07EEC28F01880CFEC2CF07AD9EF
:10FCE00069EC38F00201320E346F0101040EB36F7B
:10FCF000A30EB46FB3C10BF002016E2B320E326F44
:10FD0000E66A43EC90F0E55242ECC3F09CECC3F0A1
:10FD10005AECB5F00301DA51010814E2040EDA5D81
:10FD200011E272ECE7F0350EE66EF20EE66E010EB1
:10FD3000E66E90ECE6F0030E0301DA5D03E10101EB
:10FD4000330E1F6F030EE15C02E2E16AE552E16EE1
:10FD5000DEEFE4F09A0E0B5C03E30B509D0801E22A
:10FD6000000C010CE20E0B5C03E30B50E70801E210
:10FD7000000C010C01013C7B3CBB04803DEC0AF013
:10FD80000101289D076A120041ECEFF0ACECF1F0A4
:10FD90000101460E196F4C0E1A6F310E0A01D5255E
:10FDA00001011B6F96EC04F0B1ECF0F00050BFECD9
:10FDB000E8F004E14B5002E1A8ECEEF09FEC04F017
:10FDC000006E3A50DF6E82ECE9F001011F8F300EB9
:10FDD0001D5D07E11EC11DF11FC11EF1300EDF24A4
:10FDE0001F6FE552DEEFE4F00A01D651ACEFF4F0FC
:10FDF000D9ECE4F0016A012A0A01D52BD551040897
:10FE000001E2D56BB2ECECF00DE0050E015C0AE20C
:10FE1000ADECEEF004E0E846FE0BE706FCE107017E
:10FE2000E115E9E07DEC95F099EC5EF089ECEAF003
:10FE3000FE0EDB5002E0BDEC15F0E66AA8EC90F097
:10FE4000E552695002E0D5CAB1F282ECE6F01AE060
:10FE5000D8EC09F0000916E16F5014E1695048EC44
:10FE6000F0F0016E0150D5ECE5F00CE24A50380894
:10FE7000000E4B5407E2720EEAECE8F0FA0E096E3F
:10FE8000FE0EDB6AFE0EDB0403E17EDF640E096E0C
:10FE9000DEEFE4F00C50006E005003E0030E005C57
:10FEA0001BE1005005E10101CB7DCBAD0ED007D0A9
:10FEB00058ECE7F006E00101CB75CBA506D0048035
:10FEC00004D00101CA75CAB504803DEC0AF0B1EC5A
:10FED0004BF0E4EC1CF016D0000403E0020E005CD2
:10FEE00011E1BDEC15F0000402E1020E01D0010E9B
:10FEF000006E020E005C01E104803DEC0AF000504F
:10FF00000C6E27D839EFECF001013C51080B03E0EF
:10FF10008DECE5F002E0000E01D0010E1592E8B084
:10FF200015828DECE5F004E101013D51800B0CE1FF
:10FF30008DECE5F007E0F1ECE5F004E101013C5166
:10FF4000800B02E1000E01D0010E1590E8B0158083
:10FF500012000C50006E0050800802E2050E006E88
:10FF6000060E005C01E3006A000402E10101CA918F
:10FF7000020E005C02E10101CA8100500C6E258A6C
:10FF800021BE0CD045EC15F082ECE6F002E09CECD2
:10FF900005F0E4EC1CF04CEC05F002D0B1EC4BF0B9
:10FFA000B3EF2CF041ECEFF0030EDF6E01018FBDDB
:10FFB000DF6A4A514A6E4B6AB00E3E6E040E3F6EC7
:10FFC00089ECE5F03E50D880DF540201656FE552C0
:10FFD000DEEFE4F041ECEFF027B012D0320EDF6E2E
:10FFE00001018FAD02D0640EDF6E080E4A5D02E2A1
:10FFF000080E4A6FDF50D8804A5502E2DFCF4AF13F
:020000040001F9
:10000000D1DFE552DEEFE4F065C2ABF123AE3AD0CA
:10001000006A01013E510C0803E3050E3E5D02E259
:10002000090E3E6F050E3E5D4E6E4F6A0201655130
:10003000FDECE5F0140EB9ECE5F03EC04AF04A5094
:10004000006E1CECF1F00101AB514C6E4D6AFF0EDD
:10005000D8804C56000E4D564B504D18E8AE02D08D
:100060004D3404D04C504A5C4D504B580BE200507C
:10007000D880AB5507E224A003D00050AB2702D0B4
:100080000050AB5F1850080B08E102013D5106011A
:10009000F01106E02850400B03E11E9247EC50F0AF
:1000A0001200050EEAEFE8F0FCDF268E1200180EB3
:1000B00006ECE5F0268E1200D9ECE4F0050EE12600
:1000C00020A20FD0BAC1DFFF010EBBC1DBFF020EC1
:1000D000BCC1DBFF030EBDC1DBFF040EBEC1DBFFF5
:1000E0000ED0B5C1DFFF010EB6C1DBFF020EB7C1F6
:1000F000DBFF030EB8C1DBFF040EB9C1DBFF5CEC14
:10010000E6F01BE00101DFBD07D0DF50180815E263
:100110001C0EDF5C12E245D0190EDF5C42E01A0EC5
:10012000DF5C04E1010EDB505F083BE31B0EDF5C8C
:1001300004E1290E15ECE5F034E32C50100B14E12A
:10014000070EDF5C0EE1010EDB50360803E25CECCB
:10015000E6F027E1010EDB50400803E25CECE6F03C
:1001600020E0080EDF5C1DE02C50100B06E12F5044
:10017000800B03E0EDECE8F002E2F36A17D0790EB1
:10018000E66E020EE66EF1ECEDF0E2ECE7F009E16E
:10019000F1ECEDF0740EE66E020EE66EE2ECE7F0C6
:1001A00004E085DF010EF36E01D0F36AF46A050EF8
:1001B000E15C02E2E16AE552E16EDEEFE4F065C384
:1001C00001F023A802D075C301F00E0E015C01E21C
:1001D000010C100E015C01E2020C120E015C01E246
:1001E000030C140E015C01E2040C160E015C01E22A
:1001F000050C1B0E015C01E2060C220E015C01E203
:10020000070C080C35B603D0B0ECEFF017D0A70EF2
:10021000FAECF1F0016A006A0050D880015402E261
:100220000150006E4DECFDF048ECFDF00009FCE1E2
:10023000C450016E0050D8800154EEE32CA802D0C7
:10024000005010D00050020802E2020E005E460E7E
:10025000005C0BE2BA0E4A6EED0E4B6E010E5CECCA
:10026000F0F0F5500F6E106A12000050020D69EFA9
:10027000E5F0F00E8C16049035B8048054ECE7F0ED
:1002800006E12350100B03E0010E64ECE5F0BADF49
:100290000FC061F310C062F335B81200F00E8C1677
:1002A000030E8C1214A637D0CFC101F023B885D924
:1002B000050E01244A6E0A0EAFECE6F03F50016EC7
:1002C000015005E12350400B02E0010E016E8DEC60
:1002D000E5F003E03550400B05E001C0D5F7020121
:1002E0000A0E08D00701D551015C05E301C0D5F71E
:1002F00002010C0E3A6F63DF0701D66F2C50100B12
:1003000004E135EC0FF0000902E00701D66B5EEC6A
:10031000EAF093ECE8F06EECE7F00480005009E0BE
:100320003550400B06E1030E005C04E1020E785CE0
:1003300001E10490070E016E3250010B03E10450FD
:10034000010B04E0CD0E3DECE7F0016E0F0E011441
:100350000201886F32B002D0070E881701380F0BE8
:10036000016E04A0016A14A408D0020EE66E88C2D1
:10037000E6FF0150E66E93ECE8F02CA80AD00101EC
:100380004B510F6E106AE10ED8800F56000E1056BA
:1003900017D00FECEFF00CE25E510F6E106A770E83
:1003A000D8800F56010E105634ECEEF0FDE108D067
:1003B00053510F6E106A430ED8800F56010E10561F
:1003C000006A0301FF0ED8806155000E625501E2FC
:1003D000002A005061C34CF062C34DF005E0D89094
:1003E0004D324C32E804FBE161C33EF062C33FF0A2
:1003F000B5ECF1F0ABECF2F0B4ECF0F00FC043F080
:1004000010C044F0C9ECEFF00050E85003E034ECC9
:10041000EEF0FDE10FC0CFF1FA0E57ECE6F003E28B
:100420000101FA0ECF6F310E0101CF5D03E0330EF3
:10043000CF5D02E1320ECF6F630ECF5D03E0650E3C
:10044000CF5D02E1640ECF6F6EECE7F0040E005C4E
:1004500023E1100E016E01504A6E4B6AE8C23EF075
:10046000E9C23FF089ECE5F03EC0EAF20101CF516C
:100470006AECE7F00201E8274B50E923EA514A6EA3
:100480004B6AE8514A5CE9514B5806E2EA516AEC82
:10049000E7F0E85F4B50E95B000406E0020E005C09
:1004A00003E0030E005C08E10201EB510101D8807A
:1004B000CF5502E2CFC1EBF254ECE7F006E1235056
:1004C000100B03E0010E64ECE5F09CDE0FC063F35B
:1004D00010C064F3F00E8C1603016C0ED8806355C7
:1004E000000E645517E25CECE6F014E02E0EE66EAA
:1004F000F20EE66E010E93ECEDF00201640E2D6F2C
:1005000097ECEDF003E027ECF2F0FDE1AEECEBF060
:10051000E7EC0BF003016151635D6251645906E33E
:10052000010E6325616F000E6421626F61516325C6
:10053000676F62516421686F675167254A6E685121
:1005400068214B6E67C34CF068C34DF0030EEBECB3
:10055000EEF0E804FCE14A504C240301676F4B5075
:100560004D20686F6351615D4A6E625164554B6EF8
:10057000A1ECEFF067C33EF068C33FF0EBECFCF09A
:100580003EC067F33FC068F367C365F367C34AF0D3
:1005900068C34BF04C6A4D6A4D34000E4D1809E6A5
:1005A000D880FF0E4A54000E4B54000E4C54000EDF
:1005B0004D5402E203016569120049C101F02C505B
:1005C000100B0BE10FECEFF008E26C0E015C016E1A
:1005D0000A0E2C5D02E1040E015E1200CDECF0F07B
:1005E00007E03550400B04E1050E005C01E0000C13
:1005F000010C0482F3DF000901E00492358604A2B5
:100600003596359836DE35B812006EECE7F0049A70
:1006100004980496030E005C01E10486000403E0E4
:10062000020E005C01E104882350400B01E109D176
:100630002350100B01E005D13450080B01E101D12A
:1006400002012D5101E0FDD01A50010B01E1F9D05A
:1006500004820494C3DF000901E00492040E005CEC
:1006600001E10484AADF0150FC0BE842E842026E7B
:1006700032A01CD00201885107080AE20150E8406C
:10068000E840E8401F0B015C525D09E2522B07D0A5
:10069000445105E1525103E05207040E446F525198
:1006A000D880015405E25251015E02D00201526B22
:1006B00004900450040B03E00250EA5D07E3045089
:1006C000040B70E101500101CF5D6CE20101320EBB
:1006D000076F0A0E2C5D02E1040E07270201BA51D2
:1006E000105D02E3000E01D0010E049CE8B0048C02
:1006F000480E0F5D710E105901E394D003016C0E8A
:10070000635D000E645901E38DD05CECE6F00CE013
:100710002150800B05E06C0E01010725495D04E0C6
:100720000450400B01E17ED004B20BD00101CF5147
:10073000015C020D69ECE5F00F5002010F2710502B
:1007400005D004A405D002010F2B000E102369D0A0
:1007500002012E5167E10A0E2E6F0150EB5D20E27F
:10076000EB511EE004A802D0020E2E6F0450080BBD
:1007700012E0030E785C06E0020E785C03E088511C
:10078000010809E2320E0F27000E10232F5107E057
:100790002E912E4304D00A0E0F27000E1023048042
:1007A000EB6B40D00450040B05E002500201D880EE
:1007B000EA5508E30450040B35E101500101D880EB
:1007C000CF5530E2020E036E04A402D0010E07D012
:1007D00004A206D0320E036E04A802D0960E036E59
:1007E00003500F6E106A0450020B06E00450080B11
:1007F0000EE002012F510BE001500101CF5D4A6E66
:100800004B6AA1ECEFF0E8ECF3F0B2ECF2F002018D
:100810000F510F5C1051105805E20F500F5F105030
:10082000105B048004A00DD0020111510F1902E1E8
:100830001251101906E0E7EC0BF00FC211F210C2D2
:1008400012F20201305102E00F0E306F1200175009
:10085000100B0CE03A0E675C3EE0170E675C3BE065
:100860002A0E675C03E1E7ECEEF035E01750010B70
:1008700006E0190E675C2FE02D0E675C2CE0350E4C
:10088000675C29E0250E675C26E00E0E675C23E0BE
:10089000080E675C20E0390E675C1DE0380E675C6F
:1008A0001AE0400E671417E170ECB5F0000913E18F
:1008B000090E675C07E11750100B04E0D7EC1DF040
:1008C000000909E12150800B05E16F5003E033502E
:1008D000200B01E0000C010C020EDBECEBF0909C15
:1008E000460E33ECE7F0908E010EE66E01ECFDF063
:1008F000E552FCEC1DF0F1ECE5F003E0720EF1ECDA
:10090000E4F0F6EC18F006015091120071C249F1C2
:1009100072C20FF273C210F2E7EC0BF07EEF28F018
:100920000101AB5103E12C82A7C108F02150010B5A
:1009300012E08DECE5F00FE11750800B03E03DEC89
:10094000ECF006E02150040B06E18150010B03E0BE
:1009500097D968EC8CF012000101050EAA6F2150A6
:10096000010B05E01A50020B02E0AA6B120034BE24
:1009700013D05CC100F00A0E2C5D05E17851080B24
:1009800002E10A0E002602010E51D880005404E252
:100990000E51005C0101AA6F1200BAECF1F00101E6
:1009A000DF9982ECE6F002E00101DF892550020BBD
:1009B00004E11D50010B01E0238C23BC06D0E66A44
:1009C000E66AC80E0AECE5F010D0E7ECEEF00BE1B9
:1009D0003450080B08E097ECEDF003E027ECF2F060
:1009E000FDE1AEECEBF0E7EC0BF002010A0E2E6F2E
:1009F000EB6B21AE1D84C80E2F6FEFEC18F0780E54
:100A0000006E005033ECE7F08FEC1DF00201326B0A
:100A10008DECE5F003E03550400B07E082EC0BF085
:100A2000000903E00D0E4AECE7F02150800B06E1CF
:100A3000F1ECE5F003E0730EF1ECE4F0909E349EEF
:100A4000F8ECEAF001E0348ED5ECF3F03EE12C5006
:100A5000080B30E02350100B2DE101013B052AE08B
:100A600016C2DFFF22ECC6F0DF500201165D22E065
:100A7000010E69C3DBFF020E6AC3DBFF030E6BC30B
:100A8000DBFF010EE66ECCECC6F0E552010EDB504A
:100A90000301695D08E1020EDB506A5D04E1030EAB
:100AA000DB506B5D07E08DECC5F099EC5EF01D82CC
:100AB000960E096E3450800B08E0F0ECEAF005E188
:100AC000D5ECF3F002E12AEC0BF02150800B19E198
:100AD0002150010B16E18DECE5F009E03550400B9B
:100AE00006E102013D510DE0050100510AE101015D
:100AF000DF9BF0ECEAF003E00101DF8B02D037EC82
:100B0000E9F01EAC02D0EEEC0BF0218C328234AE58
:100B100002D0909E6ED0D5CAB0F26EECE7F0360EE1
:100B2000026E380E036E005003E03550400B03E0B8
:100B30004FC1D5FA12D0A1EC0BF0000904E085C139
:100B4000D5FA03680AD0050E005C05E10A01D56BF1
:100B50000368026802D056C1D5FA0A01D5519EEC4D
:100B6000EDF0016E0250015C04E30350D8800154A3
:100B700003E2750E77ECE5F0B5EC5DF00101DFB94D
:100B80001AD0B5C193F2B9ECF2F03FC094F2F0EC98
:100B900038F0B5C191F2B9ECF2F03FC092F220A268
:100BA0000AD0BAC191F27CECE5F0BBC13FF02FEC6A
:100BB000FDF03FC092F2909E0101DFB91AD020A251
:100BC00003D00701576B586B02019351915D0EE101
:100BD0009451925D0AE054ECE7F008E10201942997
:100BE000925D03E09405925D01E12A84308ECEECA3
:100BF0003EF0320E33ECE7F0908C9BEC0FF00701E7
:100C00001B991B9701013CA904D007011C6B1CC751
:100C10001BF788ECEBF00201FA0E336F248A268270
:100C2000329223AC02D0060150813EEC4BF002011F
:100C3000295109E00101DF51080B05E1140E58ECC0
:100C4000E5F00101DF87040EE15C02E2E16AE552B2
:100C5000E16EDEEFE4F041ECEFF005011107125117
:100C6000EA6A150FE96E050EEA22EFCFDFFF122BBD
:100C700012511F0801E2126BDF50E552DEEFE4F083
:100C800051EC29F002012A6B2AC26AF2EDECEBF07A
:100C900007E0200E01011F5D03E0200E43ECE6F0AB
:100CA0000101AB6B006A37EF91F041ECEFF00850B7
:100CB000DF6E02011E0E316F0501005102012A1183
:100CC0000BE01E50040B06E01E50080B03E08150A1
:100CD000080B02E1D5DF76D308503AE1345101E048
:100CE00071D30101E99521B002D057DE0ED08DEC11
:100CF000E5F006E002013D5108E00501005105E183
:100D0000F0ECEAF002E137ECE9F0E7ECEEF014E1A8
:100D10000201B4A50FD0330EB25D09E10101DEAFCF
:100D20000BD002EC05F00201330E4D6F05D002EC42
:100D300005F002D007EC05F00101DFA902D0AA6B93
:100D400037D10ADE050E01018703F350AA2730D1FF
:100D5000080430E10101AA5101E030D3209CD5EC18
:100D6000F3F002E0208C0FD03450800B0CE1F0EC5B
:100D7000EAF009E12AEC0BF00101DFAB02D037EC1D
:100D8000E9F00101DF9B2E50200B03E12050020B04
:100D900004E0E4C2E6FF67ECE9F00101280EAA6F67
:100DA00023A802D0AA9FAA4721AE02D0050EAB6F9E
:100DB000082A0AD0020E085C09E10101AA5102E1E9
:100DC000F9EC82F034EC0BF0ABDDF8D2030E085CEA
:100DD00042E12CA226D05CC1AAF154ECE7F005E177
:100DE0007851080B02E10A0EAA27DFB9AA6BAB51B2
:100DF00004E0050E8703F350AA272C922150010B23
:100E000004E01A50020B01E0AA6B8DECE5F006E05D
:100E100002013D5103E13550400B03E0006A37EC1D
:100E200091F00101AA5106E08DECE5F00FE035509C
:100E3000400B0CE12050400B05E102013D5102E165
:100E40002FEC0BF00101280EAA6F40D127B8B6D2C3
:100E5000F9EC82F0B3D2050E085C68E10101AA51F9
:100E600001E0ACD2082A279821B059D01C0E016E9F
:100E7000DFA902D0140E016E8751E8240124006E10
:100E800002018C5107E000508C5D04E2090E086EEF
:100E9000278845D03282909C219C34BE10D0B0C2AD
:100EA000D5FAB5EC5DF00101DFB909D0F0EC38F00E
:100EB00020A203D00701576B586BCEEC3EF0070120
:100EC0001D990101E3A102D007011D8907011D97AA
:100ED0000101E3B102D007011D8707011B99010140
:100EE000E3A302D007011B8907011B970101E3B3AC
:100EF00002D007011B8701013CA905D0B1C2E6FF62
:100F000097EC5DF0E55288ECEBF08DECE5F003E05A
:100F10003550400B03E00101050EAA6F329201012A
:100F2000DFA902D0AA6B4AD217DD48D2060E085CB0
:100F300041E10101AA5101E041D221B037D027504F
:100F4000100B19E13C51080B12E1335110E0E9514B
:100F5000040B0DE18DECE5F003E03550400B07E0AC
:100F600001013D51800B03E0E951800B04E00101D8
:100F7000E99FB2DC11D033C132F227A80DD0BDEC0D
:100F8000F4F087C13FF0D1ECF0F0006E00500201A8
:100F9000325D02E200C032F22E50200B03E12050FD
:100FA000020B04E0E4C2E6FF67ECE9F002016B6BC0
:100FB000082A04D2070E085C2EE10101AB5119E1A9
:100FC00017AE15D03DECECF003E036ECB6F00FD0E8
:100FD000B2EC0BF0000904E10101E951040B07E058
:100FE000100E675C03E10101E98101D0179EA7C1E2
:100FF00008F002013D5101E0E1D13A5106E03550DF
:10100000400B03E15EECEAF003D0E66AE66AE66ACA
:10101000A0EC30F037D0080E085C4AE10101AB517A
:1010200006E01E50040B03E01E50080B02E1A7C1AE
:1010300008F002013D5101E1C1D1F9EC82F034EC3C
:101040000BF002013E5101E0B9D18AEC0FF000092A
:1010500001E1B4D10501020E146F115115E0FBDD61
:10106000006E020E785C18E0016A0501115102E081
:10107000F2DD016E0050E66E0150E66EE70EE66EA0
:1010800055EC18F0E5520ED000510FE1006A020E47
:10109000785C02E1030E006E0050E66EE60EE66E2E
:1010A00051EC18F0E552E55289D102013D6B86D131
:1010B000090E085C2BE10101AC417F0BAC25D88007
:1010C000AC5506E202018C6B8CC2ACF1050E75D1F9
:1010D00081B674D1010EAC6F320EAA6FDFA902D0B7
:1010E000280EAA6F010E086E8DECE5F006E00201F5
:1010F0003D5103E13550400B05E0F0ECEAF002E130
:1011000037ECE9F001010B0EA76F58D10A0E085C0D
:1011100006E122BA9ED0179E0B0E086E9CD00B0ED5
:10112000085C01E09BD01750800B3CE12150010B83
:1011300006E02150040B03E18150010B33E18DECFB
:10114000E5F003E03550400B0CE02150800B09E145
:101150008150080B06E01E50040B03E01E50080BE4
:1011600021E18DECE5F00CE03550400B09E1215018
:10117000040B06E18150010B03E0B6ECECF012E049
:101180002150800B0CE08150080B0CE01E50040B2A
:1011900009E01E50080B06E08150010B03E0D5EC7E
:1011A000F3F04DE017AE18D03DECECF005E036EC76
:1011B000B6F0000911E106D1B2EC0BF0000904E130
:1011C0000101E951040B08E0100E675C03E1010125
:1011D000E98102D0179EF6D08DECE5F014E0355091
:1011E000400B11E1F1ECE5F00EE11AAA04D0A4ECF9
:1011F0000AF0DBEC22F00101895105E089C1E6FF2C
:1012000034EC29F0E552ACC18CF20101AC5102E0A2
:10121000010EAC6F27A802D0F9EC82F00701D36B66
:10122000030E086E0101800EA76F2150800B03E1B1
:101230001750800B08E021940C0EA76F04D023A850
:1012400002D086ECC7F00101AA5105E12750100B2E
:1012500002E1F9EC82F034EC0BF0B0D00C0E085C3B
:1012600001E0ACD022BAAAD0BFECB8F021AEA4D035
:101270001E50040BFDE01E50080BFAE08150080BD5
:10128000F7E02B84189A248A189826820101995134
:101290000CE020A203D099C17DFF02D099C10CF0CF
:1012A000F0EC38F0198CA9EC7FF023A803D086EC81
:1012B00084F06ED0320E026E54ECE7F002E1040EC0
:1012C0000226140E0301655D5EE22C50100B04E053
:1012D000640E0101495D0BE02C50100B54E1320EFD
:1012E0000101495D04E06C0E0224495D4CE120ECF3
:1012F00015F010C200F000504C6E4D6A0050F5EC35
:10130000E5F049C100F05CECE6F004E06C0E010190
:10131000495D006E1CECF1F0A1ECEFF09FECE5F004
:10132000000E57ECE6F02CE27D0E13ECEFF028E215
:101330000F50D5ECE8F05CECE6F025E00201710E10
:10134000BA6F030E38ECF0F0BAC23FF0D1ECF0F017
:10135000006E00500201D880105504E3030E100304
:10136000F3CFBAF2100E01012C03F350056E680E94
:101370000A6E54ECEDF0055032ECF0F00A6A03D03E
:10138000780E77ECE5F019A803D086EC84F0199874
:10139000219E82ECE6F003E0B1EC4BF005D0010EAB
:1013A000E66E5EEC4BF0E552239876ECE9F0010135
:1013B00037BF02D092ECEEF0800E086EDF50085C72
:1013C00001E01D8CE552DEEFE4F03050100B0CE133
:1013D0000701825109E125ECEFF007E0020E6F5C96
:1013E00004E00201DF5101E1000C010C070EE66E82
:1013F000E66A200EE66E440EE66E060EB4EFEBF0E3
:1014000045C644F646C645F647C646F648C647F6BC
:1014100049C648F64AC649F6120049C64AF648C6C1
:1014200049F647C648F646C647F645C646F644C698
:1014300045F60601200E446F1200D9ECE4F00101DC
:10144000E551E61103E00D0ED4ECE7F0E751E811A9
:1014500003E00A0ED4ECE7F032AA02D0E1ECEFF0A0
:101460000101DF51020B0CE0280E0901BD5D08E20D
:10147000BD51BD2BEA6A950FE96E090E00ECF3F041
:10148000DEEFE4F01CECF3F01B50010B0AE0800EE1
:1014900048ECE5F004E2FE0EDB50200802E11B9070
:1014A0005CD0AEDFFE0EDBCF4AF6DB50800804E0F6
:1014B000850E48ECE5F003E30601200E21D0FE0E78
:1014C000DB50300803E10601630E1AD02A50200BCE
:1014D0001CE02950080B19E1DF6A150EDF5C15E2EC
:1014E0008BECF2F00FE1DE52010EDD6EDF2AE9EC4B
:1014F000E7F006014A6F84DFDF2AE9ECE7F0060136
:101500004A6F03D0030EDF26E8D7020E6F5C12E0AD
:10151000010EDB5004E049C6E6FF8FDFE5524AC604
:1015200000F0630E005C02E1300E006E0050E66ECB
:1015300084DFE5524ADF000910E072ECE7F044C6B0
:1015400019F145C61AF146C61BF147C61CF148C63B
:101550001DF149C61EF14AC61FF1020EE15C02E20E
:10156000E16AE552E16EDEEFE4F041ECEFF00850A5
:10157000DF6E2492100E085C13E11C0E086E02014F
:101580006651010B03E11E50040B02E1110E92D0D3
:101590006651040B29E11E50080B01E0ABD024D0AA
:1015A000110E085C0AE12480238E0201080E666F8A
:1015B0002482086A0101120E9CD0120E085C07E119
:1015C00024902482030E086E0101130E92D0130E94
:1015D000085C0CE11C0E086E02016651040B04E16C
:1015E0001E50080B01E086D0140E64D0140E085C67
:1015F00011E12480238E180E086E1E50040B01E0AA
:1016000079D01E50080B01E075D02482086A0101D0
:10161000150E6FD0150E085C0BE101012BAF03D046
:101620000201020E666F239E2AECECF0160E61D0CA
:10163000160E085C04E12AECECF0170E5AD0180ED6
:10164000085C08E10201020E666F2482086A01014B
:10165000190E4FD0190E085C05E1239E2AECECF020
:101660001A0E47D01A0E085C04E12AECECF01B0EAF
:1016700040D0170E085C08E101012BBF03D0020126
:10168000020E666F1B0E16D01B0E085C05E124903F
:10169000238E2482030E2AD01C0E085C2BE124909A
:1016A000800E086E02016651010B03E11E50040B0F
:1016B00003E1110E086E1ED035AC03D078ECF4F0C7
:1016C00019D01750800B16E11850080B03E0090ED3
:1016D000685D0AE30601F05104E0080E0201685D4E
:1016E00003E302013D5106E02482080E086E010169
:1016F000100EA76F24A202D004EC80F0DF50085C2B
:1017000001E01D8CE552DEEFE4F04CECEFF001015E
:101710003CB902D01D9601D01D761D50080B01E08A
:10172000010E696E5751400B18E0D8EC09F005081E
:1017300014E00201325111E133510FE134510DE156
:10174000800E08140AE02D50080B07E11E50400BD4
:1017500004E12550010B01E102D854EFEFF095ECC4
:10176000F1F0D4C7DFFF020EDB6A35A003D0010E13
:101770003EECE6F0010E79C1DBFF1DA615D0020E8E
:10178000DB6A1DA803D0010E3EECE6F001018BBD23
:101790000BD0010E7AC1DBFF8D0E3DECE7F0006E41
:1017A00003EC34F00050DF6EAEECEAF003E2010E21
:1017B00005C7DBFF010EDB50DF5C0EE3020EDB50E2
:1017C00003E04E0EF1ECE4F0020EDB6A0201FA0EC9
:1017D000336F28A80CD009D0020EDB5002E122ECB6
:1017E00009F0010E3EECE6F002010A0E336F1DA671
:1017F00006D01D98020EDB5007E01D8805D03590FD
:10180000020EDB5001E03580030EE15C02E2E16A8A
:10181000E552E16EDEEFE4F002016B6BE66AE66A28
:10182000E66A93ECE8F002013A6B0701D56BD5C785
:10183000CFF121B003D02180CDEC84F0120041EC37
:10184000EFF00201050E3D6F280E3E6FE5DF020E40
:10185000785C08E1DF6A010197A102D0060EDF6E15
:1018600069ECF1F00501040E146FE552DEEFE4F0CF
:10187000358C210EA8EFF0F00101DD51020B13E0D1
:101880003D51800B10E12150010B0DE12150100B57
:101890000AE12550020B07E1DD933088190E06ECB2
:1018A000E5F0AA0E096E120001013D51800B04E122
:1018B0002150010B01E1000C010C01015751800B7B
:1018C00005E0020E005C03E0000401E0000C010CE6
:1018D00041ECEFF062EC11F0000909E0030EDF6E5D
:1018E000010197A102D0070EDF6E69ECF1F0020151
:1018F000325102E0010E326F198C0701D36B219037
:1019000021947CECE9F0E552DEEFE4F081B003D005
:101910001B0E06EFE5F081B603D01A0E06ECE5F0DB
:101920001200085009ECECF030E14B502EE11A9215
:101930000101DFA503D0DF951FEC1EF00101DF518F
:10194000080B08E02150400B05E1120E58ECE5F0C1
:101950000101DF9735AC02D078ECF4F021B00BD068
:1019600062EC11F0000903E0006A37EC91F0229676
:101970006F5001E1208622AE06D0010EE66EEAEC41
:101980000AF0E552229E082A120008507AECEAF08A
:1019900001E0CAD14B5001E0C7D121A0239C19EC32
:1019A00016F0FF0801E0F4D02E50400B01E0F0D01B
:1019B0002150200B01E1ECD01950800B01E0E8D060
:1019C0002850010B01E0E4D00101E951010B01E0D5
:1019D000DFD002018C6B8CC2ACF11A926EECE7F096
:1019E000359C1D908150080B18E1005006E02050F6
:1019F000020B13E162DF000910E00101010EAC6F80
:101A00001A82086A0B0EA76F005003E14DDF000930
:101A100001E01D80005033E134D01E50040B03E080
:101A20001E50080B30E1005013E02050020B03E180
:101A300044DF00090DE10601F25125E062EC11F0EE
:101A4000000906E12050020B1EE1F1ECE5F01BE07D
:101A50001EB402D0110E05D01EB604D00201666B72
:101A6000140E086E005003E11FDF000901E01D8025
:101A7000005007E0030E0C5C02E1E1DE89D0F8DEE5
:101A800087D0FADE85D0050100511CE0005003E04C
:101A9000F1ECE5F010E0005003E106DF000901E0A1
:101AA0001D80005001E1E8DEF1ECE5F001E0C7DE69
:101AB0001E0E086E6DD0268E810EEAECE8F049EC21
:101AC00029F066D021AE04D0086A01010A0E47D081
:101AD000005048E08150010B06E02150040B03E167
:101AE000B6ECECF03FE002012A5114E0B6ECECF069
:101AF00007E128EC09F000090DE18150010B0AE132
:101B000002014A6B4B6B2A6B2AC26AF2A4EC0AF000
:101B100051EC80F0D5ECF3F007E08150010BFDE0D3
:101B2000B6ECECF0FAE130D01850080B0FE01A5088
:101B3000400B0CE0800EE66E030EE66E990E0AEC8A
:101B4000E5F0B2EC0AF09E0E29ECE7F002013A6BE8
:101B50003AC2D5F73AC2CFF1086A01010B0EA76F5E
:101B60001D8016D0005014E12150010B11E181506D
:101B7000010B03E02150040B0BE00101DD93D5ECD8
:101B8000F3F004E081A0FED7219412001D8044DE12
:101B90002150200B04E1C3EC0BF0000907E1020126
:101BA000475104E10101E951010B27E00501006BF8
:101BB00021902194810E086E0101E951010B02E090
:101BC0006F5007E1A3DEC3EC0BF0000902E009C08F
:101BD00047F221EC08F00101E9A10FD0B2EC0BF0C3
:101BE000000907E10101E9910201476B010E096E4D
:101BF00004D021AC02D07CECE9F008507AECEAF099
:101C000001E14B502FE093EC97F002013A6B30AAC0
:101C100002D0D9EC69F031A402D09CEC6CF031AC6C
:101C200002D032EC6BF025A002D04FEC6AF033A06A
:101C300002D094EC6AF024AE02D0E2EC68F020A866
:101C400002D0A0EC12F02D50800B03E12D50400B80
:101C500002E095EC0FF0269A1BAC02D03AEC0AF0A9
:101C60001D8C12002150010B18E002013D5115E1BD
:101C70001750800B06E03DECECF009E0250E675CA8
:101C800006E02150040B09E18150010B06E015A08C
:101C900002D00101E98F68EF8CF002013A5104E0B3
:101CA0005EECEAF093ECE8F017AE6ED036ECB6F0EE
:101CB00037ECE8F017E03050200B14E13150040B02
:101CC00011E12450800B0EE13150400B0BE1255007
:101CD000010B08E13350010B05E13350020B02E127
:101CE00069EC38F0339220AA4FD0209A01013CAB26
:101CF0004BD072ECE7F0020142510FE1BDEC43F032
:101D00000D0E675C10E11750010B0DE00C507D5C6F
:101D10000AE10201C80E426F1200426B1C0EBAECBF
:101D2000E8F0960E096E1200A9ECEBF02DE14B5095
:101D30002BE12250200B28E10101E151800B24E12D
:101D400009EC08F0000912E13CECF1F009EC33F089
:101D50000D0EF1ECE4F00C5002E03C0E01D01E0E32
:101D6000BFECF2F00101E29B4CEC05F053EC0EF0FD
:101D7000248A02011783810E086E09EC08F000091D
:101D800003E069EC38F0268212000D04040F07010D
:101D9000006F04A002D0040E00271200189A1AAC9B
:101DA00011D0A4EC0AF014820201DC0E4A6F050E79
:101DB0004B6F0101DFAF14D00201E80E4A6F030E32
:101DC0004B6F12000490010139B10480DEDF07017E
:101DD000FA0E036F016B026B0201686B696B1E9058
:101DE000120000C70AF002016A5104E0800EB2EC52
:101DF000EEF01B800701035117E0035103079CEC31
:101E0000E5F0CC0E005C10E0FF0E005C0DE0800EF3
:101E1000005C06E20050E66E67EC04F0E552006EEE
:101E20000050B2ECEEF0E6D70A6A1200F9ECF3F0DB
:101E3000DBCF6AF23088006A248859EC2EF0320E2B
:101E4000096E19AA02D002016A8F02012A5102E02A
:101E5000010E2A6F179EDEEFE4F045ECEFF019AAB1
:101E600002D011EC5FF01AAC57D0AF0EDE6E0A0E46
:101E7000DD6E0101DFAF04D0530EDE6E070EDD6EA6
:101E8000A4EC0AF01492B2EC0AF0049001018BB7B2
:101E900004807BDF00C70AF0FC0E9CECE5F000C07C
:101EA00010F01EECEFF000C00FF00A6ADECF4AF02F
:101EB000DDCF4BF00F504A5C10504B5806E3010148
:101EC000D2510F5CD351105805E254EC80F002015E
:101ED0002A6B28D01482800EE66E030EE66E980EF2
:101EE0000AECE5F00101E0831FEC1EF00101D25184
:101EF0000F5ED351105A9C0E29ECE7F076EC0AF0F5
:101F00001A8A28EC09F000090DE121840101DE990B
:101F100081A008D0DE8906D0288A02013D5102E066
:101F2000010E3D6F020EE15C02E2E16AE552E16EF4
:101F3000DEEFE4F0D9ECE4F01A8C8DECE5F003E090
:101F4000F1ECE5F001E01A9C1A50400B03E031EC93
